:020000020000FC
:0A0000000C9495040C9400000C947D
:10000A0000000C9400000C9400000C9400000C9466
:10001A0000000C94DB460C94E4460C9400000C940B
:10002A0000000C9400000C9468850C9400000C9459
:10003A0000000C9400000C941E360C9400000C94E2
:10004A0000000C9400000C9400000C946AC00C94FC
:10005A0098C00C9400000C9400000C94F2360C9496
:10006A0000000C9400000C9400000C9400000C9406
:10007A0000000C9400000C9400000C9400000C94F6
:10008A0000000C9400000C94000000000000010223
:10009A00030400060705010006FF050402FF09081C
:1000AA000CFF0AFF0F0E01060807050204030C0BDA
:1000BA00100A090D0F0E04060802030107050C10A9
:1000CA00090F0D0B0E0A01010101010101010101D4
:1000DA0001010101010101FF02FF04FFFFFF03FF0C
:1000EA0005FF06FF00FF436F4465496E466F00C96E
:1000FA0002100100000FAA558A617567203331206A
:10010A00323032362031303A33383A3039000067EB
:10011A0001016564000000010101020202030303F8
:10012A00040404050505060606070707414243417C
:10013A004243414243414243414243414243414295
:10014A004341424300000000EF006A0290080000A9
:10015A000000000000000000000000000000000095
:10016A000000000064002301C602D504820F0000CB
:10017A000000000000000000000000000000000075
:10018A0000000000F000F0005402D203F60900005B
:10019A000000000000000000000000000000000055
:1001AA00000000002A03C8032105E3064D100000E1
:1001BA000000000000000000000000000000000035
:1001CA00000000000E000208040A0C000000F00003
:1001DA00000043414E72783A20253033580A000015
:1001EA0043414E696E707574436E743D25752121C5
:1001FA00210A0043414E2D25753A20300A00434119
:10020A004E2D25753A20310A0043414E2D25753A67
:10021A002025750A0043414E2025750044656C610E
:10022A00792074696D6572202575000046616374D2
:10023A006F727944656661756C740A004850383487
:10024A003433004572724C6F67506F733D25752CBD
:10025A00204E6F3D25750A004572723A2025752099
:10026A0025750A002575204F66660A002575204FF8
:10027A006E0A00466C6173682074696D6572202588
:10028A0075004850383434330043666753756D3D02
:10029A00253034580A0020557064617465640A0078
:1002AA00485038343433207665722E2025752E2531
:1002BA00752E25752061756720333120323032362C
:1002CA002031303A33383A30390A0053657269615D
:1002DA006C3A2025750A00596561723A2032302538
:1002EA003032752C205765656B3A2025750A00480F
:1002FA0057207665723A2025632E25632C204F708D
:10030A0074696F6E733A20253032580A00436C6F55
:10031A00636B3A202530386C580A00436667436895
:10032A006B53756D3A202530345820004F4B0A0024
:10033A0020457272210A00436667566572457272D9
:10034A003A2025752028257529210A004545507629
:10035A0065724572723A2025752028257529210A69
:10036A0000526573746F7265436E743D257520255E
:10037A00752025750A00446174614572723D253005
:10038A00325820253032580A004850383434330A5B
:10039A0000004144436D696E4572726F725B257548
:1003AA005D3D25752121210A0000496E707574731F
:1003BA003A002025753D257500496E2D313A2025D4
:1003CA00750A00496E2D323A2025750A00496E2DAC
:1003DA00333A2025750A00496E2D343A2025750ACC
:1003EA0000496E2D25753A2025750A00496E412D62
:1003FA002575204F66663A2025755B6D565D0A00A5
:10040A00496E412D2575204F6E3A2025755B6D5634
:10041A005D0A0053776974636820257500416E612F
:10042A006C6F6720332E257500416E616C6F6720F3
:10043A00342E257500004B65795061643D00426C8D
:10044A00696E6B3A2530325820253032580A0047F7
:10045A0072617968696C6C2043414E6F70656E0AEF
:10046A00004772617968696C6C204A313333390A02
:10047A00004850393634320A004E6F6E650A000061
:10048A004B65795061642E436F6E6E2025750A00A4
:10049A004B65795061642E4469736F6E6E6E2025C8
:1004AA00750A00004F75745075736850756C6C3A14
:1004BA002025750A004F7574486967685369646531
:1004CA004F6E6C793A2025750A0043202532753A19
:1004DA00202534750043616C69627261746520007D
:1004EA004F4B0A006F75747075742025752066610C
:1004FA00696C65642121210A002532753A20253567
:10050A002E32665B415D0A002532753A204E6F2015
:10051A00666565646261636B2C204F75742D257561
:10052A000A002532753A20466565646261636B206C
:10053A006572726F722C204F75742D25750A004FE3
:10054A0075747075742074657374004261747420D4
:10055A0063616C696220203A20257500416E616CE6
:10056A006F672063616C69623A20333D25752C20E0
:10057A00343D25750043616C6962726174696F6EFE
:10058A004D61736B3A2025580A0020202532753AAE
:10059A002534752C2536752C2536752C2536752C63
:1005AA002536750042617474657279206661696CDA
:1005BA0065642121210A00416E616C6F67206661C2
:1005CA00696C65642121210A00206E6F7420636FB3
:1005DA006D706C657465642121210A004F7574522F
:1005EA0073744572725B25755D0A004F75742D250B
:1005FA00753A204F6E0A004F75742D25753A2053AF
:10060A0025752D3E25752C204F6E3D25752C2053C2
:10061A0065743D25750A004144433A002025753D1D
:10062A002575002020426174743D2575004C6F7752
:10063A00426174744F66663D2025750A004C6F77D7
:10064A00426174744F6E3D20257530300A00426154
:10065A007474657279536B697046423A20252E315B
:10066A00665B565D0A00426174746572794642207F
:10067A004F4B3A20252E31665B565D0A00202041F9
:10068A006E612D333D202575002020416E612D3489
:10069A003D202575004F75742D25753A2025750A5C
:1006AA00004F757420257520474E442D31210A00CC
:1006BA004F757420257520474E442D32210A004F6C
:1006CA007574202575206C696D6974210A004F754F
:1006DA0074412D25753A205325752D3E25752C20FC
:1006EA004F6E3D25752C205365743D25750A004FC4
:1006FA007574707574733A0A002534753A20464247
:10070A003D2575204144433D25752025755B6D4186
:10071A005D0A0052657365744572726F720A004F02
:10072A007574707574202575004F75742D25753A8A
:10073A00205325752C204F6E3D25752025632C20CE
:10074A002575305B6D415D0A00004F7574707574D4
:10075A002067726F757020257500506F7765724437
:10076A006F776E0A0057616B6555703A2025750AD6
:10077A0000004F7574412D25753A205325752D3E7D
:10078A0025752C204F6E3D25750A000043616C6962
:10079A00622E2073746172742025755B416D705DE1
:1007AA000A0054657374206F75740A0043616C699A
:1007BA00622E20626174740A0043616C696220616E
:1007CA006E6128352C3056207265662E290A004340
:1007DA00616C69623F006330006331006333006318
:1007EA0036006332300063620063610074657374BB
:1007FA006F75740050615373576F526421005057DC
:10080A003A2027257327200050573A204E6F6E65ED
:10081A002000204D6F64653D25750A004144433F21
:10082A0000496E7075743F004C6F61643F00485018
:10083A007374617475733F0052526573746F726595
:10084A00005252204F4B0A0052657365740053657B
:10085A00744F75742025753D2025750A00526573FD
:10086A006574206572726F720A004F7074696F6ED8
:10087A003A20253032580A0052657365740A0050CE
:10088A0043204F4B0A005043204F6C64210A00005A
:10089A005365712025633A20004F66660A00256376
:1008AA000A0053657175656E636520257500202001
:1008BA004F4B0A0020204661696C65642121210A98
:1008CA00000056696E2D25753A2025750A0056696D
:1008DA00727475616C202575000057697065723AEB
:1008EA00205325752D3E5325750A000001002D4E13
:1008FA00414E00494E4600002D4E414E0000010077
:10090A000200D60100000700BC03460200000700EF
:10091A00C3038C0200000100E10DF608000000008C
:10092A00F894EE27EFBBF1E0F5BFE5BFE093740062
:10093A00E09375008DE0A2E0BB27ED938A95E9F775
:10094A0080EF9FE0A0E0B1E0ED930197E9F7E8E0DE
:10095A00F9E0D0E0DBBF87919791009781F0A791EA
:10096A00B79107901790C791D791BF01DBB7F001F4
:10097A00CBBF07900D920197E1F7FB01EBCFE0E0C7
:10098A00EEBBEFEEEDBFE0E1EEBFCCEBD3E00C94B3
:10099A00CC330E9428D2AD014093D2035093D303A3
:1009AA00A5E2B1E00E941FD4E07111F0E1E001C0BC
:1009BA00E0E0AFECB3E0E170EE0F0E2EEC91ED7FCC
:1009CA00E029EC93A6E7B2E00E941FD4E093D1039A
:1009DA00A7E7B2E00E941FD4E0935C04A091D10380
:1009EA00A13010F0AD3008F004C0E091CF03E4600C
:1009FA0003C0E091CF03EB7FE093CF03E1E0E09304
:100A0A00D800FA01E436A0E0FA0741F4E2E1E09303
:100A1A00E200ECE0E093E300E7E335C0ED37A0E065
:100A2A00FA0741F4EEE0E093E200ECE0E093E30041
:100A3A00E7E329C0E83CA0E0FA0741F4E8E0E093E4
:100A4A00E200ECE0E093E300E7E31DC0EA3FA0E048
:100A5A00FA0741F4E6E0E093E200ECE0E093E30019
:100A6A00E7E311C0E43FA1E0FA0711F4E6E005C0AC
:100A7A00E83EA3E0FA0749F4E2E0E093E200E4E0AA
:100A8A00E093E300E3E1E093E40010E1103F88F42F
:100A9A001093ED002EEE30E0E8EFF0E02E173F075E
:100AAA0030F4D901E0E0EC932F5F3F4FF5CF105FB0
:100ABA00EDCFE091D800E260E093D80010E4103F57
:100ACA00A0F41093ED002EEE30E0E8EFF0E02E17E0
:100ADA003F0730F4D901E0E0EC932F5F3F4FF5CFA9
:100AEA00E8E8E093EF00105FEACF0E942FD2269643
:100AFA00089564970E9428D2E091D003E03009F467
:100B0A0014C2E17089F0E0E0E093ED00E091EE00BC
:100B1A00E17551F0E091D003EE7FE093D003E0E07D
:100B2A00E093EE00E093EF00E091D003E27089F0E9
:100B3A00E0E1E093ED00E091EE00E17551F0E09123
:100B4A00D003ED7FE093D003E0E0E093EE00E09382
:100B5A00EF00E091D003E47089F0E0E2E093ED0069
:100B6A00E091EE00E17551F0E091D003EB7FE09364
:100B7A00D003E0E0E093EE00E093EF00E091D003D1
:100B8A00E87089F0E0E3E093ED00E091EE00E175B2
:100B9A0051F0E091D003E77FE093D003E0E0E093E7
:100BAA00EE00E093EF00A091D003AF3009F4BDC18D
:100BBA00A0915604E0915704EA1709F4B6C1A4EDCE
:100BCA00B3E0E0915604F0E0BD01ADE0B0E00E9470
:100BDA00DDD2DB01AE0FBF1FEC91E071B1F041E055
:100BEA00A4EDB3E0E0915604F0E0BD01ADE0B0E061
:100BFA000E94DDD2DB01AE0FBF1F11960E949AD36D
:100C0A00EB8BFC8B6D8B7E8B13C040E0A4EDB3E0C5
:100C1A00E0915604F0E0BD01ADE0B0E00E94DDD203
:100C2A00DB01AE0FBF1F1196ED91FD91EF8BF88F8F
:100C3A00A4EDB3E0E0915604F0E0BD01ADE0B0E010
:100C4A000E94DDD2DB01AE0FBF1FEC91EF700E2FB9
:100C5A00098F403019F0E98DE061E98FE091D00306
:100C6A00E17009F051C0E0E0E093ED00E98DE09316
:100C7A00EF004030D1F0EB89EE0FEE0FEE0FE0936C
:100C8A00F000AB89BC89E5E00E9463D2E093F100F1
:100C9A00AB89BC898D899E89EDE00E948BD2E09355
:100CAA00F200E5E10E948BD20AC0EF89E295E07F6B
:100CBA00EE0FE093F200EF89F88D0E94B6D2E0932E
:100CCA00F30010E01017B0F4A4EDB3E0E09156047D
:100CDA00F0E0BD01ADE0B0E00E94DDD2DB01AE0F75
:100CEA00BF1F1596EE27A10FBE1FEC91E093FA00E5
:100CFA001F5FE8CFE98DE05CE093EF00E091D0035D
:100D0A00E160E093D00303C1E091D003E27009F0FF
:100D1A0051C0E0E1E093ED00E98DE093EF0040304F
:100D2A00D1F0EB89EE0FEE0FEE0FE093F000AB89F6
:100D3A00BC89E5E00E9463D2E093F100AB89BC89EB
:100D4A008D899E89EDE00E948BD2E093F200E5E165
:100D5A000E948BD20AC0EF89E295E07FEE0FE09302
:100D6A00F200EF89F88D0E94B6D2E093F30010E00A
:100D7A001017B0F4A4EDB3E0E0915604F0E0BD0121
:100D8A00ADE0B0E00E94DDD2DB01AE0FBF1F1596C9
:100D9A00EE27A10FBE1FEC91E093FA001F5FE8CF88
:100DAA00E98DE05CE093EF00E091D003E260E0932C
:100DBA00D003ADC0E091D003E47009F051C0E0E285
:100DCA00E093ED00E98DE093EF004030D1F0EB893C
:100DDA00EE0FEE0FEE0FE093F000AB89BC89E5E071
:100DEA000E9463D2E093F100AB89BC898D899E8908
:100DFA00EDE00E948BD2E093F200E5E10E948BD2F3
:100E0A000AC0EF89E295E07FEE0FE093F200EF89E6
:100E1A00F88D0E94B6D2E093F30010E01017B0F4F8
:100E2A00A4EDB3E0E0915604F0E0BD01ADE0B0E01E
:100E3A000E94DDD2DB01AE0FBF1F1596EE27A10F70
:100E4A00BE1FEC91E093FA001F5FE8CFE98DE05CEA
:100E5A00E093EF00E091D003E460E093D00357C041
:100E6A00E091D003E87009F051C0E0E3E093ED00AF
:100E7A00E98DE093EF004030D1F0EB89EE0FEE0FF1
:100E8A00EE0FE093F000AB89BC89E5E00E9463D2E3
:100E9A00E093F100AB89BC898D899E89EDE00E94BF
:100EAA008BD2E093F200E5E10E948BD20AC0EF896F
:100EBA00E295E07FEE0FE093F200EF89F88D0E9451
:100ECA00B6D2E093F30010E01017B0F4A4EDB3E04B
:100EDA00E0915604F0E0BD01ADE0B0E00E94DDD241
:100EEA00DB01AE0FBF1F1596EE27A10FBE1FEC91B7
:100EFA00E093FA001F5FE8CFE98DE05CE093EF0032
:100F0A00E091D003E860E093D00301C00EC0E09105
:100F1A005604EF5FE0935604E150A0915604AA30BC
:100F2A0018F0E0E0E093560443CEE0E05E2F2E2F67
:100F3A0030E4303F08F032C13093ED00E091EE002A
:100F4A00E07209F41EC1E091EF00EF700E2EEE81FF
:100F5A00E07FE029EE83EF70E93020F0EE81E07F58
:100F6A00E860EE83E091EF00E07109F46DC0E09172
:100F7A00F300FF2766277727EB8BFC8B6D8B7E8B25
:100F8A00AB89BC898D899E89E8E00E9474D2EB8B7B
:100F9A00FC8B6D8B7E8BE091F200AB89BC898D89CD
:100FAA009E89FF2766277727EA2BFB2B682B792B4D
:100FBA00EB8BFC8B6D8B7E8BAB89BC898D899E8973
:100FCA00E8E00E9474D2EB8BFC8B6D8B7E8BE091F8
:100FDA00F100AB89BC898D899E89FF27662777270F
:100FEA00EA2BFB2B682B792BEB8BFC8B6D8B7E8B87
:100FFA00AB89BC898D899E89E5E00E9474D2EB8B0E
:10100A00FC8B6D8B7E8BE091F000F0E00E94ADD2FC
:10101A00AB89BC898D899E896F2F660F660B762FE7
:10102A00EA2BFB2B682B792BEB8BFC8B6D8B7E8B46
:10103A00EE81E061EE83EB89FC896D897E89EF831D
:10104A00F88769877A871DC0E091F300F0E0EF8B9B
:10105A00F88F0E94A4D2EF8BF88FE091F200F0E0B3
:10106A00F595E7950E94ABD2AF89B88DEA2BFB2B99
:10107A00EF8BF88FEE81EF7EEE83EF89F88DEF83A9
:10108A00F88710E0EE81EF701E1758F4E12FF0E0B8
:10109A00DE011B96AE0FBF1FE091FA00EC931F5FB3
:1010AA00F1CF2F5FE091CF03E17081F0ECEDF1E039
:1010BA0060E070E00E94B1D3EB8DFC8D6627772744
:1010CA000E94B1D384E00E94AFD12896A091D103A7
:1010DA00A03069F0AF89B88D109749F4EE81EF70AE
:1010EA00E23028F0E091D103AC85EA1709F017C085
:1010FA00EB85F0E0E130A0E0FA0721F4E091CF03BC
:10110A00EB7F0BC0E230A0E0FA0721F0E038A0E064
:10111A00FA0729F4E091CF03E460E093CF03E0916A
:10112A00CF03E47069F5DE0116960E94901AE091E9
:10113A00AF09E27021F0DE0116960E949088E091D4
:10114A00BB07F0E0E130A0E0FA0729F4DE011696C9
:10115A000E948D4815C0E230A0E0FA0721F0E33082
:10116A00A0E0FA0729F4DE0116960E944E5808C03C
:10117A00E430A0E0FA0721F4DE0116960E943D60F1
:10118A0005C0E091EE00EE7039F05F5FE0E0E093B9
:10119A00EE00E0E8E093EF00305FCBCE222319F4B3
:1011AA00552309F462C0213020F1E091CE03E030EA
:1011BA0041F4E091F508E160E093F508E0E0E0939E
:1011CA00F208EEE1E093CE03E091CF03E27089F0FA
:1011DA00A2E3B1E00E941BD4FF70A7EABDE0FF7052
:1011EA000F01ED91FD91E070F07FE029F129FE9366
:1011FA00EE93A0915804B0915904A13FEFEFBE07B6
:10120A0040F4A0915A04B0915B04A13FEFEFBE07EE
:10121A0060F1E0915804F0915904F695E795E0934E
:10122A005804F0935904E0915A04F0915B04F6953E
:10123A00E795E0935A04F0935B04A0915804B091A7
:10124A005904E22FF0E0EA0FFB1FE0935804F093F1
:10125A005904A0915A04B0915B04E52FF0E0EA0F1B
:10126A00FB1FE0935A04F0935B040E942FD26A9604
:10127A000895BA93AA9324970E9428D2E091CF03A3
:10128A00E47009F07FC1E0916304E07821F0AA8557
:10129A00BB850E94901AAA85BB85EC91EF700E2F30
:1012AA00202FEC91E07151F031E0206111960E94FB
:1012BA009AD3EE83FF836887798706C030E0AA85D0
:1012CA00BB8511964D915C91E091D003E17009F0D4
:1012DA0047C0E0E0E093ED002093EF003030D1F01A
:1012EA00EE81EE0FEE0FEE0FE093F000AE81BF81BC
:1012FA00E5E00E9463D2E093F100AE81BF81888568
:10130A009985EDE00E948BD2E093F200E5E10E941C
:10131A008BD20CC0E0E0E093F000E42FE295E07F8E
:10132A00EE0FE093F200FA010E94B6D2E093F300C6
:10133A0010E0101758F4AA85BB851596EE27A10F61
:10134A00BE1FEC91E093FA001F5FF3CFE22FE05C3F
:10135A00E093EF00E091D003E160E093D00312C183
:10136A00E091D003E27009F047C0E0E1E093ED00BC
:10137A002093EF003030D1F0EE81EE0FEE0FEE0F3A
:10138A00E093F000AE81BF81E5E00E9463D2E09372
:10139A00F100AE81BF8188859985EDE00E948BD2EC
:1013AA00E093F200E5E10E948BD20CC0E0E0E0930A
:1013BA00F000E42FE295E07FEE0FE093F200FA01ED
:1013CA000E94B6D2E093F30010E0101758F4AA85F1
:1013DA00BB851596EE27A10FBE1FEC91E093FA008C
:1013EA001F5FF3CFE22FE05CE093EF00E091D003C0
:1013FA00E260E093D003C6C0E091D003E47009F044
:10140A0047C0E0E2E093ED002093EF003030D1F0E6
:10141A00EE81EE0FEE0FEE0FE093F000AE81BF818A
:10142A00E5E00E9463D2E093F100AE81BF81888536
:10143A009985EDE00E948BD2E093F200E5E10E94EB
:10144A008BD20CC0E0E0E093F000E42FE295E07F5D
:10145A00EE0FE093F200FA010E94B6D2E093F30095
:10146A0010E0101758F4AA85BB851596EE27A10F30
:10147A00BE1FEC91E093FA001F5FF3CFE22FE05C0E
:10148A00E093EF00E091D003E460E093D0037AC0E8
:10149A00E091D003E87009F047C0E0E3E093ED0083
:1014AA002093EF003030D1F0EE81EE0FEE0FEE0F09
:1014BA00E093F000AE81BF81E5E00E9463D2E09341
:1014CA00F100AE81BF8188859985EDE00E948BD2BB
:1014DA00E093F200E5E10E948BD20CC0E0E0E093D9
:1014EA00F000E42FE295E07FEE0FE093F200FA01BC
:1014FA000E94B6D2E093F30010E0101758F4AA85C0
:10150A00BB851596EE27A10FBE1FEC91E093FA005A
:10151A001F5FF3CFE22FE05CE093EF00E091D0038E
:10152A00E860E093D0032EC0E0915704EF5F1E2FCE
:10153A001A3008F010E0E0915604E11759F4EF5F11
:10154A00E0935604E150A0915604AA3018F0E0E066
:10155A00E0935604A4EDB3E0E0915704F0E0BD0136
:10156A00ADE0B0E00E94DDD2E60FF71FFA93EA93EE
:10157A00EC85FD85FA93EA93ADE0B0E00E9415CBC5
:10158A00109357040E942FD22C9608951A930A9307
:10159A008D011396ED91FD91A091D203B091D303E1
:1015AA00EA17FB0721F0F801A381B481F2D9E0918F
:1015BA00F508E07851F4E091F508E068E093F50861
:1015CA00E1E0E093F2080E946738F801E581EF70E4
:1015DA00E93018F4D80115964CDE0991199108954D
:1015EA00A091CE03A13078F0E091CE03E150E093D0
:1015FA00CE03E03041F4E091F508EE7FE093F50880
:10160A00E0E0E093F20808951A93A3E5B5E00E949A
:10161A001FD4E093C10D11E1163048F0A8E5B5E0FA
:10162A00EE27A10FBE1F0E941FD4E03009F002C0AE
:10163A001150F2CFE12FE550E093C20DE0E0E093C4
:10164A00C30DAAE6B5E00E941FD4E093C40DAFE92A
:10165A00B5E00E941FD4E093C50DA4EDB5E00E9449
:10166A001FD4E093C60DA9E1B6E00E941FD4E0930F
:10167A00C70DA091C70DA13019F4E2E0E093C70DA0
:10168A00E091C70DE093C80DAAE1B6E00E9417D415
:10169A00E093CA0DF093CB0D6093CC0D7093CD0DF2
:1016AA00EFEFE093C90DAEE1B6E00E941BD4E093E0
:1016BA00CE0DF093CF0D309719F4E0E0E093C80D0A
:1016CA00ABE3B1E00E9417D430976040704011F448
:1016DA00E0E00BC0AFE3B1E00E941FD4E093D00D6D
:1016EA00A091D00DA63018F0E5E0E093D00D10E0FF
:1016FA001330B0F5A2EDBDE0E12FF0E0EE0FFF1FD1
:10170A00EA0FFB1F3196FF93EF93A1E2B6E0E12FB8
:10171A00F0E0BD01A5E1B0E00E94DDD2DB01AE0F31
:10172A00BF1F14960E941FD4AF91BF91EC93A2EDF4
:10173A00BDE0E12FF0E0EE0FFF1FAE0FBF1FEC91EF
:10174A00E078E560EC93A2EDBDE0E12FF0E0EE0F6A
:10175A00FF1FAE0FBF1FEC91EF77EC931F5FC8CF4F
:10176A001991089563970E9428D2E0916304E07466
:10177A0021F40E942FD269960895A091C80DA13034
:10178A0008F466C7E091C80DE150E093C80DEF5F19
:10179A00E091C80DE03009F05BC7E091C70DE09316
:1017AA00C80DE091C90DEF5FE093C90DE150A0911A
:1017BA00C90DAF3018F0E0E0E093C90DEC85E07F89
:1017CA00E860EC87FE017196FA93EA93E0E0EA9307
:1017DA00A8E0B0E00E9427CBE091C90DF0E0309775
:1017EA0009F056C1E091CE0DF091CF0DE17009F4E8
:1017FA004BC120E0E0919707E17009F02160E09188
:10180A009907E17009F02260E0919B07E17009F005
:10181A002460E0919D07E17009F02860E0919F073C
:10182A00E17009F02061E091A107E17009F02062FE
:10183A00E091A307E17009F02064E091A507E17047
:10184A0009F02068298B20E0E091A707E17009F0F0
:10185A002160E091A907E17009F02260E091AB07ED
:10186A00E17009F02460E091AD07E17009F02860A9
:10187A00FE017296208320E0E091F90CE07409F0F1
:10188A002160E091010DE07409F02260E091090DF8
:10189A00E07409F02460E091110DE07409F0286009
:1018AA00E091190DE07409F02061E091210DE074D6
:1018BA0009F02062E091290DE07409F02064E091BA
:1018CA00310DE07409F02068FE017396208320E050
:1018DA00E091390DE07409F02160E091410DE07466
:1018EA0009F02260E091490DE07409F02460E0916A
:1018FA00510DE07409F02860E091590DE07409F087
:10190A002061E091610DE07409F02062E091690DB7
:10191A00E07409F02064E091710DE07409F0206828
:10192A00FE017496208320E0E0917704E07809F0C4
:10193A002160E0918504E07809F02260E091930447
:10194A00E07809F02460E091A104E07809F02860C9
:10195A00E091AF04E07809F02061E091BD04E078FD
:10196A0009F02062E091CB04E07809F02064E0916C
:10197A00D904E07809F02068FE017596208320E0FA
:10198A00E091E704E07809F02160E091F504E0785D
:10199A0009F02260E0910305E07809F02460E09103
:1019AA001105E07809F02860E0911F05E07809F058
:1019BA002061E0912D05E07809F02062E0913B0575
:1019CA00E07809F02064E0914905E07809F02068A0
:1019DA00FE017696208320E0E0915705E07809F031
:1019EA002160E0916505E07809F02260E0917305D5
:1019FA00E07809F02460E0918105E07809F0286038
:101A0A00E0918F05E07809F02061E0919D05E0788A
:101A1A0009F02062E0919D05E07809F02064E091E8
:101A2A00B905E07809F02068FE017796208320E066
:101A3A00E091C705E07809F02160E091D505E078EA
:101A4A0009F02260E091E305E07809F02460E09172
:101A5A00F105E07809F02860E091FF05E07809F0E7
:101A6A002061E0910D06E07809F02062E0911B0602
:101A7A00E07809F02064E0912906E07809F020680E
:101A8A00FE0178962083AAC5E1E0E093C90D05C05E
:101A9A00E130A0E0FA0709F0DCC0E091CE0DF09148
:101AAA00CF0DE27009F4D1C0E0910A09E077E03382
:101ABA0021F4E0910A09E47009F403C0E6E6E98B2F
:101ACA000DC0E0910A09E295E770FF27662777279C
:101ADA00E85EFE4F6F4F6BBF0690098AE0911409CA
:101AEA00E077E03321F4E0911409E47009F403C0CB
:101AFA00E6E6EA8B0DC0E0911409E295E770FF274C
:101B0A0066277727E85EFE4F6F4F6BBF06900A8AFB
:101B1A00E0911E09E077E03321F4E0911E09E470B8
:101B2A0009F403C0E6E6EB8B0DC0E0911E09E295CD
:101B3A00E770FF2766277727E85EFE4F6F4F6BBF78
:101B4A0006900B8AE0912809E077E03321F4E091CE
:101B5A002809E47009F403C0E6E6EC8B0DC0E091B5
:101B6A002809E295E770FF2766277727E85EFE4F88
:101B7A006F4F6BBF06900C8AE0913209E077E03331
:101B8A0021F4E0913209E47009F403C0E6E6ED8B32
:101B9A000DC0E0913209E295E770FF2766277727A3
:101BAA00E85EFE4F6F4F6BBF06900D8AE0913C09CD
:101BBA00E077E03321F4E0913C09E47009F403C0D2
:101BCA00E6E6EE8B0DC0E0913C09E295E770FF274F
:101BDA0066277727E85EFE4F6F4F6BBF06900E8A27
:101BEA00E0914609E077E03321F4E0914609E47098
:101BFA0009F403C0E6E6EF8B0DC0E0914609E295D1
:101C0A00E770FF2766277727E85EFE4F6F4F6BBFA7
:101C1A0006900F8AE0915009E077E03321F4E091D1
:101C2A005009E47009F403C0E6E6E88F0DC0E091BC
:101C3A005009E295E770FF2766277727E85EFE4F8F
:101C4A006F4F6BBF0690088EC9C4E2E0E093C90DDE
:101C5A0005C0E230A0E0FA0709F0DCC0E091CE0D41
:101C6A00F091CF0DE47009F4D1C0E0915A09E07700
:101C7A00E03321F4E0915A09E47009F403C0E6E67E
:101C8A00E98B0DC0E0915A09E295E770FF276627B4
:101C9A007727E85EFE4F6F4F6BBF0690098AE09187
:101CAA006409E077E03321F4E0916409E47009F40F
:101CBA0003C0E6E6EA8B0DC0E0916409E295E7709D
:101CCA00FF2766277727E85EFE4F6F4F6BBF0690A8
:101CDA000A8AE0916E09E077E03321F4E0916E0917
:101CEA00E47009F403C0E6E6EB8B0DC0E0916E09DF
:101CFA00E295E770FF2766277727E85EFE4F6F4F6A
:101D0A006BBF06900B8AE0917809E077E03321F403
:101D1A00E0917809E47009F403C0E6E6EC8B0DC0A3
:101D2A00E0917809E295E770FF2766277727E85E52
:101D3A00FE4F6F4F6BBF06900C8AE0918209E077E5
:101D4A00E03321F4E0918209E47009F403C0E6E685
:101D5A00ED8B0DC0E0918209E295E770FF276627B7
:101D6A007727E85EFE4F6F4F6BBF06900D8AE091B2
:101D7A008C09E077E03321F4E0918C09E47009F4EE
:101D8A0003C0E6E6EE8B0DC0E0918C09E295E770A0
:101D9A00FF2766277727E85EFE4F6F4F6BBF0690D7
:101DAA000E8AE0919609E077E03321F4E0919609F2
:101DBA00E47009F403C0E6E6EF8B0DC0E0919609E2
:101DCA00E295E770FF2766277727E85EFE4F6F4F99
:101DDA006BBF06900F8AE091A009E077E03321F407
:101DEA00E091A009E47009F403C0E6E6E88F0DC0AB
:101DFA00E091A009E295E770FF2766277727E85E5A
:101E0A00FE4F6F4F6BBF0690088EE8C3E3E0E09386
:101E1A00C90D04C0E330A0E0FA0721F4E4E0E0933E
:101E2A00C90D04C0E430A0E0FA0721F4E5E0E0932C
:101E3A00C90D05C0E530A0E0FA0709F0C8C0E09175
:101E4A00CE0DF091CF0DE07209F4BDC0E0911109F9
:101E5A00F0911209EA87FB87AA85BB85AC3EE3E1CC
:101E6A00BE0730F4E4E1F0E00E9423D32E2F01C034
:101E7A002FEF298BA0911709A63319F4E0E0EA8B1A
:101E8A0016C0E0911B09F0911C09EA87FB87AA8515
:101E9A00BB85AC3EE3E1BE0730F4E4E1F0E00E942A
:101EAA0023D32E2F01C02FEFFE0172962083E091DB
:101EBA002509F0912609EA87FB87AA85BB85AC3EEE
:101ECA00E3E1BE0730F4E4E1F0E00E9423D32E2FD1
:101EDA0001C02FEFFE0173962083A0912B09A63330
:101EEA0019F4E0E0EC8B16C0E0912F09F09130096B
:101EFA00EA87FB87AA85BB85AC3EE3E1BE0730F4DF
:101F0A00E4E1F0E00E9423D32E2F01C02FEFFE015F
:101F1A0074962083E0913909F0913A09EA87FB87A0
:101F2A00AA85BB85AC3EE3E1BE0730F4E4E1F0E00C
:101F3A000E9423D32E2F01C02FEFFE017596208316
:101F4A00E0914309F0914409EA87FB87AA85BB859A
:101F5A00AC3EE3E1BE0730F4E4E1F0E00E9423D3B3
:101F6A002E2F01C02FEFFE0176962083E0914D09B6
:101F7A00F0914E09EA87FB87AA85BB85AC3EE3E16F
:101F8A00BE0730F4E4E1F0E00E9423D32E2F01C013
:101F9A002FEFFE0177962083E0915709F0915809B7
:101FAA00EA87FB87AA85BB85AC3EE3E1BE0730F42E
:101FBA00E4E1F0E00E9423D32E2F01C02FEFFE01AF
:101FCA00789620830BC3E6E0E093C90D05C0E6309E
:101FDA00A0E0FA0709F0BAC0E091CE0DF091CF0D5A
:101FEA00E07409F4AFC0E0916109F0916209EA87EF
:101FFA00FB87AA85BB85AC3EE3E1BE0730F4E4E18A
:10200A00F0E00E9423D32E2F01C02FEF298BE091FD
:10201A006B09F0916C09EA87FB87AA85BB85AC3E00
:10202A00E3E1BE0730F4E4E1F0E00E9423D32E2F6F
:10203A0001C02FEFFE0172962083E0917509F0919D
:10204A007609EA87FB87AA85BB85AC3EE3E1BE0732
:10205A0030F4E4E1F0E00E9423D32E2F01C02FEFE9
:10206A00FE0173962083E0917F09F0918009EA8747
:10207A00FB87AA85BB85AC3EE3E1BE0730F4E4E109
:10208A00F0E00E9423D32E2F01C02FEFFE01749699
:10209A002083E0918909F0918A09EA87FB87AA855A
:1020AA00BB85AC3EE3E1BE0730F4E4E1F0E00E9418
:1020BA0023D32E2F01C02FEFFE0175962083E091C6
:1020CA009309F0919409EA87FB87AA85BB85AC3E00
:1020DA00E3E1BE0730F4E4E1F0E00E9423D32E2FBF
:1020EA0001C02FEFFE0176962083E0919D09F091C1
:1020FA009E09EA87FB87AA85BB85AC3EE3E1BE075A
:10210A0030F4E4E1F0E00E9423D32E2F01C02FEF38
:10211A00FE0177962083E091A709F091A809EA8742
:10212A00FB87AA85BB85AC3EE3E1BE0730F4E4E158
:10213A00F0E00E9423D32E2F01C02FEFFE017896E4
:10214A0020834CC2E7E0E093C90D04C0E730A0E069
:10215A00FA0721F4E8E0E093C90D04C0E830A0E0F2
:10216A00FA0721F4E9E0E093C90D04C0E930A0E0E0
:10217A00FA0759F5E091CE0DF091CF0DF27009F101
:10218A00A091FD08AA237AF0A091FC08B091FD085D
:10219A00EAE0F0E00E940BD3EA87FB870E94B4D200
:1021AA00EA87FB8703C0E0E0EA87EB87EB85E98BE8
:1021BA00EA85EA8BE091BD0DEB8BE091BC0DEC8BCF
:1021CA000DC2EAE0E093C90D04C0EA30A0E0FA07C4
:1021DA00E1F4E091CE0DF091CF0DF47091F0A09161
:1021EA000509B0910609E4E1F0E00E9423D3EA87E9
:1021FA00FB87EB85ED8BEA85EE8BE0E0EF8BE88FD2
:10220A00EDC1EBE0E093C90D04C0EB30A0E0FA07A2
:10221A00C9F5E091CE0DF091CF0DF87079F120E07B
:10222A00E091790DE07409F02160E091810DE0748C
:10223A0009F02260E091890DE07409F02460E091D0
:10224A00910DE07409F02860298BE091B509E170DD
:10225A0021F0E091B609E695EE8BE091BD09E170B7
:10226A0021F0E091BE09E695EF8BE091C509E17096
:10227A0021F0E091C609E695E88FB0C1ECE0E09361
:10228A00C90D04C0EC30A0E0FA07C9F5E091CE0D03
:10229A00F091CF0DF07179F1E2E0E98BE0E1EA8BA0
:1022AA00A6E1B0E00E941FD4EB8BA5E1B0E00E944A
:1022BA001FD4EC8BE091CD09E17021F0E091CE09B9
:1022CA00E695ED8BE091D509E17021F0E091D60910
:1022DA00E695EE8BE091DD09E17021F0E091DE09EF
:1022EA00E695EF8BE091E509E17021F0E091E609CE
:1022FA00E695E88F73C1EDE0E093C90D05C0ED30B6
:10230A00A0E0FA0709F0A6C0E091CE0DF091CF0D3A
:10231A00F07209F49BC0E091D10DEF5FE093D10D0B
:10232A00E150E98B20E0E091BF0DE03009F0216037
:10233A00E091C00DE03009F02260E0910009E170FF
:10234A0009F02460E0910009E27009F02860E09148
:10235A000009E07209F02061E091FF08E07809F0D5
:10236A002062A5E3B1E00E941FD4A091B30DAE177D
:10237A0008F02064A091CE03A13008F02068FE0185
:10238A0072962083E091A70DF091A80DFF70EF2FB0
:10239A00F0E0EB8BE091A70DF091A80DEC8BE0E05B
:1023AA001E2F2E2F51E0183060F4A3E01A9FF0017F
:1023BA00ED5BF84FE081E27009F0252B1F5F550FA6
:1023CA00F2CFFE017596208320E018E051E010312B
:1023DA0060F4A3E01A9FF001ED5BF84FE081E27030
:1023EA0009F0252B1F5F550FF2CFFE017696208349
:1023FA0020E010E151E0143160F4A3E01A9FF001EB
:10240A00ED5BF84FE081E27009F0252B1F5F550F55
:10241A00F2CFFE0177962083E0E01E2F2E2F51E0A7
:10242A00153080F4E12FAFE7B7E0F0E00E94A6D2C2
:10243A00AE0FBF1F1396EC91E17009F0252B1F5FB9
:10244A00550FEECFFE0178962083C8C0EEE0E093E8
:10245A00C90D05C0EE30A0E0FA0709F0BFC0E0914F
:10246A00CE0DF091CF0DF07409F4B4C0E091850857
:10247A00F09186080E94B8D2EA87FB87EB85E98B40
:10248A00EA85EA8BE0918708F09188080E94B8D221
:10249A00EA87FB87EB85EB8BEA85EC8B20E0E09102
:1024AA000009E47009F02160E0910009E87009F080
:1024BA002260E0910009E07109F02460E0910009CE
:1024CA00E07209F02860FE0175962083E091BB074F
:1024DA00F0E0E130A0E0FA0711F5E091BC07E078FE
:1024EA00E9F0E091C507EE8BA091C607E091DE07FF
:1024FA00E295E07FEA2BEF8BE091DE07F0E00E94A5
:10250A00ABD2309749F4E091DF07F0E00E94A2D203
:10251A00309711F4E0E001C0E1E0E88F5AC0E23000
:10252A00A0E0FA0721F0E330A0E0FA07A1F5E09174
:10253A00BE07E03079F1E0E01E2F3E2F0E2F35E086
:10254A0021E0E091BD071E17E0F4A2EEB7E0E12F0B
:10255A00F0E00E94A6D2AE0FBF1F1296EC91E17076
:10256A0009F0022B220F203051F4E32F3F5FF0E0F5
:10257A00DE015196EA0FFB1F008300E021E01F5F96
:10258A00E0CF203039F0E32FF0E0DE015196EA0F78
:10259A00FB1F00831EC0E430A0E0FA07D1F4A0912B
:1025AA00C007A130B0F0E091C307EE8B3091EB0782
:1025BA00A091C607E32FE295E07FEA2BEF8BE32F8A
:1025CA00E295EF70AE2FE091EE07E295E07FEA2BFD
:1025DA00E88F04C0E0E0E093C90DFEC8A091CA0DDF
:1025EA00B091CB0D8091CC0D9091CD0DE091C90D9C
:1025FA00F0E06F2F660F660B762FEA0FFB1F681F3E
:10260A00791FEE83FF8368877987AE81BF818885CA
:10261A009985A030E8E0BE07E0E08E07E0E09E077B
:10262A0040F4EC85EF7EEC87EE81FF81ED87FE8733
:10263A000BC0EC85E061EC87EE81FF8168857985C6
:10264A00ED87FE876F87788BDE011C960E943E0914
:10265A000E942FD26996089564970E9428D2E09129
:10266A006304E07409F424C4EF81E07FE860EF8337
:10267A00A091D00DA13008F450C0E091D00DE150E6
:10268A00E093D00DEF5FE091D00DE03009F045C046
:10269A00AFE3B1E00E941FD4E093D00DABE3B1E009
:1026AA000E9417D4EC8BFD8B6E8B7F8BAC89BD8916
:1026BA008E899F89A030E8E0BE07E0E08E07E0E05F
:1026CA009E0740F4EF81EF7EEF83EC89FD89E8876E
:1026DA00F9870BC0EF81E061EF83EC89FD896E8990
:1026EA007F89E887F9876A877B87A9E3B1E00E9437
:1026FA001FD4EC87AAE3B1E00E941FD4ED87E2E081
:10270A00EE87E0E1EF87E1E0E88BE0E0E98BEA8B36
:10271A00EB8BDE0117960E943E09A091C10DA130F4
:10272A0008F421C1E091C10DE150E093C10DE03000
:10273A0009F019C1FE013C96FA93EA93E0E0EA93A4
:10274A00A8E0B0E00E9427CBA3E5B5E00E941FD421
:10275A00E093C10DA4E5B5E00E9417D4EC8BFD8B84
:10276A006E8B7F8BAC89BD898E899F89A030E8E00A
:10277A00BE07E0E08E07E0E09E0740F4EF81EF7EBF
:10278A00EF83EC89FD89E887F9870BC0EF81E06167
:10279A00EF83EC89FD896E897F89E887F9876A87E3
:1027AA007B87A091C20DA13090F1E091C30DEF5F3C
:1027BA00E093C30DE150A091C30DE091C20DEA1759
:1027CA0018F4E1E0E093C30DE091C30DEC87A8E5AE
:1027DA00B5E0F0E03496AE0FBF1F0E941FD44E2F13
:1027EA004F3010F04F3108F012C0E42FF0E03F975D
:1027FA00AAE0B0E00E94DDD2EF5EF64FDF01ED9174
:10280A00FD91DF01E4E1F0E00E9423D3EB8BADE51B
:10281A00B5E00E941FD44E2F4F3010F04F3108F010
:10282A0012C0E42FF0E03F97AAE0B0E00E94DDD2A8
:10283A00EF5EF64FDF01ED91FD91DF01E4E1F0E09B
:10284A000E9423D3EA8BACE5B5E00E941FD44E2F39
:10285A004F3010F04F3108F012C0E42FF0E03F97EC
:10286A00AAE0B0E00E94DDD2EF5EF64FDF01ED9103
:10287A00FD91DF01E4E1F0E00E9423D3E98BABE5AF
:10288A00B5E00E941FD44E2F4F3010F04F3108F0A0
:10289A0012C0E42FF0E03F97AAE0B0E00E94DDD238
:1028AA00EF5EF64FDF01ED91FD91DF01E4E1F0E02B
:1028BA000E9423D3E88BAAE5B5E00E941FD44E2FCD
:1028CA004F3010F04F3108F012C0E42FF0E03F977C
:1028DA00AAE0B0E00E94DDD2EF5EF64FDF01ED9193
:1028EA00FD91DF01E4E1F0E00E9423D3EF87A9E53F
:1028FA00B5E00E941FD44E2F4F3010F04F3108F030
:10290A0012C0E42FF0E03F97AAE0B0E00E94DDD2C7
:10291A00EF5EF64FDF01ED91FD91DF01E4E1F0E0BA
:10292A000E9423D3EE87A8E5B5E00E941FD44E2F5C
:10293A004F3010F04F3108F012C0E42FF0E03F970B
:10294A00AAE0B0E00E94DDD2EF5EF64FDF01ED9122
:10295A00FD91DF01E4E1F0E00E9423D3ED87DE017F
:10296A0017960E943E09A091C40DA13008F47CC0BC
:10297A00E091C40DE150E093C40DEF5FE091C40D06
:10298A00E03009F071C0FE013C96FA93EA93E0E068
:10299A00EA93A8E0B0E00E9427CBAAE6B5E00E943D
:1029AA001FD4E093C40DABE6B5E00E9417D4EC8BBC
:1029BA00FD8B6E8B7F8BAC89BD898E899F89A030F8
:1029CA00E8E0BE07E0E08E07E0E09E0740F4EF8112
:1029DA00EF7EEF83EC89FD89E887F9870BC0EF81E9
:1029EA00E061EF83EC89FD896E897F89E887F98741
:1029FA006A877B87E0E00E2F1E2F2E2F51E01033BF
:102A0A0000F5AFE6B5E0EE27A10FBE1F0E941FD466
:102A1A004E2F403031F0A42F0E94713CE03009F073
:102A2A00052B503859F4E22F2F5FF0E0DE011C9697
:102A3A00EA0FFB1F008351E000E001C0550F1F5F42
:102A4A00DECFA0910509B0910609AC39E3E6BE07CD
:102A5A0028F4E4E6F0E00E9423D301C0EFEFEA8B0A
:102A6A00DE0117960E943E09A091C50DA13008F417
:102A7A00A9C0E091C50DE150E093C50DEF5FE0916B
:102A8A00C50DE03009F09EC0AFE9B5E00E941FD441
:102A9A00E093C50DA0EAB5E00E9417D4EC8BFD8B3C
:102AAA006E8B7F8BAC89BD898E899F89A030E8E0C7
:102ABA00BE07E0E08E07E0E09E0740F4EF81EF7E7C
:102ACA00EF83EC89FD89E887F9870BC0EF81E06124
:102ADA00EF83EC89FD896E897F89E887F9876A87A0
:102AEA007B87E0E00E2F1E2F2E2F51E0103308F0C7
:102AFA0055C0A4EAB5E0EE27A10FBE1F0E941FD45D
:102B0A004E2F4030D9F14F3010F04F3108F024C029
:102B1A004F3108F5E42FF0E03F97AAE0B0E00E94B9
:102B2A00DDD2E65FF64FE081E295E770EE83E42FAF
:102B3A00F0E03F97AAE0B0E00E94DDD2E65FF64FF0
:102B4A00E081E47039F4AE81A13021F0A43011F0B3
:102B5A00A53009F4052B12C0473310F04C3308F0A6
:102B6A0007C0A42F0E94E980E03009F0052B06C0B7
:102B7A00A42F0E94713CE03009F0052B503859F41B
:102B8A00E22F2F5FF0E0DE011C96EA0FFB1F0083A5
:102B9A0051E000E001C0550F1F5FA8CFA091FC08CB
:102BAA00B091FD0800240A160B0624F4EA89E2957E
:102BBA00EF7001C0E0E0EA8BE0E0EB8BDE011796F4
:102BCA000E943E09A091C60DA13008F4A8C0E09168
:102BDA00C60DE150E093C60DEF5FE091C60DE030FF
:102BEA0009F09DC0FE013C96FA93EA93E0E0EA936D
:102BFA00A8E0B0E00E9427CBA4EDB5E00E941FD464
:102C0A00E093C60DA5EDB5E00E9417D4EC8BFD8BC1
:102C1A006E8B7F8BAC89BD898E899F89A030E8E055
:102C2A00BE07E0E08E07E0E09E0740F4EF81EF7E0A
:102C3A00EF83EC89FD89E887F9870BC0EF81E061B2
:102C4A00EF83EC89FD896E897F89E887F9876A872E
:102C5A007B87E0E00E2F1E2F2E2F51E0103408F054
:102C6A005AC0A9EDB5E0EE27A10FBE1F0E941FD4DE
:102C7A004E2F403009F43FC0103220F04F3010F090
:102C8A004F3108F024C04F3108F5E42FF0E03F97A8
:102C9A00AAE0B0E00E94DDD2E65FF64FE081E2955D
:102CAA00E770EE83E42FF0E03F97AAE0B0E00E94DD
:102CBA00DDD2E65FF64FE081E47039F4AE81A130EF
:102CCA0021F0A43011F0A53009F4052B14C01032FC
:102CDA0020F0473310F04C3308F007C0A42F0E94AD
:102CEA00E980E03009F0052B06C0A42F0E94713C50
:102CFA00E03009F0052B503859F4E22F2F5FF0E04D
:102D0A00DE011C96EA0FFB1F008351E000E001C0C0
:102D1A00550F1F5FA3CFDE0117960E943E0910E0F0
:102D2A00133008F0C5C0A2EDBDE0E12FF0E0EE0FD0
:102D3A00FF1FAE0FBF1F11964C91403009F4B6C069
:102D4A00A2EDBDE0E12FF0E0EE0FFF1FAE0FBF1FB7
:102D5A00EC91EF773E2FA42F0E94713C0E2FA2ED2B
:102D6A00BDE0E12FF0E0EE0FFF1FAE0FBF1FEC91A9
:102D7A00EE1FE0E0EE1FE1700E1799F031E0A2EDD0
:102D8A00BDE0E12FF0E0EE0FFF1FAE0FBF1FE02FF7
:102D9A00E170E795E0E0E7950E2EEC91EF77E029F8
:102DAA00EC93313008F473C03150303009F06FC001
:102DBA00A0E2B6E00E941FD43E2FA1E2B6E0E12FC6
:102DCA00F0E0BD01A5E1B0E00E94DDD2DB01AE0F6B
:102DDA00BF1F0E9417D4EC8BFD8B6E8B7F8BAC8947
:102DEA00BD898E899F89A030E8E0BE07E0E08E07A2
:102DFA00E0E09E0740F4EF81EF7EEF83EC89FD89E6
:102E0A00E887F9870BC0EF81E061EF83EC89FD89E0
:102E1A006E897F89E887F9876A877B87EF81E07FF8
:102E2A00E860EF83A2EDBDE0E12FF0E0EE0FFF1FB7
:102E3A00AE0FBF1FEC91E07869F0A1E2B6E0E12F96
:102E4A00F0E0BD01A5E1B0E00E94DDD2E60FF71F78
:102E5A0035960CC0A1E2B6E0E12FF0E0BD01A5E194
:102E6A00B0E00E94DDD2E60FF71F3D96E88FF98F9A
:102E7A00FE013C96FA93EA93EA8DFB8DFA93EA9364
:102E8A00A8E00E94B726DE0117960E943E09A2ED2D
:102E9A00BDE0E12FF0E0EE0FFF1FAE0FBF1FE32FE3
:102EAA00EF770E2EEC91E078E029EC931F5F38CF94
:102EBA000E942FD26A9608951A93A3E5B5E0E0E03E
:102ECA000E943BD4A4E5B5E0E0E0F0E060E070E009
:102EDA000E942BD410E0123148F4A8E5B5E0EE27A1
:102EEA00A10FBE1F0E943BD41F5FF5CFE0E2F6E0C0
:102EFA00FA93EA93AAE60E94EC26E0E9F6E4FA934A
:102F0A00EA93A0E5B0E00E948C2AAAE6B5E0E0E0E8
:102F1A000E943BD4ABE6B5E0E0E0F0E060E070E0B0
:102F2A000E942BD410E0103348F4AFE6B5E0EE2748
:102F3A00A10FBE1F0E943BD41F5FF5CFAFE9B5E0DA
:102F4A00E0E00E943BD4A0EAB5E0E0E0F0E060E017
:102F5A0070E00E942BD410E0103348F4A4EAB5E0E4
:102F6A00EE27A10FBE1F0E943BD41F5FF5CFA4ED31
:102F7A00B5E0E0E00E943BD4A5EDB5E0E0E0F0E08A
:102F8A0060E070E00E942BD410E0103448F4A9ED00
:102F9A00B5E0EE27A10FBE1F0E943BD41F5FF5CFFD
:102FAA00A9E1B6E0E0E00E943BD4AAE1B6E0E0E0A5
:102FBA00F0E060E070E00E942BD4AEE1B6E0E7E614
:102FCA00FEEF0E9433D4A5C21A93ACE6B2E00E9487
:102FDA001BD4DF010E94CE04A5E7B2E00E941FD4F1
:102FEA00E170A5EFB8E0E170E795E0E0E7950E2E15
:102FFA00EC91EF77E029EC93E0E0E093F208EDE55D
:10300A00F4E0FA93EA93E0E0EA93A6EEB2E00E94D3
:10301A0027CBA0E7B2E00E941FD4E0935E04A09100
:10302A005E04A53018F4E5E0E0935E04A5E7B2E09B
:10303A000E941FD4E695E170A3E6B4E0E170E7953B
:10304A00E0E0E7950E2EEC91EF77E029EC93A1E70B
:10305A00B2E00E9417D4E0935F04F0936004609397
:10306A00610470936204E0E0E0936A0410E01433B0
:10307A0008F01DC2ABE7B2E0E12FF0E0BD01AEE01F
:10308A00B0E00E94DDD2DB01AE0FBF1F1A960E948C
:10309A001FD4E07809F409C2ABE6B4E0E12FF0E00E
:1030AA00BD01AEE0B0E00E94DDD2DB01AE0FBF1F72
:1030BA001A96EC91E068EC93ABE6B4E0E12FF0E00D
:1030CA00BD01AEE0B0E00E94DDD2E60FF71FFF932C
:1030DA00EF93ABE7B2E0E12FF0E0BD01AEE0B0E084
:1030EA000E94DDD2DB01AE0FBF1F0E9417D4AF9141
:1030FA00BF91ED93FD936D937C93ABE6B4E0E12F22
:10310A00F0E0BD01AEE0B0E00E94DDD2E60FF71FAD
:10311A003496FF93EF93ABE7B2E0E12FF0E0BD0105
:10312A00AEE0B0E00E94DDD2DB01AE0FBF1F149605
:10313A000E941BD4AF91BF91ED93FC93ABE6B4E030
:10314A00E12FF0E0BD01AEE0B0E00E94DDD2E60F73
:10315A00F71F3696FF93EF93ABE7B2E0E12FF0E06B
:10316A00BD01AEE0B0E00E94DDD2DB01AE0FBF1FB1
:10317A0016960E941BD4AF91BF91ED93FC93ABE6D8
:10318A00B4E0E12FF0E0BD01AEE0B0E00E94DDD294
:10319A00E60FF71F3896FF93EF93ABE7B2E0E12F04
:1031AA00F0E0BD01AEE0B0E00E94DDD2DB01AE0F7F
:1031BA00BF1F18960E941BD4AF91BF91ED93FC9349
:1031CA00ABE6B4E0E12FF0E0BD01AEE0B0E00E9472
:1031DA00DDD2E60FF71F3A96FF93EF93ABE7B2E023
:1031EA00E12FF0E0BD01AEE0B0E00E94DDD2DB01EC
:1031FA00AE0FBF1F1A960E941FD4EF70AF91BF91F6
:10320A00EF700E2EEC91E07FE029EC93ABE6B4E090
:10321A00E12FF0E0BD01AEE0B0E00E94DDD2E60FA2
:10322A00F71F3A96FF93EF93ABE7B2E0E12FF0E096
:10323A00BD01AEE0B0E00E94DDD2DB01AE0FBF1FE0
:10324A001A960E941FD4E295E770AF91BF91E7707A
:10325A00E295E07F0E2EEC91EF78E029EC93ABE655
:10326A00B4E0E12FF0E0BD01AEE0B0E00E94DDD2B3
:10327A00E60FF71F3B96FF93EF93ABE7B2E0E12F20
:10328A00F0E0BD01AEE0B0E00E94DDD2DB01AE0F9E
:10329A00BF1F1B960E941FD4EF70AF91BF91EF70B2
:1032AA000E2EEC91E07FE029EC93ABE6B4E0E12F3F
:1032BA00F0E0BD01AEE0B0E00E94DDD2E60FF71FFC
:1032CA003B96FF93EF93ABE7B2E0E12FF0E0BD014D
:1032DA00AEE0B0E00E94DDD2DB01AE0FBF1F1B964D
:1032EA000E941FD4E295EF70AF91BF91EF70E29503
:1032FA00E07F0E2EEC91EF70E029EC93ABE6B4E0A0
:10330A00E12FF0E0BD01AEE0B0E00E94DDD2E60FB1
:10331A00F71F3C96FF93EF93ABE7B2E0E12FF0E0A3
:10332A00BD01AEE0B0E00E94DDD2DB01AE0FBF1FEF
:10333A001C960E941FD4E170AF91BF91E1700E2ECE
:10334A00EC91EE7FE029EC93ABE6B4E0E12FF0E0FC
:10335A00BD01AEE0B0E00E94DDD2E60FF71F3C9659
:10336A00FF93EF93ABE7B2E0E12FF0E0BD01AEE0EF
:10337A00B0E00E94DDD2DB01AE0FBF1F1C960E9497
:10338A001FD4E695E170AF91BF91E170EE0F0E2E5A
:10339A00EC91ED7FE029EC93ABE6B4E0E12FF0E0AD
:1033AA00BD01AEE0B0E00E94DDD2E60FF71F3C9609
:1033BA00FF93EF93ABE7B2E0E12FF0E0BD01AEE09F
:1033CA00B0E00E94DDD2DB01AE0FBF1F1C960E9447
:1033DA001FD4E695E695E370AF91BF91E370EE0FC7
:1033EA00EE0F0E2EEC91E37FE029EC93ABE6B4E00E
:1033FA00E12FF0E0BD01AEE0B0E00E94DDD2E60FC1
:10340A00F71F3C96FF93EF93ABE7B2E0E12FF0E0B2
:10341A00BD01AEE0B0E00E94DDD2DB01AE0FBF1FFE
:10342A001C960E941FD4E295E170AF91BF91E170A2
:10343A00E295E07F0E2EEC91EF7EE029EC93ABE66D
:10344A00B4E0E12FF0E0BD01AEE0B0E00E94DDD2D1
:10345A00DB01AE0FBF1F1C96EC91EC70E43089F0D3
:10346A00ABE6B4E0E12FF0E0BD01AEE0B0E00E94CF
:10347A00DDD2DB01AE0FBF1F1C96EC91EC70EC3075
:10348A0081F4ABE6B4E0E12FF0E0BD01AEE0B0E0DC
:10349A000E94DDD2DB01AE0FBF1F1C96EC91E068E3
:1034AA00EC93E12FEF5FE0936A041F5FE0CDE4E65F
:1034BA00F4E0FA93EA93E0E4F1E0FA93EA93A5E000
:1034CA000E94B726E0916504F09166046091670452
:1034DA007091680430976040704021F4E091640470
:1034EA00EF7E15C0E0916404E061E0936404F0E0CB
:1034FA00F695E795E370F070E330A0E0FA0721F063
:10350A00E130A0E0FA0729F4E0916404E860E0936E
:10351A00640419910895BA93AA936D970E9428D2C8
:10352A00E0E0EE8BABA1BCA1EC91E295E1703E2FFD
:10353A003030C1F01196ED91FD916D917D91ED8F35
:10354A00FE8F6F8F78A3E0915F04F0916004609121
:10355A00610470916204AD8DBE8D8F8D98A10E9419
:10356A00D5D20CC0ABA1BCA111964D915C91A09192
:10357A005F04B0916004FA010E94C3D2E88FE03080
:10358A00A9F1ABA1BCA1EC91EF70E13048F0EBA13D
:10359A00FCA1A581A17021F00E9499280E94A37E16
:1035AA00ABA1BCA1EC91EF70E63000F120E0E1E0C4
:1035BA00EA8FE98F2031D0F4ABA1BCA11596EA8D30
:1035CA00F0E0AE0FBF1FEC91A98DEA2319F0A22FEC
:1035DA000E946F70E98DEE0FE98FE03029F4EA8DD1
:1035EA00EF5FEA8FE1E0E98F2F5FE4CFE0916404B7
:1035FA00E07109F43FC0303079F0E0916504F09150
:10360A0066046091670470916804AD8DBE8D8F8DDC
:10361A0098A10E94D5D207C0A0916504B091660412
:10362A00FA010E94C3D2E88FE03021F1EBA1FCA19C
:10363A00A581A17071F0E0916404E17021F0E0913C
:10364A006404E77F03C0E0916404E860E0936404E3
:10365A000DC0E0916404E17021F0E0916404E86037
:10366A0003C0E0916404E77FE0936404E0915E04A0
:10367A00E0936904E0916304EF70E23011F4E1E051
:10368A00EE8BA0916A04A433A0F0EAEEF1E060E0C8
:10369A0070E00E94B1D3E0916A04FF27662777277A
:1036AA000E94B1D384E00E94AFD12896E4E3E0936C
:1036BA006A0420E0E0916A042E1708F04FC5ABE6D1
:1036CA00B4E0E22FF0E0BD01AEE0B0E00E94DDD24E
:1036DA00E60FF71F8F01E285E07809F43DC5303027
:1036EA0061F0D801ED91FD916D917D91AD8DBE8D09
:1036FA008F8D98A10E94D5D207C0D801ED91FD9176
:10370A00DF01FA010E94C3D2E88FE03009F424C530
:10371A00E0916304E07409F40DC5F801E485E071F1
:10372A0071F1ABE7B2E0E22FF0E0BD01AEE0B0E04C
:10373A000E94DDD2DB01AE0FBF1F1C960E941FD470
:10374A00E295EF70E695E770ABA1BCA11596F0E0A3
:10375A00AE0FBF1FEC91EF93ABE7B2E0E22FF0E0C0
:10376A00BD01AEE0B0E00E94DDD2DB01AE0FBF1FAB
:10377A001D960E941FD4AF91EA1709F0DBC4ABE68D
:10378A00B4E0E22FF0E0BD01AEE0B0E00E94DDD28D
:10379A00DB01AE0FBF1F1D96E0915E04EC93E0E0E3
:1037AA00E9A3EAA3F801E385EF70E13038F1ABA1B0
:1037BA00BCA11596F801E385F0E0EF70F07031973F
:1037CA00AE0FBF1FEC91F0E0E9A3FAA3F9A1E0E084
:1037DA00E9A3FAA3ABA1BCA11596F801E385F0E031
:1037EA000E94B4D2EF70F0703197AE0FBF1FEC9108
:1037FA00A9A1BAA1F0E0EA2BFB2B0FC0ABA1BCA197
:10380A001596F801E385F0E00E94B4D2EF70F070EB
:10381A003197AE0FBF1FEC91F0E0E9A3FAA3D801EC
:10382A001896ED91FD91A9A1BAA1EA23FB23E9A378
:10383A00FAA3F801E485E17059F0F801A085B18591
:10384A00FD01F695E795A9A1BAA1EA17FB0708F0C9
:10385A000CC0D8011896ED91FD91E095F095A9A1BB
:10386A00BAA1EA2BFB2BE9A3FAA3F801E485E295B6
:10387A00EF70E695E695E170EF8BF801E485E1706B
:10388A0009F456C2E9A1FAA1EB8FFC8FF801E2858F
:10389A00F0E0EF70F070E630A0E0FA0709F4C7C173
:1038AA003097C9F4AB8DBC8D00240A160B0624F49C
:1038BA00EB8DFC8DF29606C0AC8DAA232AF4EB8D13
:1038CA00FC8DF297EB8FFC8FAB8DBC8DE4E6F0E0BC
:1038DA000E9436D3AAC1E130A0E0FA07C9F4AB8D41
:1038EA00BC8D00240A160B0624F4EB8DFC8D799608
:1038FA0006C0AC8DAA232AF4EB8DFC8D7997EB8F49
:10390A00FC8FAB8DBC8DE2E3F0E00E9436D38DC113
:10391A00E230A0E0FA07C9F4AB8DBC8D00240A1688
:10392A000B0624F4EB8DFC8D3A9606C0AC8DAA23C7
:10393A002AF4EB8DFC8D3A97EB8FFC8FAB8DBC8D07
:10394A00E4E1F0E00E9436D370C1E330A0E0FA0768
:10395A00C9F4AB8DBC8D00240A160B0624F4EB8D3A
:10396A00FC8D359606C0AC8DAA232AF4EB8DFC8D0E
:10397A003597EB8FFC8FAB8DBC8DEAE0F0E00E94AF
:10398A0036D353C1E430A0E0FA07C9F4AB8DBC8D3D
:10399A0000240A160B0624F4EB8DFC8D339606C020
:1039AA00AC8DAA232AF4EB8DFC8D3397EB8FFC8F19
:1039BA00AB8DBC8DE5E0F0E00E9436D336C1E53030
:1039CA00A0E0FA07C9F4AB8DBC8D00240A160B06D9
:1039DA0024F4EB8DFC8D329606C0AC8DAA232AF412
:1039EA00EB8DFC8D3297EB8FFC8FAB8DBC8DE2E0BB
:1039FA00F0E00E9436D319C1E730A0E0FA0741F59A
:103A0A00AB8DBC8D00240A160B0674F4AF3FEFE3AE
:103A1A00BE071CF0EFEFFFE704C0EB8DFC8DEE0F45
:103A2A00FF1FEB8FFC8F13C0AC8DAA2382F4AB8DE2
:103A3A00BC8DE0E0F0ECEA17FB071CF0E0E0F0E8F0
:103A4A0004C0EB8DFC8DEE0FFF1FEB8FFC8FEFC0D8
:103A5A00E830A0E0FA0761F5AB8DBC8D00240A16A8
:103A6A000B0684F4A939E9E1BE071CF0EFEFFFE782
:103A7A0006C0EB8DFC8DA5E0B0E00E940BD3EB8F66
:103A8A00FC8F15C0AC8DAA2392F4AB8DBC8DE7E6F2
:103A9A00F6EEEA17FB071CF0E0E0F0E806C0EB8D53
:103AAA00FC8DA5E0B0E00E940BD3EB8FFC8FBFC06A
:103ABA00E930A0E0FA0761F5AB8DBC8D00240A1647
:103ACA000B0684F4AC3CECE0BE071CF0EFEFFFE71A
:103ADA0006C0EB8DFC8DAAE0B0E00E940BD3EB8F01
:103AEA00FC8F15C0AC8DAA2392F4AB8DBC8DE4E398
:103AFA00F3EFEA17FB071CF0E0E0F0E806C0EB8DF5
:103B0A00FC8DAAE0B0E00E940BD3EB8FFC8F8FC034
:103B1A00EA30A0E0FA0761F5AB8DBC8D00240A16E5
:103B2A000B0684F4A636E6E0BE071CF0EFEFFFE7CB
:103B3A0006C0EB8DFC8DA4E1B0E00E940BD3EB8FA5
:103B4A00FC8F15C0AC8DAA2392F4AB8DBC8DEAE92B
:103B5A00F9EFEA17FB071CF0E0E0F0E806C0EB8D8E
:103B6A00FC8DA4E1B0E00E940BD3EB8FFC8F5FC009
:103B7A00EB30A0E0FA0761F5AB8DBC8D00240A1684
:103B8A000B0684F4AF38E2E0BE071CF0EFEFFFE764
:103B9A0006C0EB8DFC8DA2E3B0E00E940BD3EB8F45
:103BAA00FC8F15C0AC8DAA2392F4AB8DBC8DE1E7D6
:103BBA00FDEFEA17FB071CF0E0E0F0E806C0EB8D2A
:103BCA00FC8DA2E3B0E00E940BD3EB8FFC8F2FC0D9
:103BDA00EC30A0E0FA0759F5AB8DBC8D00240A162B
:103BEA000B0684F4A734E1E0BE071CF0EFEFFFE711
:103BFA0006C0EB8DFC8DA4E6B0E00E940BD3EB8FE0
:103C0A00FC8F15C0AC8DAA2392F4AB8DBC8DE1E775
:103C1A00FDEFEA17FB071CF0E0E0F0E806C0EB8DC9
:103C2A00FC8DA4E6B0E00E940BD3EB8FFC8FF80169
:103C3A00E285F0E00E94B4D2E770F070309769F440
:103C4A00F801A481B581EB8DFC8DEA17FB0711F40D
:103C5A00E1E001C0E0E0EF8B6AC0E130A0E0FA07E2
:103C6A0069F4F801A481B581EB8DFC8DEA17FB0795
:103C7A0011F4E0E001C0E1E0EF8B59C0E230A0E0CE
:103C8A00FA07D9F4EF89E03061F0D8011696ED9180
:103C9A00FD91AB8DBC8DEA17FB0714F0E0E0EF8BCA
:103CAA000BC0D8011496ED91FD91AB8DBC8DEA172E
:103CBA00FB0714F4E1E0EF8B3AC0E330A0E0FA0727
:103CCA00D9F4EF89E03061F0D8011696ED91FD91B3
:103CDA00AB8DBC8DAE17BF0714F0E0E0EF8B0BC0C5
:103CEA00D8011496ED91FD91AB8DBC8DAE17BF072F
:103CFA0014F4E1E0EF8B1BC0E430A0E0FA07B9F45A
:103D0A00D8011496ED91FD91AB8DBC8DAE17BF070E
:103D1A004CF0D8011696ED91FD91AB8DBC8DEA174A
:103D2A00FB070CF402C0E1E001C0E0E0EF8B75C1D3
:103D3A00F801E285F0E0EF70F070E630A0E0FA07F3
:103D4A0009F4CCC0309761F4E9A1FAA1F296E9A38B
:103D5A00FAA3A9A1BAA1E4E6F0E00E9423D3BCC069
:103D6A00E130A0E0FA0761F4E9A1FAA17996E9A3A2
:103D7A00FAA3A9A1BAA1E2E3F0E00E9423D3ACC05E
:103D8A00E230A0E0FA0761F4E9A1FAA13A96E9A3C0
:103D9A00FAA3A9A1BAA1E4E1F0E00E9423D39CC04E
:103DAA00E330A0E0FA0761F4E9A1FAA13596E9A3A4
:103DBA00FAA3A9A1BAA1EAE0F0E00E9423D38CC039
:103DCA00E430A0E0FA0761F4E9A1FAA13396E9A385
:103DDA00FAA3A9A1BAA1E5E0F0E00E9423D37CC02E
:103DEA00E530A0E0FA0741F4E9A1FAA13196E9A386
:103DFA00FAA3F695E79570C0E730A0E0FA0781F4D8
:103E0A00A9A1BAA1AF3FEFE7BE0728F4E9A1FAA139
:103E1A00EE0FFF1F02C0EFEFFFEFE9A3FAA35EC0A8
:103E2A00E830A0E0FA0779F4A9A1BAA1A333E3E341
:103E3A00BE0720F4E5E00E9405D302C0EFEFFFEFD2
:103E4A00E9A3FAA34BC0E930A0E0FA0779F4A9A1E3
:103E5A00BAA1A939E9E1BE0720F4EAE00E9405D334
:103E6A0002C0EFEFFFEFE9A3FAA338C0EA30A0E0FF
:103E7A00FA0779F4A9A1BAA1AC3CECE0BE0720F498
:103E8A00E4E10E9405D302C0EFEFFFEFE9A3FAA332
:103E9A0025C0EB30A0E0FA0779F4A9A1BAA1AE31A6
:103EAA00E5E0BE0720F4E2E30E9405D302C0EFEF8B
:103EBA00FFEFE9A3FAA312C0EC30A0E0FA0771F40D
:103ECA00A9A1BAA1AF38E2E0BE0720F4E4E60E9455
:103EDA0005D302C0EFEFFFEFE9A3FAA3F801E285E9
:103EEA00F0E00E94B4D2E770F070309769F4F801FC
:103EFA00A481B581E9A1FAA1EA17FB0711F4E1E06F
:103F0A0001C0E0E0EF8B89C0E130A0E0FA0769F474
:103F1A00F801A481B581E9A1FAA1EA17FB0711F01A
:103F2A00E0E001C0E1E0EF8B78C0E230A0E0FA0700
:103F3A00D1F5F801E485E170D9F0EF89E03061F05C
:103F4A00D8011696ED91FD91A9A1BAA1EA17FB072E
:103F5A0014F0E0E0EF8B0BC0D8011496ED91FD91BF
:103F6A00A9A1BAA1EA17FB0714F4E1E0EF8B1AC082
:103F7A00EF89E03061F0D8011696ED91FD91A9A183
:103F8A00BAA1EA17FB0710F0E0E0EF8B0BC0D801EB
:103F9A001496ED91FD91A9A1BAA1EA17FB0710F4B5
:103FAA00E1E0EF8B3AC0E330A0E0FA07D9F4EF89F9
:103FBA00E03061F0D8011696ED91FD91A9A1BAA160
:103FCA00AE17BF0710F0E0E0EF8B0BC0D8011496D4
:103FDA00ED91FD91A9A1BAA1AE17BF0710F4E1E0D6
:103FEA00EF8B1BC0E430A0E0FA07B9F4D8011496AD
:103FFA00ED91FD91A9A1BAA1AE17BF0748F0D8016A
:10400A001696ED91FD91A9A1BAA1EA17FB0708F44A
:10401A0002C0E1E001C0E0E0EF8BF801E485E27064
:10402A0009F448C0F801E485E07419F4EF89E03036
:10403A0009F43FC0F801E485E078F1F0D8011C9654
:10404A00EC91EF77EC93E0916304E073E03298F03F
:10405A00EDEFF1E060E070E00E94B1D3E22FF0E012
:10406A0031966F2F660F660B762F0E94B1D384E0CC
:10407A000E94AFD128961DC0D8011C96EC91E06829
:10408A00EC93E0916304E073E03298F0E8E0F2E048
:10409A0060E070E00E94B1D3E22FF0E031966F2F1A
:1040AA00660F660B762F0E94B1D384E00E94AFD1CF
:1040BA00289633C0F801E485EE1FE0E0EE1FE170B8
:1040CA00AE2FEF89EA1749F1D8011C96E170E795FE
:1040DA00E0E0E7950E2EEC91EF77E029EC93E09182
:1040EA006304E073E032C8F0E3E1F2E060E070E01C
:1040FA000E94B1D3E22FF0E031966F2F660F660B64
:10410A00762F0E94B1D3EF8DFF27662777270E946B
:10411A00B1D388E00E94AFD12C96D8011C96EF89C2
:10412A00E170E295E07FEE0FEE0F0E2EEC91EF7B41
:10413A00E029EC93E0916304EF70E13059F0E091EB
:10414A006304EF70AE2FE22FF0E03396B0E0EA1787
:10415A00FB0711F4E1E0EE8B2F5FACCAE091630438
:10416A00EF70E23019F0EE89E030A1F1ABA1BCA109
:10417A00EC91EF70ED87AD85A93010F0E8E0ED879E
:10418A00ED85E85FEF83E6E0E887ABA1BCA1EC919F
:10419A00E07121F011960E949AD307C0ABA1BCA18D
:1041AA001196ED91FD9166277727E987FA876B8744
:1041BA007C87FE013E96FA93EA93EDA1FEA135961D
:1041CA00FA93EA93A989BB270E9415CBDE011696BA
:1041DA000E9457970E942FD2A59608951A930A9380
:1041EA00AEE6B2E00E941FD40E2F003029F0A02FB5
:1041FA000E94713CE03021F0E0916304E06403C066
:10420A00E0916304EF7BE093630410E0E0916A04B9
:10421A001E1708F07DC0ABE6B4E0E12FF0E0BD0167
:10422A00AEE0B0E00E94DDD2DB01AE0FBF1F1D96EB
:10423A00AC91A13008F46AC0ABE6B4E0E12FF0E03B
:10424A00BD01AEE0B0E00E94DDD2DB01AE0FBF1FC0
:10425A001D96EC91E150EC93ABE6B4E0E12FF0E06F
:10426A00BD01AEE0B0E00E94DDD2DB01AE0FBF1FA0
:10427A001D96EC91E03009F049C0ABE6B4E0E12FBD
:10428A00F0E0BD01AEE0B0E00E94DDD2DB01AE0F8E
:10429A00BF1F1C96EC91F0E00E94B8D2E370F07058
:1042AA00309781F4ABE6B4E0E12FF0E0BD01AEE077
:1042BA00B0E00E94DDD2DB01AE0FBF1F1C96EC916D
:1042CA00EF7713C0E130A0E0FA0701F5ABE6B4E0FE
:1042DA00E12FF0E0BD01AEE0B0E00E94DDD2DB01EB
:1042EA00AE0FBF1F1C96EC91E068EC93ABE6B4E00E
:1042FA00E12FF0E0BD01AEE0B0E00E94DDD2DB01CB
:10430A00AE0FBF1F1C96EC91EF7BEC931F5F7ECF25
:10431A00A0916904A13000F1E0916904E150E093B1
:10432A006904EF5FE0916904E030B1F4E09164045C
:10433A00F0E0F695E795E370F070309721F4E0919C
:10434A006404E77F07C0E130A0E0FA0729F4E091AE
:10435A006404E860E09364040C94B426A0971A936A
:10436A00A1E4B1E0E0E0F0E060E070E00E942BD46C
:10437A00ACE6B2E0E4EFF1E00E9433D4AEE6B2E09C
:10438A00E0E00E943BD4AFE6B2E00E943BD4A7E74C
:10439A00B2E0E0E10E943BD4A0E7B2E0E5E00E948F
:1043AA003BD4A1E7B2E0E0E0F0E060E070E00E9418
:1043BA002BD4A5E7B2E00E941FD4E1600E943BD44F
:1043CA00FE017196FA93EA93E0E0EA93A0E1B0E085
:1043DA000E9427CBFE013196FA93EA93E0E0EA9332
:1043EA00A0E1B0E00E9427CB10E0143308F046C1E8
:1043FA00ABE7B2E0E12FF0E0BD01AEE0B0E00E9431
:10440A00DDD2DB01AE0FBF1FE0E0F0E060E070E05C
:10441A000E942BD4ABE7B2E0E12FF0E0BD01AEE0A1
:10442A00B0E00E94DDD2DB01AE0FBF1F1496E0E0C0
:10443A00F0E00E9433D4ABE7B2E0E12FF0E0BD0137
:10444A00AEE0B0E00E94DDD2DB01AE0FBF1F1696D0
:10445A00E0E0F0E00E9433D4ABE7B2E0E12FF0E015
:10446A00BD01AEE0B0E00E94DDD2DB01AE0FBF1F9E
:10447A001896EFEFFFEF0E9433D4ABE7B2E0E12FDB
:10448A00F0E0BD01AEE0B0E00E94DDD2DB01AE0F8C
:10449A00BF1F1A960E941FD4E07FE6600E943BD499
:1044AA00ABE7B2E0E12FF0E0BD01AEE0B0E00E9480
:1044BA00DDD2DB01AE0FBF1F1A960E941FD4EF7820
:1044CA00E0620E943BD4ABE7B2E0E12FF0E0BD012D
:1044DA00AEE0B0E00E94DDD2DB01AE0FBF1F1A963C
:1044EA000E941FD4EF770E943BD4ABE7B2E0E12FE2
:1044FA00F0E0BD01AEE0B0E00E94DDD2DB01AE0F1C
:10450A00BF1F1C960E941FD4EE7F0E943BD4ABE7CC
:10451A00B2E0E12FF0E0BD01AEE0B0E00E94DDD2F2
:10452A00DB01AE0FBF1F1B960E941FD4E07F0E94C3
:10453A003BD4ABE7B2E0E12FF0E0BD01AEE0B0E082
:10454A000E94DDD2DB01AE0FBF1F1B960E941FD453
:10455A00EF700E943BD4ABE7B2E0E12FF0E0BD017F
:10456A00AEE0B0E00E94DDD2DB01AE0FBF1F1C96A9
:10457A000E941FD4ED7F0E943BD4ABE7B2E0E12F4B
:10458A00F0E0BD01AEE0B0E00E94DDD2DB01AE0F8B
:10459A00BF1F1C960E941FD4E37F0E943BD4ABE747
:1045AA00B2E0E12FF0E0BD01AEE0B0E00E94DDD262
:1045BA00DB01AE0FBF1F1C960E941FD4EF7E0E9424
:1045CA003BD4ABE7B2E0E12FF0E0BD01AEE0B0E0F2
:1045DA000E94DDD2DB01AE0FBF1F1C960E941FD4C2
:1045EA00EF710E943BD4ABE7B2E0E12FF0E0BD01EE
:1045FA00AEE0B0E00E94DDD2DB01AE0FBF1F1D9618
:10460A00E0E00E943BD4FE017196FA93EA93EFE14F
:10461A00F2E060E070E00E94B1D3E12FF0E0319661
:10462A006F2F660F660B762F0E94B1D384E00E942B
:10463A0074D12A96E12FF0E0A0E6BBE30E94A2D251
:10464A00EA0FFB1FFA93EA93FE017396FA93EA9331
:10465A00A0E10E948229E12FF0E0A0EABEE30E94D5
:10466A00A4D2EA0FFB1FFA93EA93FE013396FA9358
:10467A00EA93A8E00E9482291F5FB7CE0E94E91739
:10468A001881A19608951A93E3E4F7E0FA93EA935E
:10469A00E0E0EA93ACE3B0E00E9427CB10E01431EB
:1046AA0008F040C0AEEBB6E0E12FF0E0BD01A6E0B5
:1046BA00B0E00E94DDD2DB01AE0FBF1F0E941FD403
:1046CA00E03071F1A3E01A9FF001ED5BF84FDF01D2
:1046DA00EC91E160EC93A3E01A9FF001ED5BF84FD7
:1046EA00FF93EF93AEEBB6E0E12FF0E0BD01A6E059
:1046FA00B0E00E94DDD2DB01AE0FBF1F12960E940E
:10470A001BD4DF01EEE00E9463D2E370AF91BF9148
:10471A00E370E295E07F0E2EEC91EF7CE029EC93BA
:10472A001F5FBDCF199108950E9428D210E014315D
:10473A0008F013C2A3E01A9FF001ED5BF84FE08185
:10474A00E17009F408C2AEEBB6E0E12FF0E0BD017A
:10475A00A6E0B0E00E94DDD2DB01AE0FBF1F0E94CF
:10476A001FD4AE2F0E94713C0E2FA3E01A9FF001B6
:10477A00ED5BF84FE081F0E00E94B4D2E370F07094
:10478A00309709F07AC0003009F45BC01A9FF00133
:10479A00ED5BF84FE081E47009F052C0AEEBB6E091
:1047AA00E12FF0E0BD01A6E0B0E00E94DDD2DB011E
:1047BA00AE0FBF1F12960E941BD4FF73AF010024D5
:1047CA000416050688F4A3E01A9FF001ED5BF84F82
:1047DA00DF01EC91E860EC93A3E01A9FF001EC5B37
:1047EA00F84F408351832CC0A3E01A9FF001ED5B80
:1047FA00F84FDF01EC91E77FEC93A3E01A9FF001F9
:10480A00ED5BF84FDF01EC91E260EC93A3E01A9FB5
:10481A00F001EC5BF84FFF93EF93AEEBB6E0E12FBC
:10482A00F0E0BD01A6E0B0E00E94DDD2DB01AE0FF0
:10483A00BF1F14960E941BD4AF91BF91ED93FC93B6
:10484A001BC0A3E01A9FF001EC5BF84FA0E0B0E0B8
:10485A00A083B183A3E01A9FF001ED5BF84FDF015B
:10486A00EC91E77FEC93A3E01A9FF001ED5BF84F20
:10487A00DF01EC91ED7FEC931DC1E130A0E0FA0776
:10488A0009F063C0A091B30DAB3008F413C1003036
:10489A0041F4A3E01A9FF001ED5BF84FE081E47068
:1048AA0009F452C0AEEBB6E0E12FF0E0BD01A6E09C
:1048BA00B0E00E94DDD2DB01AE0FBF1F12960E944C
:1048CA001BD4FF73AF0100240416050688F4A3E085
:1048DA001A9FF001ED5BF84FDF01EC91E860EC9371
:1048EA00A3E01A9FF001EC5BF84F408351832CC080
:1048FA00A3E01A9FF001ED5BF84FDF01EC91E8604D
:10490A00EC93A3E01A9FF001ED5BF84FDF01EC9105
:10491A00E260EC93A3E01A9FF001EC5BF84FFF937F
:10492A00EF93AEEBB6E0E12FF0E0BD01A6E0B0E018
:10493A000E94DDD2DB01AE0FBF1F14960E941BD46A
:10494A00AF91BF91ED93FC93B5C0E230A0E0FA07B6
:10495A0009F05EC0003041F0A3E01A9FF001ED5B60
:10496A00F84FE081E47009F052C0AEEBB6E0E12FF7
:10497A00F0E0BD01A6E0B0E00E94DDD2DB01AE0F9F
:10498A00BF1F12960E941BD4FF73AF0100240416A6
:10499A00050688F4A3E01A9FF001ED5BF84FDF01EA
:1049AA00EC91E860EC93A3E01A9FF001EC5BF84FFE
:1049BA00408351832CC0A3E01A9FF001ED5BF84FAE
:1049CA00DF01EC91E860EC93A3E01A9FF001ED5B44
:1049DA00F84FDF01EC91E260EC93A3E01A9FF0013B
:1049EA00EC5BF84FFF93EF93AEEBB6E0E12FF0E00C
:1049FA00BD01A6E0B0E00E94DDD2DB01AE0FBF1F11
:104A0A0014960E941BD4AF91BF91ED93FC9352C0B0
:104A1A00E330A0E0FA0709F04DC0A091B30DAB3026
:104A2A0008F448C0003099F0A3E01A9FF001ED5B4A
:104A3A00F84FDF01EC91E260EC93A3E01A9FF001DA
:104A4A00EC5BF84FA0E0B0E0A083B18333C0A3E0F1
:104A5A001A9FF001ED5BF84FE081E47059F11A9F5B
:104A6A00F001ED5BF84FDF01EC91E77FEC93A3E0F7
:104A7A001A9FF001ED5BF84FDF01EC91E260EC93D5
:104A8A00A3E01A9FF001EC5BF84FFF93EF93AEEBB4
:104A9A00B6E0E12FF0E0BD01A6E0B0E00E94DDD271
:104AAA00DB01AE0FBF1F14960E941BD4AF91BF91BA
:104ABA00ED93FC93A3E01A9FF001ED5BF84FDF0141
:104ACA00E02FE170EE0FEE0F0E2EEC91EB7FE02956
:104ADA00EC93AEEBB6E0E12FF0E0BD01A6E0B0E06A
:104AEA000E94DDD2DB01AE0FBF1F11960E941FD4B8
:104AFA003E2F3030A1F0A3E01A9FF001ED5BF84F92
:104B0A00E081E87039F41A9FF001ED5BF84FE0811B
:104B1A00E27029F0A32F0E94713CE03009F41BC017
:104B2A00A3E01A9FF001ED5BF84FDF01EC91E77FFC
:104B3A00EC93A3E01A9FF001ED5BF84FDF01EC91D3
:104B4A00ED7FEC93A3E01A9FF001EC5BF84FA0E035
:104B5A00B0E0A083B1831F5FEACD0E942FD249C182
:104B6A001A9310E0143108F069C0A3E01A9FF0010B
:104B7A00ED5BF84FE081E17061F01A9FF001EC5BA8
:104B8A00F84FDF01ED91FC91119700240E160F06E4
:104B9A0008F052C0A3E01A9FF001EC5BF84FDF0166
:104BAA00ED91FD913197FE93EE93A3E01A9FF001E8
:104BBA00EC5BF84FDF01ED91FC9111973097E1F52D
:104BCA00A3E01A9FF001ED5BF84FE081E87059F11C
:104BDA001A9FF001ED5BF84FDF01EC91E77FEC9350
:104BEA00A3E01A9FF001EC5BF84FFF93EF93AEEB53
:104BFA00B6E0E12FF0E0BD01A6E0B0E00E94DDD210
:104C0A00DB01AE0FBF1F14960E941BD4AF91BF9158
:104C1A00ED93FC93A3E01A9FF001ED5BF84FDF01DF
:104C2A00EC91E26008C0A3E01A9FF001ED5BF84F37
:104C3A00DF01EC91ED7FEC931F5F94CF0C945D2B19
:104C4A0060971A93FE013196FA93EA93E0E0EA93A9
:104C5A00A0E1B0E00E9427CB10E0143108F047C071
:104C6A00FE013196FA93EA93E0E0EA93A6E0B0E017
:104C7A000E9427CBAEEBB6E0E12FF0E0BD01A6E043
:104C8A00B0E00E94DDD2E60FF71FFA93EA93FE0125
:104C9A003396FA93EA93A6E080D0FE013196FA930E
:104CAA00EA93E6E2F2E060E070E00E94B1D3E12F1D
:104CBA00F0E031966F2F660F660B762F0E94B1D304
:104CCA0084E00E9474D12A96E12FF0E0A0E1B1E4D9
:104CDA000E94A2D2EA0FFB1FFA93EA93FE013396CF
:104CEA00FA93EA930E948229A8951F5FB6CF18818A
:104CFA00619608951A930A93E6E3F2E060E070E0A1
:104D0A000E94B1D380E00E94AFD124960FE010E058
:104D1A00E5E4F1E00E171F0738F4D801E0E00E943D
:104D2A003BD40F5F1F4FF4CF0E940E2EA0E0B0E0DD
:104D3A00E0E50E943BD4A1E0B0E0E3E40E943BD46A
:104D4A00A2E0B0E0EDE40E943BD4A3E0B0E0E0E5ED
:104D5A000E943BD4A4E0B0E0E0E00E943BD4099179
:104D6A00199108950E9428D20A2F2E813F814885E1
:104D7A00598510E0101778F4E12FF0E0E40FF51FE1
:104D8A000F01D901EE27A10FBE1F0E941FD4D00127
:104D9A00EC931F5FEFCF0C94882A0E9428D20A2F27
:104DAA002E813F814885598510E0101778F4E12F4C
:104DBA00F0E0E40FF51F0F01D901EE27A10FBE1F86
:104DCA00EC91D0010E943BD41F5FEFCF9CC30E949D
:104DDA002AD20A2F2C813D8110E0101740F4D90104
:104DEA00EE27A10FBE1F0E943BD41F5FF6CF0E9481
:104DFA0031D2269608950E9428D23A2F4E815F8199
:104E0A0010E0E32FF0E03197A12FB0E0AE17BF0713
:104E1A008CF4DA01EE27A10FBE1F0C91003051F07D
:104E2A00A885B985EE27A10FBE1FE02F0E943BD4AB
:104E3A001F5FE7CFA885B985EE27A10FBE1F0E9485
:104E4A003BD4E12F60C30E9428D23A2F4E815F8162
:104E5A0010E0E32FF0E03197A12FB0E0AE17BF07C3
:104E6A0094F4DA01EE27A10FBE1F0E941FD40E2F61
:104E7A00003049F0E12FA885B985F0E0EA0FFB1F61
:104E8A0000831F5FE6CFA885B985EE27A10FBE1F55
:104E9A00EC93E12F38C32E97D1500E942AD210E00A
:104EAA00133030F5FE01E250FF4FFA93EA93E0E047
:104EBA00F0E0FA93EA93A4E1B0E06CD1E03089F033
:104ECA00E091AE0DEE7FE093AE0DFE01E250FF4F92
:104EDA00FA93EA93ACEBB3E00E9437CBE03041F0AF
:104EEA0005C0E091AE0DE160E093AE0D1F5FD8CF33
:104EFA00133011F42CD194C0E0E0F0E0E093CC033D
:104F0A00F093CD0320E030E0283EE3E03E0708F0CE
:104F1A0059C0203DE3E03E0710F409E103C0E8EE82
:104F2A00E21B0E2FFE013496FA93EA93E091CA032C
:104F3A00F091CB0360E870E0AAE0B0E00E94DDD215
:104F4A00E60FF71FFA93EA93EAE0E09FF001DF0128
:104F5A0021D1E030A1F110E0101788F52F5F3F4F03
:104F6A00AAE01A9FF001DE011496AE0FBF1F169633
:104F7A00EC91E03021F1AAE01A9FF001DE011496CB
:104F8A00AE0FBF1FED91FD91A091CC03B091CD035F
:104F9A00AE17BF0790F4AAE01A9FF001DE0114963B
:104FAA00AE0FBF1FED91FC911197E093CC03F093E4
:104FBA00CD032093CA033093CB031F5FCDCF1017C5
:104FCA0008F0A2CFACECB3E0ED91FD913196FE93DF
:104FDA00EE93A091CA03B091CB03A83EE3E0BE07CB
:104FEA0028F0E0E0E093CA03E093CB03EDE4F2E0BB
:104FFA0060E070E00E94B1D3E091CA03F091CB0364
:10500A00662777270E94B1D3E091CC03F091CD03B4
:10501A00662777270E94B1D388E00E94AFD12C96E9
:10502A000E9431D26296DF5F08951A931A2F1A935B
:10503A00E0E0EA93A0E0B0E001D03AC32A970E94E8
:10504A0028D29D0108895989E2E6F2E060E070E021
:10505A000E94B1D3E52FFF27662777270E94B1D395
:10506A00E02FFF27662777270E94B1D388E00E94A6
:10507A00AFD12C96543638F0ABE7B9E00E941BD476
:10508A0031960E9433D4E091CC03F091CD03EE83A4
:10509A00FF83E091F410F091F5106091F610709191
:1050AA00F710E887F9876A877B875C870D872E87E1
:1050BA003F8710E01330A0F5E091CA03F091CB03CB
:1050CA0060E870E0AAE0B0E00E94DDD2E60FF71FC8
:1050DA00FA93EA93FE013896FA93EA93AAE00DD17D
:1050EA00E030E1F0ACECB3E0ED91FD913196FE9346
:1050FA00EE93AAECB3E0ED91FD913196FE93EE9317
:10510A00A091CA03B091CB03A83EE3E0BE0728F002
:10511A00E0E0E093CA03E093CB0302C01F5FCACF6B
:10512A000E942FD262960895E1E0F0E0E093CC036A
:10513A00F093CD03E0E0E093CA03E093CB03E0E809
:10514A00F0E0FA93EA93A0E1B7E2E1D10895649717
:10515A00FE01FA93EA93E0E0EA93A4E1B0E00E9448
:10516A0027CBFE01FA93EA93A6E4B2E080E090E04E
:10517A000E946FCBE2E0E887E0E1E987E0E0F0E057
:10518A00FA93EA93FE013296FA93EA93A4E1B5D030
:10519A00649608950E9428D2AD0110E01436C0F436
:1051AA001298EDB5E093A50DE5E0EEBDEDB5E7FF8C
:1051BA00FDCFE0E0EEBDEDB5E7FFFDCF0EB5129AEB
:1051CA0000FF06C080E991E00197F1F71F5FE6CF83
:1051DA00143659F4E885F985FA93EA93E0E0EA93FC
:1051EA00DA010E9427CBE0E08EC11298EDB5E09378
:1051FA00A50DE3E0EEBDEDB5E7FFFDCFEF81F07061
:10520A00EEBDEDB5E7FFFDCFEE81EEBDEDB5E7FFF3
:10521A00FDCF20E030E02417350788F4EDB5E093A0
:10522A00A50DE0E0EEBDEDB5E7FFFDCFA885B98598
:10523A00A20FB31FEEB5EC932F5F3F4FECCF129A3C
:10524A0061C10E9428D22A2F4E815F8110E0143654
:10525A00C0F41298EDB5E093A50DE5E0EEBDEDB50D
:10526A00E7FFFDCFE0E0EEBDEDB5E7FFFDCF3EB5D0
:10527A00129A30FF06C080E991E00197F1F71F5FAB
:10528A00E6CF143629F4A885B985E0E0EC933BC152
:10529A00213008F021501298EDB5E093A50DE3E016
:1052AA00EEBDEDB5E7FFFDCFE52FF070EEBDEDB534
:1052BA00E7FFFDCF4EBDEDB5E7FFFDCF00E00217DA
:1052CA00A0F4EDB5E093A50DE0E0EEBDEDB5E7FF86
:1052DA00FDCFA885B985EE27A00FBE1FEEB5EC93CA
:1052EA00EEB5E03011F00F5FEACF129AA885B985C2
:1052FA00EE27A00FBE1FEC9305C10E9428D25A2F99
:10530A0010E0513008F47AC000E00436C0F4129874
:10531A00EDB5E093A50DE5E0EEBDEDB5E7FFFDCFF8
:10532A00E0E0EEBDEDB5E7FFFDCF3EB5129A30FFE6
:10533A0006C080E991E00197F1F70F5FE6CF0436E6
:10534A0011F4E0E0E0C01298EDB5E093A50DE6E0B7
:10535A00EEBDEDB5E7FFFDCF129A000000001298EE
:10536A00EDB5E093A50DE5E0EEBDEDB5E7FFFDCFA8
:10537A00E0E0EEBDEDB5E7FFFDCF3EB5129A31FF95
:10538A003AC0E885EF77A0E8AE1B2A2F521708F437
:10539A00252F1298EDB5E093A50DE2E0EEBDEDB52F
:1053AA00E7FFFDCFE985F070EEBDEDB5E7FFFDCF74
:1053BA00E885EEBDEDB5E7FFFDCF00E0021780F40A
:1053CA00EDB5E093A50DAE81BF81EE27A10FBE1FFB
:1053DA00EC91EEBDEDB5E7FFFDCF0F5F1F5FEECF9E
:1053EA00129A521BE22FF0E0A885B985EA0FFB1F3B
:1053FA00E887F98702C0E0E086C083CF83C00E94B5
:10540A0028D25A2F10E0513008F47CC000E004364C
:10541A00C0F41298EDB5E093A50DE5E0EEBDEDB54B
:10542A00E7FFFDCFE0E0EEBDEDB5E7FFFDCF3EB50E
:10543A00129A30FF06C080E991E00197F1F70F5FF9
:10544A00E6CF043611F4E0E05EC01298EDB5E093C1
:10545A00A50DE6E0EEBDEDB5E7FFFDCF129A00001F
:10546A0000001298EDB5E093A50DE5E0EEBDEDB5AF
:10547A00E7FFFDCFE0E0EEBDEDB5E7FFFDCF3EB5BE
:10548A00129A31FF3CC0E885EF77A0E8AE1B2A2FBD
:10549A00521708F4252F1298EDB5E093A50DE2E016
:1054AA00EEBDEDB5E7FFFDCFE985F070EEBDEDB5D8
:1054BA00E7FFFDCFE885EEBDEDB5E7FFFDCF00E0E4
:1054CA00021780F4AE81BF81EE27A10FBE1F3C9167
:1054DA00EDB5E093A50D3EBDEDB5E7FFFDCF0F5F3E
:1054EA001F5FEECF129A303069F0521BE22FF0E0C4
:1054FA00A885B985EA0FFB1FE887F98702C0E0E0B3
:10550A0002C081CFE1E00E942FD22A9608950E941C
:10551A0028D2AD0110E000240416050608F07BC06D
:10552A0000E00436C0F41298EDB5E093A50DE5E06D
:10553A00EEBDEDB5E7FFFDCFE0E0EEBDEDB5E7FF6F
:10554A00FDCF3EB5129A30FF06C080E991E001977F
:10555A00F1F70F5FE6CF043611F4E0E05DC0129870
:10556A00EDB5E093A50DE6E0EEBDEDB5E7FFFDCFA5
:10557A00129A000000001298EDB5E093A50DE5E03F
:10558A00EEBDEDB5E7FFFDCFE0E0EEBDEDB5E7FF1F
:10559A00FDCF3EB5129A31FF3BC0EE81EF77A0E80E
:1055AA00AE1B2A2FFA01B0E0EA17FB0708F4242FF2
:1055BA001298EDB5E093A50DE2E0EEBDEDB5E7FF7B
:1055CA00FDCFEF81F070EEBDEDB5E7FFFDCFEE81C7
:1055DA00EEBDEDB5E7FFFDCF00E0021758F4EDB5DB
:1055EA00E093A50DE0E0EEBDEDB5E7FFFDCF0F5F5F
:1055FA001F5FF3CF129AA22FBB274A1B5B0BE22F26
:10560A00F0E0AE81BF81EA0FFB1FEE83FF8302C089
:10561A00E0E002C080CFE1E00E942FD228960895F0
:10562A001A93EFE7F7E0FA93EA93E0E0EA93A4E14A
:10563A00B0E00E9427CB10E01530D0F5E12FAFE79C
:10564A00B7E0F0E00E94A6D2EA0FFB1F0F01AAE81A
:10565A00B6E0E12FF0E00E94A6D2AE0FBF1F0E9473
:10566A001FD4D001EC93E12FAFE7B7E0F0E00E943E
:10567A00A6D2EA0FFB1F33960F01AAE8B6E0E12F84
:10568A00F0E00E94A6D2AE0FBF1F13960E941FD44D
:10569A00EE1FE0E0EE1FE170D001E170EE0FEE0FB9
:1056AA00EE0F0E2EEC91E77FE029EC931F5FC4CF3B
:1056BA00199108950E942AD22A2F10E0153008F075
:1056CA00CFC1E12FAFE7B7E0F0E00E94A6D2AE0F5C
:1056DA00BF1FAC91A03081F0E12FAFE7B7E0F0E057
:1056EA000E94A6D2AE0FBF1F1396EC91E695E695DF
:1056FA00E695E1702E1709F0B1C1E12FAFE7B7E0E7
:10570A00F0E00E94A6D2AE0FBF1FAC910E94713C7E
:10571A00E03009F479C0E12FAFE7B7E0F0E00E948A
:10572A00A6D2AE0FBF1F1396EC91E47009F06BC0BE
:10573A00E12FAFE7B7E0F0E00E94A6D2AE0FBF1F9D
:10574A001396EC91E160EC93E12FAFE7B7E0F0E05C
:10575A000E94A6D2AE0FBF1F1396EC91E460EC93A1
:10576A00E12FAFE7B7E0F0E00E94A6D2EA0FFB1FF5
:10577A0033960F01AAE8B6E0E12FF0E00E94A6D224
:10578A00AE0FBF1F13960E941FD4EF77E13010F0BF
:10579A00E1E001C0E0E0D001E170EE0F0E2EEC91E5
:1057AA00ED7FE029EC93E12FAFE7B7E0F0E00E944C
:1057BA00A6D2EA0FFB1F32960F01AAE8B6E0E12F44
:1057CA00F0E00E94A6D2AE0FBF1F13960E941FD40C
:1057DA00EF77D001EC93E12FAFE7B7E0F0E00E945A
:1057EA00A6D2EA0FFB1F31960F01AAE8B6E0E12F15
:1057FA00F0E00E94A6D2AE0FBF1F11960E941FD4DE
:10580A00D001EC932BC12FC0E12FAFE7B7E0F0E056
:10581A000E94A6D2AE0FBF1F1396EC91EB7FEC93BA
:10582A00E12FAFE7B7E0F0E00E94A6D2AE0FBF1FAC
:10583A001396EC91E270B9F4E12FAFE7B7E0F0E02C
:10584A000E94A6D2AE0FBF1F1396EC91EE7FEC9387
:10585A00E12FAFE7B7E0F0E00E94A6D2AE0FBF1F7C
:10586A001196E0E0EC93E12FAFE7B7E0F0E00E9499
:10587A00A6D2AE0FBF1F1196AC91A13008F4EEC0AC
:10588A00E12FAFE7B7E0F0E00E94A6D2AE0FBF1F4C
:10589A001196EC91E150EC93E12FAFE7B7E0F0E01D
:1058AA000E94A6D2AE0FBF1F1196EC91E03009F00C
:1058BA00D5C0E12FAFE7B7E0F0E00E94A6D2AE0F65
:1058CA00BF1F1396EC91E17009F48CC0EEE6F2E08A
:1058DA0060E070E00E94B1D3E12FF0E031966F2FC3
:1058EA00660F660B762F0E94B1D384E00E94AFD177
:1058FA002896E12FAFE7B7E0F0E00E94A6D2AE0FFC
:10590A00BF1F1396EC91EE7FEC93E12FAFE7B7E060
:10591A00F0E00E94A6D2AE0FBF1F1396EC91E27080
:10592A0009F442C0E12FAFE7B7E0F0E00E94A6D247
:10593A00AE0FBF1F1296AC91A130A8F1E12FAFE7CD
:10594A00B7E0F0E00E94A6D2AE0FBF1F1296EC910C
:10595A00E150EC93E12FAFE7B7E0F0E00E94A6D266
:10596A00AE0FBF1F1296AC91A130E8F0AAE8B6E0DC
:10597A00E12FF0E00E94A6D2AE0FBF1F12960E943E
:10598A001FD40E2FE295EF70E695E6953E2F031B86
:10599A00E6950E1BE12FAFE7B7E0F0E00E94A6D232
:1059AA00EA0FFB1F01831DC0AAE8B6E0E12FF0E071
:1059BA000E94A6D2AE0FBF1F12960E941FD40E2FAE
:1059CA00E295EF70E695E6953E2F031BE6950E1BD2
:1059DA00E12FAFE7B7E0F0E00E94A6D2EA0FFB1F83
:1059EA0001833CC0E6E7F2E060E070E00E94B1D3D8
:1059FA00E12FF0E031966F2F660F660B762F0E942B
:105A0A00B1D384E00E94AFD12896E12FAFE7B7E087
:105A1A00F0E00E94A6D2AE0FBF1F1396EC91E16090
:105A2A00EC93AAE8B6E0E12FF0E00E94A6D2AE0F0E
:105A3A00BF1F11960E941FD40E2FE295EF70E695B4
:105A4A00E6953E2F031BE6950E1BE12FAFE7B7E065
:105A5A00F0E00E94A6D2EA0FFB1F01831F5F2ECE41
:105A6A00BAC160971A93FE013196FA93EA93E0E07D
:105A7A00EA93A0E1B0E00E9427CB10E0153008F0CD
:105A8A0069C0AAE8B6E0E12FF0E00E94A6D2AE0F04
:105A9A00BF1FE0E00E943BD4AAE8B6E0E12FF0E0A5
:105AAA000E94A6D2AE0FBF1F1196E5E00E943BD41A
:105ABA00AAE8B6E0E12FF0E00E94A6D2AE0FBF1F1F
:105ACA001296E5E00E943BD4AAE8B6E0E12FF0E0A6
:105ADA000E94A6D2AE0FBF1F13960E941FD4E07871
:105AEA000E943BD4AAE8B6E0E12FF0E00E94A6D2D9
:105AFA00AE0FBF1F13960E941FD4EF770E943BD4AC
:105B0A00FE013196FA93EA93EDE7F2E060E070E085
:105B1A000E94B1D3E12FF0E031966F2F660F660B2A
:105B2A00762F0E94B1D384E00E9474D12A96E12F85
:105B3A00F0E0A0E4B0E40E94A2D2EA0FFB1FFA93BD
:105B4A00EA93FE013396FA93EA93A0E10E9482292E
:105B5A001F5F94CF65DD188161960895E0E0E2B990
:105B6A00EFEFE1B9E1E0E5B9E7EFE4B9E8E1E8B977
:105B7A00EFE9E7B9E5E2EBB9E8EBEAB9E2E0EEB959
:105B8A00EEE3EDB9E0EAE0936A00E0E0E1BBEFE0C2
:105B9A00E0937E00E0EFE0BBE0E0E4BBEFE1E3BBD3
:105BAA00E1E5ECBDE1E0EDBDE6E0E093C200E8E945
:105BBA00E093C100E0E0E093C500E3E0E093C400B5
:105BCA00EDE0E4BDE0E0E6BDEFE4E7BDE2E0E0934E
:105BDA006E000895E0E0E093B30D0E942E360E9415
:105BEA0055660E94D3800E94783B0E94E9170E9462
:105BFA00090B16DD0E9448230E9443C80E94BDC0BB
:105C0A000E94A8C20E94090B0E9474850E94F8464D
:105C1A0008956097A6E2B1E00E941FD4E07F0E9437
:105C2A003BD4A6E2B1E00E941FD4EF7E0E943BD48F
:105C3A00A6E2B1E00E941FD4E0620E943BD4A5E232
:105C4A00B1E0E0E00E943BD4A7E2B1E00E943BD47D
:105C5A00A8E2B1E00E943BD4A9E2B1E00E943BD4A1
:105C6A00AAE2B1E00E943BD4ABE2B1E00E943BD48D
:105C7A00ACE2B1E00E943BD4ADE2B1E0E4E10E94C3
:105C8A003BD4AEE2B1E0E0E00E943BD4AFE2B1E047
:105C9A000E943BD4A0E3B1E00E943BD4A1E3B1E06F
:105CAA000E943BD4FE01FA93EA93E0E0EA93A0E172
:105CBA00B0E00E9427CBFE01FA93EA93A3ECB3E08B
:105CCA000E9462CBE0E0F8E3FA93EA93FE0132968F
:105CDA00FA93EA93A0E10E948229E0E0E883E0E9EE
:105CEA00F4E4FA93EA93FE013296FA93EA93A1E076
:105CFA000E948229A2E3B1E0EEE1F0E0FF700F0119
:105D0A000E941BD4E070F07FE029F1290E9433D46D
:105D1A00A4E3B1E0E0E00E943BD4A5E3B1E0EAE00D
:105D2A000E943BD4A6E3B1E0E0E80E943BD4A7E39B
:105D3A00B1E00E943BD4E9E3F1E0FA93EA93A7E0E9
:105D4A000E94EC260E94CE7F0E9416810E94E345A3
:105D5A000E94B3210E94611784DE0E9425260E94B8
:105D6A00D7CA0E9428C20E9440C70E94C0940E94BB
:105D7A00A37E0E9485480E9499282CDFA8E0B0E003
:105D8A00E3E00E943BD46AD1609608950E942AD229
:105D9A00A89522E231E000E010E02638E9E03E076B
:105DAA0048F4D9010E941FD4F0E00E0F1F1F2F5F85
:105DBA003F4FF3CFE3E9F2E060E070E00E94B1D335
:105DCA00F801662777270E94B1D384E00E94AFD1F9
:105DDA002896A895F8010E9431D224960895EF9743
:105DEA00EF9726970E9428D2E091B40DED7FE093B9
:105DFA00B40DEB7FE093B40DE77FE093B40DE0E0E0
:105E0A00E093B60DA8E0B0E00E941FD4E330B1F5EC
:105E1A00E091B40DE260E093B40DA2E2B1E00E9419
:105E2A001FD4E13039F5E091B40DE460E093B40D8C
:105E3A00ADDFAF01A3E2B1E00E941BD4E887F98786
:105E4A00E985F0E0F0E04E1B5F0BE885F985F0E0AC
:105E5A00F0E04E1B5F0BE885F985E417F50731F48E
:105E6A00E091B40DE860E093B40D03C0E4E0E09380
:105E7A00B60D03C0E2E0E093B60D03C0E1E0E093A3
:105E8A00B60D30E040E050E0E2E2F1E0EE83FF835D
:105E9A00AE81BF81A638E9E0BE0708F04BC0E6E84C
:105EAA00F9E0EA1BFB0BE138A0E0FA0710F010E872
:105EBA0004C0AE81E6E8EA1B1E2FFE013A96FA9369
:105ECA00EA93E2E2F1E0A0E0B8E20E94C1D3EA1B61
:105EDA00FB0BA885B985EA0FFB1FFA93EA93A12F5A
:105EEA00BB270E94CF28303071F4AA85A13031F047
:105EFA00E091B60DE061E093B60D1CC0EB85FC8520
:105F0A00E887F98731E000E0011760F4E02FF0E05C
:105F1A00DE011A96AE0FBF1FEC91F0E04E0F5F1F25
:105F2A000F5FF2CFA895EE81FF81E058FF4FEE8315
:105F3A00FF83AECF313009F08BC0E985F0E0F0E0A5
:105F4A004E1B5F0BE885F985F0704E1B5F0BE885E9
:105F5A00F985E417F50709F076C0E091B40DE87009
:105F6A0009F070C0AFEFBFE00E941FD4EF5F0E943C
:105F7A003BD4E091B60DE064E093B60DE2E2F1E0C5
:105F8A00EE83FF83AE81BF81A638E9E0BE07B8F58C
:105F9A00E6E8F9E0EA1BFB0BE138A0E0FA0710F0AB
:105FAA0010E804C0AE81E6E8EA1B1E2FFE013A960D
:105FBA00FA93EA93E2E2F1E0A0E0B8E20E94C1D3E8
:105FCA00EA1BFB0BA885B985EA0FFB1FFA93EA9334
:105FDA00A12FBB270E94CF28EE81FF81FA93EA9373
:105FEA00FE013C96FA93EA93A12F0E94D226A89525
:105FFA00EE81FF81E058FF4FEE83FF83C3CFC6DEF9
:10600A00AF01A3E2B1E00E941BD4E887F987E985D2
:10601A00F0E0F0E04E1B5F0BE885F985F0E0F0E078
:10602A004E1B5F0BE885F985E417F50731F4E0911B
:10603A00B40DE860E093B40D05C0E091B60DE068D8
:10604A00E093B60D05C0E091B60DE062E093B60D9F
:10605A000E942FD2EF96EF962C960895EF97EF971E
:10606A0024970E9428D2E0EAF2E060E070E00E9401
:10607A00B1D380E00E94AFD12496A2E2B1E0E1E080
:10608A000E943BD4A3E2B1E0E0E0F0E00E9433D406
:10609A007DDEAF01A3E2B1E00E941BD4EE83FF8351
:1060AA00EF81F0E0F0E04E1B5F0BEE81FF81F0E044
:1060BA00F0E04E1B5F0BA3E2B1E0FA010E9433D479
:1060CA0022E231E02638E9E03E0760F5E6E8F9E049
:1060DA00E21BF30BE138A0E0FA0710F010E803C066
:1060EA00E6E8E21B1E2FFE013896FA93EA933A93EA
:1060FA002A93A12F0E94B726E2E2F1E0A0E0B8E2DB
:10610A000E94C1D3EA1BFB0BE20FF31FFA93EA9337
:10611A00FE013A96FA93EA93A12F0E948229205807
:10612A003F4FD0CFE091B40DE460E093B40DE86046
:10613A00E093B40DE0E0E093B60DE091B40DE071A8
:10614A0029F0E091B40DE160E093B40D0E942FD2E2
:10615A00EF96EF962A960895EF97EF9722970E9467
:10616A0028D24A2F403039F5A4E1B0E0E3E70E9493
:10617A003BD4A3E2B0E0E1E00E943BD4A4E2B0E069
:10618A00E0E0F0E00E9433D420E030E004E110E0E7
:10619A00E8E1F1E00E171F0748F4D8010E941FD466
:1061AA00F0E02E0F3F1F0F5F1F4FF2CFA4E2B0E0C7
:1061BA00F9010E9433D400E010E00430E1E01E0748
:1061CA0048F5E4E0F1E0E01BF10BE138A0E0FA0762
:1061DA0010F050E803C0E4E0E01B5E2FFE013696A3
:1061EA00FA93EA93E4E1F0E0E00FF11FFA93EA93FD
:1061FA00A52F0E94B726F801E058F140FA93EA93D6
:10620A00FE013896FA93EA93A52F0E948229005834
:10621A001F4FD3CF0E942FD2EF96EF96289608955C
:10622A000E9428D220E030E004E110E0E8E1F1E049
:10623A000E171F0748F4D8010E941FD4F0E02E0F52
:10624A003F1F0F5F1F4FF2CFA4E2B0E00E941BD4A2
:10625A00AF01E52FF0E0F0E02E1B3F0BFA01F0E072
:10626A00F0E02E1B3F0B4217530711F4E1E001C087
:10627A00E0E00E942FD226960895EF97EF97259790
:10628A000E9428D2E091B40DEF7EE093B40DE0E0D5
:10629A00DE01A957BF4FEC93DE01A957BF4FAC915E
:1062AA00A53038F5A0E0B0E00E941FD4E035C1F473
:1062BA00A1E0B0E00E941FD4E33491F4A2E0B0E080
:1062CA000E941FD4ED3461F4A3E0B0E00E941FD411
:1062DA00E03531F4A4E0B0E00E941FD4E03009F0C8
:1062EA0001C007C0DE01A957BF4FEC91EF5FEC93E5
:1062FA00D3CFDE01A957BF4FAC91A53039F40E9424
:10630A007F26E091B50DE160E093B50DA3E2B0E020
:10631A000E941FD4E03061F4A4E2B0E00E941BD4D2
:10632A00309731F4A2E2B0E00E941FD4EF3109F0B5
:10633A0008C0E091B50DE260E093B50DA0E00CDF76
:10634A000EC06EDFE03031F0E091B40DE061E09311
:10635A00B40D05C0E091B50DE460E093B50DE0E041
:10636A00DE01AA57BF4FEC93E0E0F0E08F019F01F6
:10637A000430E1E01E0708F061C0E4E0F1E0E01B50
:10638A00F10BE138A0E0FA0710F0E0E802C0E4E01F
:10639A00E01BDE01A857BF4FEC93FE013696FA9335
:1063AA00EA93F801E058F140FA93EA93DE01A45720
:1063BA00BF4FAC91BB270E94CF28FE01EA57FF4F7F
:1063CA00E081E030A9F4AE81A33719F4AD89A13098
:1063DA0009F008C04E895F89E1E0DE01AA57BF4F84
:1063EA00EC9306C0E091B50DE860E093B50D26C0C8
:1063FA00E0E0DE01A957BF4FEC93FE01E857FF4FDB
:10640A00E081DE01A957BF4FAC91AE17A0F4FE019F
:10641A00E957FF4FE081F0E0DE011696AE0FBF1F8D
:10642A00EC91F0E02E0F3F1FDE01A957BF4FEC9110
:10643A00EF5FEC93E2CF00581F4F9ACFE52FF0E0C1
:10644A00F0E02E1B3F0BFA01F0E0F0E02E1B3F0BB1
:10645A00DE01AA57BF4FAC91A13019F44217530776
:10646A0009F059C0E091B40DE07109F053C0E09110
:10647A00B50DE061E093B50D00E010E00430E1E015
:10648A001E0798F5E6E8F9E0E01BF10BE138A0E019
:10649A00FA0710F0E0E802C0E6E8E01BDE01A857C0
:1064AA00BF4FEC93FE013696FA93EA93F801E0584F
:1064BA00F140FA93EA93DE01A457BF4FAC91BB2790
:1064CA000E94CF28E4E1F0E0E00FF11FFA93EA938B
:1064DA00FE013896FA93EA93DE01A457BF4FAC91B6
:1064EA000E94D22600581F4FC9CF9ADEE03069F0C9
:1064FA00E091B40DE061E093B40DAEEFBFE00E940D
:10650A001FD4EF5F0E943BD405C0E091B50DE06255
:10651A00E093B50D17C0E091B50DE064E093B50DB9
:10652A00E091B40DE07171F0A1E016DEADEFBFE0CD
:10653A000E941FD4EF5F0E943BD4E091B50DE06842
:10654A00E093B50D0E942FD2EF96EF962B96089501
:10655A00EAEAF2E060E070E00E94B1D3E2E0F0E043
:10656A0060E070E00E94B1D3E0E1F0E060E070E04A
:10657A000E94B1D3E1E0F0E060E070E00E94B1D3A4
:10658A008CE00E94AFD16096E5EDF2E060E070E049
:10659A000E94B1D3A5E1B0E00E941BD466277727F9
:1065AA000E94B1D384E00E94AFD12896E1EEF2E0D6
:1065BA0060E070E00E94B1D3A7E1B0E00E941FD46E
:1065CA00FF27662777270E94B1D3A8E1B0E00E948F
:1065DA001FD4FF27662777270E94B1D388E00E943D
:1065EA00AFD12C96E9EFF2E060E070E00E94B1D3FF
:1065FA00E091B00DFF27662777270E94B1D3E0917B
:10660A00B10DFF27662777270E94B1D3AAE1B0E030
:10661A000E941FD4FF27662777270E94B1D38CE0F8
:10662A000E94AFD16096E7E1F3E060E070E00E947B
:10663A00B1D3E091F410F091F5106091F6107091D9
:10664A00F7100E94B1D384E00E94AFD12896E0915E
:10665A00B40DE27009F444C0E091B40DE47031F174
:10666A00E5E2F3E060E070E00E94B1D3A3E2B1E0BA
:10667A000E941BD4662777270E94B1D384E00E9428
:10668A00AFD12896E091B40DE87029F0E6E3F3E083
:10669A0060E070E004C0EAE3F3E060E070E00E94CA
:1066AA00B1D380E00E94AFD1249619C0E1E4F3E0AF
:1066BA0060E070E00E94B1D3A2E2B1E00E941FD470
:1066CA00FF27662777270E94B1D3E1E0F0E060E078
:1066DA0070E00E94B1D388E00E94AFD12C9619C015
:1066EA00E6E5F3E060E070E00E94B1D3A8E0B0E034
:1066FA000E941FD4FF27662777270E94B1D3E3E0C1
:10670A00F0E060E070E00E94B1D388E00E94AFD16F
:10671A002C96EBE6F3E060E070E00E94B1D3AFEFB5
:10672A00BFE00E941FD4FF27662777270E94B1D3B4
:10673A00ADEFBFE00E941FD4FF27662777270E948C
:10674A00B1D3AEEFBFE00E941FD4FF276627772799
:10675A000E94B1D38CE00E94AFD16096E0E8F3E0EA
:10676A0060E070E00E94B1D3E091B50DFF27662783
:10677A0077270E94B1D3E091B60DFF2766277727C6
:10678A000E94B1D388E00E94AFD12C960895ABE065
:10679A00B0E00E941FD4E093B00DACE0B0E00E94DC
:1067AA001FD4E093B10DDAD90E944D967894A1E0F6
:1067BA000E94FF370E945027A8955FDD10DBE09109
:1067CA00B40DE07121F0E091B40DE87009F405C050
:1067DA00E091B40DE160E093B40DFCD9A091F01002
:1067EA00B091F1108091F2109091F310AA3AE5E578
:1067FA00BE07E0E08E07EFEF9E0719F4E4B7E0FF6B
:10680A001AC0EAEAF5E560E07FEFE093F010F09352
:10681A00F1106093F2107093F310E0E0F0E060E0A2
:10682A0070E8E093F410F093F5106093F61070930B
:10683A00F710E093F810A2E3B1E00E941BD4FF70B6
:10684A00A7EABDE0FF700F01ED91FD91E070F07FC6
:10685A00E029F129FE93EE93E091A70DF091A80D9E
:10686A00FF703A9758F4E091A70DF091A80DE070E7
:10687A00F07FEA60E093A70DF093A80DE4B7E3FF79
:10688A0004C0A091F810A03009F002C0A4E006C02C
:10689A00E4B7E2FF02C0A5E001C0A2E00E941A2804
:1068AA00E0E0E4BFE093F810E3E9F3E060E070E0D1
:1068BA000E94B1D380E00E94AFD12496F09A4CD2C4
:1068CA00E091FF08E87FE260E093FF08E09163044B
:1068DA00EF7CE062E0936304E2E0E093F80CE1E02D
:1068EA00E093AB0DA2E3B1E00E941BD4FF70339793
:1068FA0070F4A2E3B1E0E3E0F0E0FF700F010E9460
:10690A001BD4E070F07FE029F1290E9433D4E09192
:10691A00B50DE03049F0EAE0EA93E0E0EA93A091AD
:10692A00B50DBB270E942328E091B60DE03049F04F
:10693A00EBE0EA93E0E0EA93A091B60DBB270E9450
:10694A002328A091060AA03071F4A091F10AE091DF
:10695A00F20AEA1741F4A0917A00A03021F4A0913A
:10696A00AB0DA03009F005C0E1E0E3BF8895E0E097
:10697A00E3BFA091B80DA13060F0E091B80DE150ED
:10698A00E093B80DEF5FE091B40DE07211F40E944C
:10699A00B70B0E947E05A0914608A43038F00E94E9
:1069AA00CF3E0E946DC9E0E0E0934608A091AB0D8E
:1069BA00A13008F428C1E091AB0DE150E093AB0D92
:1069CA00EF5FE5E0E093B80DA0E0F799A1E0E1E020
:1069DA00EA2711F4F79801C0F79AF79BE5C00E94DD
:1069EA0049C50E9496C9E091B40DE072D9F4E091CC
:1069FA00BB07F0E0E130A0E0FA0719F40E947E4AF2
:106A0A0011C0E230A0E0FA0721F0E330A0E0FA0773
:106A1A0019F40E94A55A06C0E430A0E0FA0711F45E
:106A2A000E941661A1E00E945F2BA0E020FCA1E079
:106A3A00E1E0EA27E894EE2309F0689420F820FEC2
:106A4A000FC00E941CC10E949923E091990DE07425
:106A5A0039F0E091990DEF7BE093990D0E946E8ACF
:106A6A00A091D80DA43030F4E091D80DEF5FE093F7
:106A7A00D80D91C0E0E0E093D80DA0E021FCA1E0A0
:106A8A00E1E0EA27E894EE2309F0689421F821FE70
:106A9A0082C0A895A091B30DAF3F30F4E091B30D39
:106AAA00EF5FE093B30DE150A091B70DA13060F014
:106ABA00E091B70DE150E093B70DEF5FE091B70DAC
:106ACA00E03011F4A0E048DBA091A60DA13030F02F
:106ADA00E091A60DE150E093A60D16C0E4E0E09324
:106AEA00A60DA5EFB8E00A2EEC91E695E170A1E0BB
:106AFA00EA27A02DE170EE0F0E2EEC91ED7FE02932
:106B0A00EC93E0E0E093F208A0914508A03131F45B
:106B1A001CD10E946E8A0E941D7311C0E091430825
:106B2A00EF70E13060F0A3E4B8E080E0EFE00E94AB
:106B3A00E5D3E0914308E061E093430801C00CD13A
:106B4A000E9455C40E94C1430E94F3200E9499CA20
:106B5A00A0E00E945F2B0E9431130E94B525E091AC
:106B6A00BB07F0E0E130A0E0FA0711F40E941855E3
:106B7A000E9458960E94F50AA091D90DA93030F4C6
:106B8A00E091D90DEF5FE093D90D05C0E0E0E09305
:106B9A00D90D0E94CFC4E091990DEF7BE093990D36
:106BAA000E94CE700E946738E091AC0DF091AD0D55
:106BBA007096E093AC0DF093AD0DA091AC0DB09131
:106BCA00AD0DA533ECE0BE07F0F0E091AC0DF0910D
:106BDA00AD0DE553FC40E093AC0DF093AD0DA4EF81
:106BEA00B0E1ED91FD916D917D91EF5FFF4F6F4F98
:106BFA007F4F7E936E93FE93EE930E9458810E947C
:106C0A00147E0E949639E0914308E07121F0A09128
:106C1A004508A03109F009C0E0914308EF7EE093EE
:106C2A00430893D00E941D7397D00E94B89689CECC
:106C3A00FFCFEA93EFB7EA93E1E0E093AA0DE09180
:106C4A00AB0DEF5FE093AB0DE150E991EFBFE99136
:106C5A00189524970E942AD210E01031B8F5A2E3C1
:106C6A00B0E0E12FF0E0BD01AAE0B0E00E94DDD281
:106C7A00DB01AE0FBF1F0E941BD40E94B6D29F0138
:106C8A002030E1E03E0788F0ECE9F3E060E070E0F4
:106C9A000E94B1D3F901662777270E94B1D384E015
:106CAA000E94AFD128962FEF30E0ADEBB8E0E12F8C
:106CBA00FF2766277727E054FF4F6F4F6BBFE69198
:106CCA00F0E0EA0FFB1F20831F5FC7CFABE1B0E004
:106CDA000E941BD49F0100240216030690F5E6E8E1
:106CEA00E0937A00E3E0E0937C00E6ECE0937A003C
:106CFA00E0917A00E074E1F7E0917800F091790090
:106D0A000E94A6D266277727A0ECB4ED81E090E036
:106D1A000E94E5D2EC83FD836E837F83F901AC8107
:106D2A00BD818E819F81662777270E943BD3E0939E
:106D3A00BC0DF093BD0DE0E0F0E0E093BA0DF093E6
:106D4A00BB0D0E9431D228960895E6E8E0937A00B6
:106D5A00E0E0E09342080895E6E8E0937A00E0E98B
:106D6A00E8B9E0E0E0937C00E0934408E09345084A
:106D7A00E1E0E0934208E1E5F8E0FA93EA93E0E023
:106D8A00EA93A4E3B0E00E9427CBE9E8F8E0FA939B
:106D9A00EA93E0E0EA93AAE1B0E00E9427CBE3EAB3
:106DAA00F8E0FA93EA93E0E0EA93AAE1B0E00E94FD
:106DBA0027CBE7EDF8E0FA93EA93E0E0EA93AAE159
:106DCA00B0E00E9427CBEEEDE0937A00E091430811
:106DDA00E07FE560E093430808950A921A928A9345
:106DEA00AA93BA93EA93FA93EFB7EA93E091420827
:106DFA00F0E0E130A0E0FA0739F4EFECE0937A0032
:106E0A00E2E0E0934208ECC0E230A0E0FA0709F0C1
:106E1A00E7C046B0E0914408EF5FE0934408E150D0
:106E2A00A0914408A731D0F4E0914408E770E869DA
:106E3A00E8B9A83010F443980AC0A0914408A031D8
:106E4A0010F4449804C0E3E0E0937C004798EEEC29
:106E5A00E0937A00E1E0E093420835C0A09144084B
:106E6A00A73161F4E1E0E0937C00E8E9E8B980E564
:106E7A008A95F1F7EFECE0937A0025C0A0914408D7
:106E8A00A83151F4E2E0E0937C0080E58A95F1F7BD
:106E9A00EFECE0937A0017C0E0E9E8B9E0E0E093AC
:106EAA004408E0937C00EEECE0937A00E1E0E093A2
:106EBA004208A0914508A03130F4E0914508EF5FFF
:106ECA00E0934508E150A0914408A13010F0A831A0
:106EDA0008F02DC0E0914408E770E093DA0DA7E4CA
:106EEA00B8E0F0E0EA0FFB1F4082E091DA0DE030F3
:106EFA0031F4E0914608EF5FE0934608E150A9E8D3
:106F0A00B8E0E0914408F0E0AE0FBF1FEC91E4292D
:106F1A00EC93A3EAB8E0E0914408F0E0EA0FFB1F23
:106F2A000F01A081E42DE095EA2BD001EC93A0910A
:106F3A004508A03108F054C0ADEBB8E0E091440830
:106F4A00F0E0AE0FBF1FEC91E093DA0DE09178000C
:106F5A00F0917900A091DA0DB0E0AE17BF0798F46E
:106F6A00A1E5B8E0E0914408F0E0EE0FFF1FEA0F58
:106F7A00FB1F0F01DF01ED91FD91DF01E091780028
:106F8A00F091790011C0A1E5B8E0E0914408F0E081
:106F9A00EE0FFF1FEA0FFB1F0F01DF01ED91FD91BD
:106FAA00DF01E091DA0DF0E0EA0FFB1FD001ED936B
:106FBA00FC93A0914408A13140F4A0917800B091CB
:106FCA007900A03FE3E0BE0708F40AC0A7EDB8E0E5
:106FDA00E0914408F0E0AE0FBF1FEC91EF5FEC9335
:106FEA00E991EFBFF991E991B991A9918991199024
:106FFA00099018951A931A2F103041F05C988BE07B
:10700A008A95F1F75C9A8BE08A95F1F72898EDB5A5
:10701A00E093A50DE0E4EEBDEDB5E7FFFDCFE5E0B9
:10702A00EEBDEDB5E7FFFDCFE8E0EEBDEDB5E7FF5C
:10703A00FDCF289AE091F508EF7BE093F508A5E7E4
:10704A00B2E00E941FD4E170A5EFB8E0E170E795C5
:10705A00E0E0E7950E2EEC91EF77E029EC93E091D2
:10706A00F508E860E093F508E460E093F5082898ED
:10707A00EDB5E093A50DE0E4EEBDEDB5E7FFFDCF7C
:10708A00EAE0EEBDEDB5E7FFFDCFE091F508EEBD14
:10709A00EDB5E7FFFDCF289A2898EDB5E093A50D49
:1070AA00E0E4EEBDEDB5E7FFFDCFE0E0EEBDEDB506
:1070BA00E7FFFDCFE4E0EEBDEDB5E7FFFDCF289A8F
:1070CA000C946F3CA091F208A13030F0E091F208E4
:1070DA00E150E093F20818C0E3E6E093F20828983A
:1070EA00EDB5E093A50DE0E4EEBDEDB5E7FFFDCF0C
:1070FA00EAE0EEBDEDB5E7FFFDCFE091F508EEBDA4
:10710A00EDB5E7FFFDCF289AA091F308A13038F03A
:10711A00E091F308E150E093F308EF5F2DC0E3E656
:10712A00E093F3082898EDB5E093A50DE2E4EEBDEF
:10713A00EDB5E7FFFDCFEAE0EEBDEDB5E7FFFDCF28
:10714A00E091F708EEBDEDB5E7FFFDCF289A289844
:10715A00EDB5E093A50DE2E4EEBDEDB5E7FFFDCF99
:10716A00E0E0EEBDEDB5E7FFFDCFE091F608EEBD3C
:10717A00EDB5E7FFFDCF289AA091F408A13038F0C9
:10718A00E091F408E150E093F408EF5F2DC0E3E6E4
:10719A00E093F4082898EDB5E093A50DE4E4EEBD7C
:1071AA00EDB5E7FFFDCFEAE0EEBDEDB5E7FFFDCFB8
:1071BA00E091F908EEBDEDB5E7FFFDCF289A2898D2
:1071CA00EDB5E093A50DE4E4EEBDEDB5E7FFFDCF27
:1071DA00E0E0EEBDEDB5E7FFFDCFE091F808EEBDCA
:1071EA00EDB5E7FFFDCF289A08950E942AD2589A52
:1071FA00509AE091FA08E07CE093FA08E9B1E3706A
:10720A00E330A9F0E0E0E093BC0010E0E9B1E370FC
:10721A00E33011F01A3008F00AC058988BE08A95CA
:10722A00F1F7589A8BE08A95F1F71F5FEFCFEFE0FD
:10723A00E093B800E4EAE093BC0020E030E0E0919B
:10724A00BC00E07821F42436E0E03E0708F003C0F1
:10725A002F5F3F4FF4CFE091B900E87FE83009F0A3
:10726A0052C0E0E9E093BB00E4E8E093BC0020E010
:10727A0030E0E091BC00E07821F42436E0E03E07FB
:10728A0008F003C02F5F3F4FF4CFE091B900E87FC9
:10729A00E831C9F5E1E0E093BB00E4E8E093BC0023
:1072AA0020E030E0E091BC00E07821F42436E0E010
:1072BA003E0708F003C02F5F3F4FF4CFE091B900BB
:1072CA00E87FE83201F5E1E6E093BB00E4E9E09308
:1072DA00BC0020E030E0E091BC00E07821F42436E4
:1072EA00E0E03E0708F003C02F5F3F4FF4CFE09184
:1072FA00B900E87FE83239F4E0E0E093BC0058983E
:10730A0050980C94CB3EE4E9E093BC00A2E0B0E0D4
:10731A000E94F3D5E0E0E093BC00589850980C9492
:10732A00CB3E0E9428D2E091FA08EF73E13030F0A8
:10733A00AAEFB8E080E0EFE30E94E5D3589A509AAA
:10734A00E9B1E370E330A9F0E0E0E093BC0010E0BB
:10735A00E9B1E370E33011F01A3008F00AC0589826
:10736A008BE08A95F1F7589A8BE08A95F1F71F5FBF
:10737A00EFCFE091FA08EF7309F0D1C0E091FA0873
:10738A00E07CE560E093FA08EFE0E093B800E4EA15
:10739A00E093BC0020E030E0E091BC00E07821F40A
:1073AA002436E0E03E0708F003C02F5F3F4FF4CFDA
:1073BA00E091B900E87FE83009F088C1E0E9E0939C
:1073CA00BB00E4E8E093BC0020E030E0E091BC00C0
:1073DA00E07821F42436E0E03E0708F003C02F5F8E
:1073EA003F4FF4CFE091B900E87FE83109F06EC170
:1073FA00E1E0E093BB00E4E8E093BC0020E030E089
:10740A00E091BC00E07821F42436E0E03E0708F081
:10741A0003C02F5F3F4FF4CFE091B900E87FE83215
:10742A0009F054C1E0E6E093BB00E4E8E093BC0055
:10743A0020E030E0E091BC00E07821F42436E0E07E
:10744A003E0708F003C02F5F3F4FF4CFE091B90029
:10745A00E87FE83209F03AC1E4EAE093BC0020E0B0
:10746A0030E0E091BC00E07821F42436E0E03E0709
:10747A0008F003C02F5F3F4FF4CFE091B900E87FD7
:10748A00E03109F023C1E0E9E093BB00E4E8E093CE
:10749A00BC0020E030E0E091BC00E07821F4243622
:1074AA00E0E03E0708F003C02F5F3F4FF4CFE091C2
:1074BA00B900E87FE83109F009C1E0E0E093BB00D8
:1074CA00E4E8E093BC0020E030E0E091BC00E07822
:1074DA0021F42436E0E03E0708F003C02F5F3F4F57
:1074EA00F4CFE091B900E87FE83209F0EFC0E4E9AF
:1074FA00E093BC0020E030E0E091BC00E07821F4A9
:10750A002436E0E03E0708F003C02F5F3F4FF4CF78
:10751A00E091FA08E07CEE61E093FA08D6C0E4EA6A
:10752A00E093BC0020E030E0E091BC00E07821F478
:10753A002436E0E03E0708F003C02F5F3F4FF4CF48
:10754A00E091B900E87FE83009F0C0C0E1E9E093D2
:10755A00BB00E4E8E093BC0020E030E0E091BC002E
:10756A00E07821F42436E0E03E0708F003C02F5FFC
:10757A003F4FF4CFE091B900E87FE03409F0A6C0AC
:10758A00E4ECE093BC0020E030E0E091BC00E0785D
:10759A0021F42436E0E03E0708F003C02F5F3F4F96
:1075AA00F4CFE091B900E87FE03509F08FC040914F
:1075BA00BB005527E4E8E093BC00FA010E94A2D27E
:1075CA00AF0120E030E0E091BC00E07821F42436FD
:1075DA00E0E03E0708F003C02F5F3F4FF4CFE09191
:1075EA00B900E87FE83509F071C0E091BB00F0E02E
:1075FA000E94ABD24E2B5F2BE4E9E093BC0053FD13
:10760A00506F20E030E0E091BC00E07821F42436AD
:10761A00E0E03E0708F003C02F5F3F4FF4CF4093EE
:10762A00FC085093FD08A091FC08B091FD08E0E128
:10763A00F0E00E9436D3E093B20DA6E3B1E00E94D7
:10764A001FD40E2FE2EEE017E4F4E091BF0DE03014
:10765A0089F0A091B20DE02FF0E0E7FDFFEF31973E
:10766A00B0E0A7FDBFEFAE17BF071CF4E0E0E09360
:10767A00BF0D07C0A091B20DA0171CF0E1E0E09386
:10768A00BF0DA7E3B1E00E941FD40E2FE2EEE01770
:10769A00E4F4E091C00DE03089F0A091B20DE02F42
:1076AA00F0E0E7FDFFEF3197B0E0A7FDBFEFAE17BF
:1076BA00BF071CF4E0E0E093C00D07C0A091B20D33
:1076CA00A0171CF0E1E0E093C00D09C0E091FA08B0
:1076DA00E07CE560E093FA08E4E9E093BC000E94EC
:1076EA002FD2269608951A93F298F398F498F5985B
:1076FA00E0917E00E97FE0937E00E7E9F7E0FA9304
:10770A00EA93E0E0EA93A8E1B0E00E9427CB10E018
:10771A001C3008F05AC0E12FA7E9B7E0F0E0EE0FFD
:10772A00FF1FEA0FFB1F0F01AAEBB1E0EE27A10F23
:10773A00BE1F0E941FD4E370D001E370EE0FEE0F5C
:10774A000E2EEC91E37FE029EC93E12FA7E9B7E055
:10775A00F0E0EE0FFF1FEA0FFB1F0F01AAEBB1E0EB
:10776A00EE27A10FBE1F0E941FD4E695E695E17091
:10777A00D001E170EE0F0E2EEC91ED7FE029EC9333
:10778A00E12FA7E9B7E0F0E0EE0FFF1FAE0FBF1F32
:10779A00EC91F0E00E94B8D2E370F070309741F4B7
:1077AA00123011F0133011F4F49A01C0F29A0BC09E
:1077BA00E130A0E0FA0739F4123011F0133011F475
:1077CA00F59A01C0F39A1F5FA3CFE89423F8EDB3AB
:1077DA00EF73EDBBE0919707EC70EC3019F4EE9A79
:1077EA00689423F8E0919907EC70EC3019F4EF9A59
:1077FA00689423F8E0919B07EC70E83031F0AEEC26
:10780A00B1E00E941FD4E37051F0E0917E00E26083
:10781A00E0937E00E1E0E0934F08F59AF498E09156
:10782A009D07EC70E83031F0AEECB1E00E941FD455
:10783A00EC7051F0E0917E00E460E0937E00E1E0BC
:10784A00E0935008F59AF498F29B02C0F39B01C0AA
:10785A0002C0169A01C01698F49B02C0F59B01C09B
:10786A0002C0159A01C0159835C01A93E4EBF3E0EB
:10787A0060E070E00E94B1D380E00E94AFD124960C
:10788A0010E01C3020F5ECEBF3E060E070E00E94C1
:10789A00B1D3E12FF0E031966F2F660F660B762F8A
:1078AA000E94B1D3E12FA7E9B7E0F0E0EE0FFF1F86
:1078BA00AE0FBF1FEC91E170FF27662777270E9462
:1078CA00B1D388E00E94AFD12C961F5FDACFAAE02D
:1078DA000E949596199108950E942AD23A2FE09112
:1078EA00B40DE17011F0303009F44FC2373310F0A3
:1078FA003C3308F006C0E32FF0E0F797E655F64F61
:10790A003081313059F4A091BC0DB091BD0DA03732
:10791A00E7E1BE0710F0E1E039C237C2333010F0B8
:10792A003F3008F00CC0E32FF0E03397A7E9B7E047
:10793A00EE0FFF1FAE0FBF1FEC91E17027C23F3061
:10794A0010F03F3108F020C03F31E8F4E32FF0E0B7
:10795A003F97AAE0B0E00E94DDD2E65FF64FE081F1
:10796A00E17079F0E32FF0E03F97AAE0B0E00E94DF
:10797A00DDD2E65FF64FE081E077E03410F4E1E033
:10798A0001C0E0E003C201C23C3310F0303708F016
:10799A0014C0ABE6B4E0E32FF0E0FC97BD01AEE023
:1079AA00B0E00E94DDD2DB01AE0FBF1F1C96EC9146
:1079BA00EE1FE0E0EE1FE170E9C1303710F0343815
:1079CA0008F011C0A9EFBCE0E32FF0E0E057F04067
:1079DA000E94A4D2AE0FBF1FEC91E295EF70E6951C
:1079EA00E695E170D3C1343810F0383908F00EC08A
:1079FA00E32FF0E0E458F040A3E0B0E00E94DDD2CB
:107A0A00ED5BF84FE081E695E170C0C1383910F0BE
:107A1A003D3908F00EC0E32FF0E0E859F040AFE737
:107A2A00B7E00E94A6D2AE0FBF1F1396EC91E17089
:107A3A00ADC13D39B9F4E091990DEF70E33079F0B9
:107A4A00E091990DEF70E43051F0E091990DEF70EB
:107A5A00E13029F0E091990DEF70E63011F4E1E0A0
:107A6A0095C193C13E3969F4E091990DEF70E53003
:107A7A0029F0E091990DEF70E23011F4E1E086C14E
:107A8A0084C13F3910F0373B08F06FC0E32FEF593C
:107A9A001E2FFF2766277727E25EFE4F6F4F6BBFC9
:107AAA000691E12FFF2766277727EA5CFE4F6F4F83
:107ABA006BBF1691113449F5A3E00A9FF001E15119
:107ACA00F64FE081E07FE03111F4E1E05FC1A3E02D
:107ADA000A9FF001E151F64FE081E07FE03288F041
:107AEA000A9FF001E151F64FE081E770E33041F07F
:107AFA000A9FF001E151F64FE081E770E43009F4A2
:107B0A0001C002C0E1E042C12FC0123401F5A3E076
:107B1A000A9FF001E151F64FE081E07FE03211F473
:107B2A00E1E034C1A3E00A9FF001E151F64FE081A0
:107B3A00E07FE03340F00A9FF001E151F64FE08127
:107B4A00E770E43009F002C0E1E020C10DC013344F
:107B5A0059F4A3E00A9FF001E151F64FE081E07F7A
:107B6A00E03311F4E1E012C110C13A3B10F0363CA7
:107B7A0008F009C0E32FEA5B0E2FF0E0E155F84F59
:107B8A00E081E17003C1373C10F03F3D08F0D6C0F8
:107B9A00E091BB07F0E0E130A0E0FA0709F064C029
:107BAA003F3C88F4E32FE75C1E2FA1E0B0E00E947F
:107BBA0052D2A091C507B0E0EA23FB23309711F017
:107BCA00E1E0E4C050C0E091BC07EF77EF3099F4F0
:107BDA00363D80F4E32FEF5C1E2FA1E0B0E00E9457
:107BEA0052D2A091C607B0E0EA23FB23309711F0E6
:107BFA00E1E0CCC038C0333D88F4E32FEF5C1E2FA0
:107C0A00A1E0B0E00E9452D2A091C607B0E0EA23F8
:107C1A00FB23309711F0E1E0B9C025C03B3D88F461
:107C2A00E32FE35D1E2FA1E0B0E00E9452D2A091A3
:107C3A00DE07B0E0EA23FB23309711F0E1E0A6C0AB
:107C4A0012C03F3D80F4E32FEB5D1E2FA1E0B0E0B0
:107C5A000E9452D2A091DF07B0E0EA23FB233097BB
:107C6A0011F0E1E093C069C0E230A0E0FA0721F028
:107C7A00E330A0E0FA0789F4A2EEB7E0E32FF0E0E0
:107C8A00E75CF0400E94A6D2AE0FBF1F1296EC919D
:107C9A00E17011F0E1E07AC050C0E430A0E0FA07E8
:107CAA0009F04BC03F3C88F4E32FE75C1E2FA1E0AC
:107CBA00B0E00E9452D2A091C307B0E0EA23FB23AE
:107CCA00309711F0E1E062C038C0333D88F4E32F09
:107CDA00EF5C1E2FA1E0B0E00E9452D2A091C6072D
:107CEA00B0E0EA23FB23309711F0E1E04FC025C052
:107CFA003B3D88F4E32FE35D1E2FA1E0B0E00E9434
:107D0A0052D2A091EB07B0E0EA23FB23309711F09F
:107D1A00E1E03CC012C03F3D80F4E32FEB5D1E2F33
:107D2A00A1E0B0E00E9452D2A091EE07B0E0EA23AF
:107D3A00FB23309711F0E1E029C027C03F3D39F419
:107D4A00E091BF0DE03011F0E1E020C01EC0303EEE
:107D5A0039F4E091C00DE03011F0E1E017C015C030
:107D6A00323059F4A5E3B1E00E941FD4A091B30DBB
:107D7A00AE1710F0E1E00AC008C0313E31F4E091DC
:107D8A006404E87011F0E1E001C0E0E00E9431D241
:107D9A002496089523970E9428D2F39904C0F5994E
:107DAA0002C022FE01C003C0689422F8E1C4F09B1D
:107DBA0010C0E0919707E1704E2FE0919907E170AA
:107DCA00E887E0919B07E170EF83E0919D07E170FE
:107DDA00EE8322FE47C0E0919707EC7009F041C09C
:107DEA0010919807669B02C0F19B01C027C0E091E1
:107DFA009707E07111F0123008F001C012E012305A
:107E0A0010F41F5F1AC01230B9F4E0919707E270BC
:107E1A0071F0E0919707E17021F0E0919707EE7F0A
:107E2A0003C0E0919707E160E093970705C0E091EE
:107E3A009707E160E09397071FE011C01B3010F02D
:107E4A0011500DC0113020F0E0919707E27009F04F
:107E5A0005C0E0919707EE7FE093970710E0109333
:107E6A00980743C0E0919707EC70E430F1F5109160
:107E7A009807669B12C01B3010F011500DC01130CC
:107E8A0020F0E0919707E27009F005C0E0919707AA
:107E9A00EE7FE093970710E026C0E0919707E07124
:107EAA0011F0123008F001C012E0123010F41F5F16
:107EBA0019C01230B9F4E0919707E27071F0E091BD
:107ECA009707E17021F0E0919707EE7F03C0E091F8
:107EDA009707E160E093970705C0E0919707E16093
:107EEA00E09397071FE01093980722FE51C0E09194
:107EFA009907EC7009F04BC010919A07679B02C072
:107F0A00F19B01C031C0E0919907E07111F0123084
:107F1A0008F001C012E0123010F41F5F24C0E09193
:107F2A009907E07111F0123008F001C012E0123026
:107F3A00C9F4E0919907E27081F0E0919907E17044
:107F4A0031F0A9E9B7E0EC91EE7FEC9305C0E0913E
:107F5A009907E160E093990705C0E0919907E1600C
:107F6A00E09399071FE011C01B3010F011500DC0AB
:107F7A00113020F0E0919907E27009F005C0A9E9F3
:107F8A00B7E0EC91EE7FEC9310E010939A073DC0B6
:107F9A00E0919907EC70E430C1F510919A07679B5C
:107FAA0012C01B3010F011500DC0113020F0E091BA
:107FBA009907E27009F005C0A9E9B7E0EC91EE7FF4
:107FCA00EC9310E020C0123010F41F5F1CC0123076
:107FDA00C9F4E0919907E27081F0E0919907E170A4
:107FEA0031F0A9E9B7E0EC91EE7FEC9305C0E0919E
:107FFA009907E160E093990705C0E0919907E1606C
:10800A00E09399071FE010939A07E0919B07EC70A1
:10801A00E830E1F5E0918508F091860834960E94EF
:10802A00B6D25E2F10919C07A8ECB1E00E941FD433
:10803A003E2FA9ECB1E00E941FD42E2F321728F54B
:10804A00E0919B07E17089F0351768F01B3010F05A
:10805A00115008C0113028F0ABE9B7E0EC91EE7F7F
:10806A00EC9310E001C01FE010C0521768F0123004
:10807A0010F41F5F08C0123029F4E0919B07E160F9
:10808A00E0939B071FE001C010E08CC022FE46C0AF
:10809A00E0919B07EC7009F040C010919C07799B16
:1080AA0012C01B3010F011500DC0113020F0E091B9
:1080BA009B07E27009F005C0ABE9B7E0EC91EE7FEF
:1080CA00EC9310E028C0E0919B07E07111F01230A8
:1080DA0008F001C012E0123010F41F5F1CC0123009
:1080EA00C9F4E0919B07E27081F0E0919B07E1708F
:1080FA0031F0ABE9B7E0EC91EE7FEC9305C0E0918B
:10810A009B07E160E0939B0705C0E0919B07E16054
:10811A00E0939B071FE010939C0746C0E0919B07E2
:10812A00EC70E43009F040C010919C07799B29C09B
:10813A00E0919B07E07111F0123008F001C012E0E3
:10814A00123010F41F5F1CC01230C9F4E0919B0773
:10815A00E27081F0E0919B07E17031F0ABE9B7E0A2
:10816A00EC91EE7FEC9305C0E0919B07E160E09310
:10817A009B0705C0E0919B07E160E0939B071FE026
:10818A0011C01B3010F011500DC0113020F0E091D9
:10819A009B07E27009F005C0ABE9B7E0EC91EE7F0E
:1081AA00EC9310E010939C07E0919D07EC70E83087
:1081BA00E1F5E0918708F091880834960E94B6D2DA
:1081CA005E2F10919E07ACECB1E00E941FD43E2FA7
:1081DA00ADECB1E00E941FD42E2F321728F5E091A2
:1081EA009D07E17089F0351768F01B3010F01150C7
:1081FA0008C0113028F0ADE9B7E0EC91EE7FEC93BE
:10820A0010E001C01FE010C0521768F0123010F4DD
:10821A001F5F08C0123029F4E0919D07E160E093E6
:10822A009D071FE001C010E084C022FE42C0E09119
:10823A009D07EC70E9F510919E077A9B0FC01B30E1
:10824A0010F011500AC0E0919D07E27029F4ADE9DF
:10825A00B7E0EC91EE7FEC9310E028C0E0919D0727
:10826A00E07111F0123008F001C012E0123010F47F
:10827A001F5F1CC01230C9F4E0919D07E27081F0C3
:10828A00E0919D07E17031F0ADE9B7E0EC91EE7F46
:10829A00EC9305C0E0919D07E160E0939D0705C05E
:1082AA00E0919D07E160E0939D071FE010939E0710
:1082BA0042C0E0919D07EC70E430E9F510919E0709
:1082CA007A9B29C0E0919D07E07111F0123008F005
:1082DA0001C012E0123010F41F5F1CC01230C9F442
:1082EA00E0919D07E27081F0E0919D07E17031F025
:1082FA00ADE9B7E0EC91EE7FEC9305C0E0919D0704
:10830A00E160E0939D0705C0E0919D07E160E0937D
:10831A009D071FE00EC01B3010F011500AC0E091FB
:10832A009D07E27029F4ADE9B7E0EC91EE7FEC939A
:10833A0010E010939E07F09B5FC0E0919707E170F1
:10834A00E41791F0E3ECF3E060E070E00E94B1D34F
:10835A00E0919707E170FF27662777270E94B1D33C
:10836A0084E00E94AFD12896E0919907E170A88530
:10837A00EA1791F0EDECF3E060E070E00E94B1D30F
:10838A00E0919907E170FF27662777270E94B1D30A
:10839A0084E00E94AFD12896E0919B07E170AF81FB
:1083AA00EA1791F0E7EDF3E060E070E00E94B1D3E4
:1083BA00E0919B07E170FF27662777270E94B1D3D8
:1083CA0084E00E94AFD12896E0919D07E170AE81CA
:1083DA00EA1791F0E1EEF3E060E070E00E94B1D3B9
:1083EA00E0919D07E170FF27662777270E94B1D3A6
:1083FA0084E00E94AFD1289654E05C3008F084C132
:10840A00E52FA7E9B7E0F0E0EE0FFF1FAE0FBF1FA1
:10841A00EC91E1704E2F22FEA5C0E52FA7E9B7E047
:10842A00F0E0EE0FFF1FAE0FBF1FEC91EC7009F0EA
:10843A0098C0F19B02C000E011C0A7E4B8E0E52FA4
:10844A00FF2766277727EC56FF4F6F4F6BBFE691E2
:10845A00F0E0AE0FBF1FEC91E0720E2FE52FA7E9F7
:10846A00B7E0F0E0EE0FFF1FAE0FBF1F11961C9191
:10847A00003009F44FC0E52FA7E9B7E0F0E0EE0FAE
:10848A00FF1FAE0FBF1FEC91E07111F0123008F020
:10849A0001C012E0123010F41F5F3BC01230C1F568
:1084AA00E52FA7E9B7E0F0E0EE0FFF1FAE0FBF1F01
:1084BA00EC91E27011F1E52FA7E9B7E0F0E0EE0FD9
:1084CA00FF1FAE0FBF1FEC91E17059F0E52FA7E92E
:1084DA00B7E0F0E0EE0FFF1FAE0FBF1FEC91EE7F8B
:1084EA000AC0E52FA7E9B7E0F0E0EE0FFF1FAE0FD5
:1084FA00BF1FEC91E160EC930BC0E52FA7E9B7E051
:10850A00F0E0EE0FFF1FAE0FBF1FEC91E160EC939E
:10851A001FE01EC01B3010F011501AC0113058F065
:10852A00E52FA7E9B7E0F0E0EE0FFF1FAE0FBF1F80
:10853A00EC91E27009F00BC0E52FA7E9B7E0F0E093
:10854A00EE0FFF1FAE0FBF1FEC91EE7FEC9310E012
:10855A00E52FA7E9B7E0F0E0EE0FFF1FEA0FFB1FD8
:10856A001183A0C0E52FA7E9B7E0F0E0EE0FFF1FE7
:10857A00AE0FBF1FEC91EC70E43009F093C0A7E492
:10858A00B8E0E52FFF2766277727EC56FF4F6F4F96
:10859A006BBFE691F0E0AE0FBF1FEC91E0720E2FB9
:1085AA00E52FA7E9B7E0F0E0EE0FFF1FAE0FBF1F00
:1085BA0011961C910030F9F01B3010F011501AC0BE
:1085CA00113058F0E52FA7E9B7E0F0E0EE0FFF1FF2
:1085DA00AE0FBF1FEC91E27009F00BC0E52FA7E9BF
:1085EA00B7E0F0E0EE0FFF1FAE0FBF1FEC91EE7F7A
:1085FA00EC9310E04EC0E52FA7E9B7E0F0E0EE0FEC
:10860A00FF1FAE0FBF1FEC91E07111F0123008F09E
:10861A0001C012E0123010F41F5F3BC01230C1F5E6
:10862A00E52FA7E9B7E0F0E0EE0FFF1FAE0FBF1F7F
:10863A00EC91E27011F1E52FA7E9B7E0F0E0EE0F57
:10864A00FF1FAE0FBF1FEC91E17059F0E52FA7E9AC
:10865A00B7E0F0E0EE0FFF1FAE0FBF1FEC91EE7F09
:10866A000AC0E52FA7E9B7E0F0E0EE0FFF1FAE0F53
:10867A00BF1FEC91E160EC930BC0E52FA7E9B7E0CF
:10868A00F0E0EE0FFF1FAE0FBF1FEC91E160EC931D
:10869A001FE0E52FA7E9B7E0F0E0EE0FFF1FEA0FB2
:1086AA00FB1F1183F09B2EC0E52FA7E9B7E0F0E08E
:1086BA00EE0FFF1FAE0FBF1FEC91E170E41711F12F
:1086CA00EBEEF3E060E070E00E94B1D3E52FF0E05A
:1086DA0031966F2F660F660B762F0E94B1D3E52F66
:1086EA00A7E9B7E0F0E0EE0FFF1FAE0FBF1FEC9156
:1086FA00E170FF27662777270E94B1D388E00E949E
:10870A00AFD12C965F5F79CEF39B06C0F29904C075
:10871A00F59B02C0F49B01C002C0E89414C0F3990F
:10872A0006C0F29B04C0F59902C0F49901C002C0C8
:10873A00689409C0A0E022FCA1E0E1E0EA27E894FD
:10874A00EE2309F0689422F8F39B02C0F29901C063
:10875A0005C022FE02C0169A01C01698F59B02C0F7
:10876A00F49901C005C022FE02C0159A01C01598ED
:10877A000E942FD22996089524970E9428D223FE78
:10878A0093C0A091DF0DA13030F0E091DF0DE150F0
:10879A00E093DF0D89C0E2E0E093DF0DF894E09109
:1087AA00DB0DF091DC0DE0939307F0939407E0E082
:1087BA00E093DB0DE093DC0DE091DD0DF091DE0D31
:1087CA00E0939507F0939607E0E0E093DD0DE093E0
:1087DA00DE0D7894E0919707EC70EC3051F5A0919A
:1087EA009307B091940788279927E9E00E9474D2E9
:1087FA00DF01CB01EDE9F0E060E070E00E943BD3DD
:10880A00E0939307F0939407ADE7B9E00E941BD475
:10881A00A0919307B0919407AE17BF0720F0E0919B
:10882A009707E16003C0E0919707EE7FE09397070F
:10883A0005C0E0E0E0939307E0939407E09199077D
:10884A00EC70EC3061F5A0919507B09196078827F6
:10885A009927E9E00E9474D2DF01CB01EDE9F0E04B
:10886A0060E070E00E943BD3E0939507F09396078F
:10887A00AFE7B9E00E941BD4A0919507B091960783
:10888A00AE17BF0730F0E0919907E160E0939907CE
:10889A0005C0A9E9B7E0EC91EE7FEC9305C0E0E0F2
:1088AA00E0939507E0939607AEECB1E00E941FD4DF
:1088BA00E3703E2F303009F4B9C0AFECB1E00E944A
:1088CA001FD42E2FA0EDB1E00E941FD45E2F3130AD
:1088DA0029F4E0918508F091860804C0E0918708A0
:1088EA00F091880834960E94B8D2E887F98710E098
:1088FA00163008F09BC0A1EDB1E0EE27A10FBE1F14
:10890A000E941FD40E2F013008F48EC0F0E0EE83CF
:10891A00FF83EE0FFF1FEE83FF83E12FF0E0E155A7
:10892A00F84FE081E17009F443C0E22FF0E0A88536
:10893A00B985AE0FBF1FEE27A50FBE1FEE81FF81BF
:10894A00AE17BF0778F0E22FF0E0AE81BF81AE0F1D
:10895A00BF1FE52FF0E0EA0FFB1FA885B985EA17CC
:10896A00FB0728F5F09B1CC0E6EFF3E060E070E03F
:10897A000E94B1D3E12FF0E031966F2F660F660B9C
:10898A00762F0E94B1D3A889B989EAE00E9405D35B
:10899A00662777270E94B1D388E00E94AFD12C9630
:1089AA00A12FB0E0A155B84FEC91EE7FEC933CC0FB
:1089BA00E22FF0E0A885B985AE0FBF1FEE81FF81D7
:1089CA00AE17BF0758F0E22FF0E0AE81BF81EA0F81
:1089DA00FB1FA885B985EA17FB0708F425C0F09B99
:1089EA001CC0EAE0F4E060E070E00E94B1D3E12F3D
:1089FA00F0E031966F2F660F660B762F0E94B1D387
:108A0A00A889B989EAE00E9405D3662777270E94D8
:108A1A00B1D388E00E94AFD12C96A12FB0E0A15526
:108A2A00B84FEC91E160EC931F5F62CFAEECB1E01E
:108A3A000E941FD4E695E695E3703E2F303009F484
:108A4A00B9C0AFECB1E00E941FD42E2FA0EDB1E067
:108A5A000E941FD45E2F313029F4E0918508F091ED
:108A6A00860804C0E0918708F091880834960E942D
:108A7A00B8D2E887F98716E01C3008F09BC0A1ED50
:108A8A00B1E0EE27A10FBE1F0E941FD40E2F0130A6
:108A9A0008F48EC0F0E0EE83FF83EE0FFF1FEE8333
:108AAA00FF83E12FF0E0E155F84FE081E17009F42E
:108ABA0043C0E22FF0E0A885B985AE0FBF1FEE27AD
:108ACA00A50FBE1FEE81FF81AE17BF0778F0E22F18
:108ADA00F0E0AE81BF81AE0FBF1FE52FF0E0EA0FD5
:108AEA00FB1FA885B985EA17FB0728F5F09B1CC070
:108AFA00E6EFF3E060E070E00E94B1D3E12FF0E02E
:108B0A0031966F2F660F660B762F0E94B1D3A88914
:108B1A00B989EAE00E9405D3662777270E94B1D374
:108B2A0088E00E94AFD12C96A12FB0E0A155B84F92
:108B3A00EC91EE7FEC933CC0E22FF0E0A885B9857A
:108B4A00AE0FBF1FEE81FF81AE17BF0758F0E22FAD
:108B5A00F0E0AE81BF81EA0FFB1FA885B985EA174D
:108B6A00FB0708F425C0F09B1CC0EAE0F4E060E0D3
:108B7A0070E00E94B1D3E12FF0E031966F2F660FBB
:108B8A00660B762F0E94B1D3A889B989EAE00E94C0
:108B9A0005D3662777270E94B1D388E00E94AFD118
:108BAA002C96A12FB0E0A155B84FEC91E160EC935F
:108BBA001F5F62CF0E942FD22A96089560971A9358
:108BCA00FE013196FA93EA93E0E0EA93A0E1B0E07D
:108BDA000E9427CB10E01C3008F03FC0AAEBB1E09E
:108BEA00EE27A10FBE1F0E941FD4EC7F0E943BD428
:108BFA00AAEBB1E0EE27A10FBE1F0E941FD4EB7FA4
:108C0A000E943BD4FE013196FA93EA93EDE1F4E037
:108C1A0060E070E00E94B1D3E12FF0E031966F2F4F
:108C2A00660F660B762F0E94B1D384E00E9474D13E
:108C3A002A96E12FF0E0A0E6B9E30E94A2D2EA0F59
:108C4A00FB1FFA93EA93FE013396FA93EA93A0E1A3
:108C5A000E948229A8951F5FBECFA6ECB1E0E0E092
:108C6A000E943BD4A7ECB1E0EAEF0E943BD4A8EC07
:108C7A00B1E0E4E60E943BD4A9ECB1E0E6E90E9447
:108C8A003BD4AAECB1E0E0E00E943BD4ABECB1E00B
:108C9A00EAEF0E943BD4ACECB1E0E4E60E943BD49C
:108CAA00ADECB1E0E6E90E943BD4AEECB1E00E9443
:108CBA001FD4EC7F0E943BD4AEECB1E00E941FD4DB
:108CCA00E37F0E943BD4AEECB1E00E941FD4EF7068
:108CDA000E943BD4AFECB1E0E8E10E943BD4A0EDA6
:108CEA00B1E0E2E00E943BD4E1EDF1E0FA93EA93CD
:108CFA00ACE00E94EC2610E0163008F054C0FE01E9
:108D0A003196FA93EA93E7E2F4E060E070E00E94B9
:108D1A00B1D3E12FF0E031966F2F660F660B762FF5
:108D2A000E94B1D384E00E9474D12A96E12FF0E028
:108D3A00A0EDB3E40E94A2D2EA0FFB1FFA93EA93D2
:108D4A00FE013396FA93EA93A0E10E948229FE017A
:108D5A003196FA93EA93E3E3F4E060E070E00E946C
:108D6A00B1D3E12FF0E031966F2F660F660B762FA5
:108D7A000E94B1D384E00E9474D12A96E12FF0E0D8
:108D8A003696A0EDB3E40E94A2D2EA0FFB1FFA9333
:108D9A00EA93FE013396FA93EA93A0E10E948229AC
:108DAA00A8951F5FA9CF188161960895AA93BA93CF
:108DBA00EA93FA93EFB7EA93ABEDBDE008C0AA9342
:108DCA00BA93EA93FA93EFB7EA93ADEDBDE0ED916A
:108DDA00FD913196FE93EE93E991EFBFF991E991F6
:108DEA00B991A99118950E9428D2EBEBF7E0FA9372
:108DFA00EA93E0E0EA93A7E8B0E00E9427CBA8E371
:108E0A00B1E00E941FD4E093BB07E0E4F4E060E025
:108E1A0070E00E94B1D380E00E94AFD12496E09125
:108E2A00BB07F0E0E130A0E0FA0709F028C100E052
:108E3A00023008F007C1A9E2B8E0E02FF0E0BD0176
:108E4A00A1E7B0E00E94DDD2DB01AE0FBF1F0E9496
:108E5A001FD4E03009F4F4C0ACEBB7E0E02FF0E047
:108E6A00BD01A9E1B0E00E94DDD2E60FF71FFF9332
:108E7A00EF93A9E2B8E0E02FF0E0BD01A1E7B0E08E
:108E8A000E94DDD2DB01AE0FBF1F11960E941FD4D4
:108E9A00E295EF70AF91BF91EF770E2EEC91E078EB
:108EAA00E029EC93ACEBB7E0E02FF0E0BD01A9E1DB
:108EBA00B0E00E94DDD2DB01AE0FBF1F1296E5E0E3
:108ECA00EC9331E0E0E01E2F5E2F2E2F183008F0D1
:108EDA0040C0A9E2B8E0E02FF0E0BD01A1E7B0E0B0
:108EEA000E94DDD2DB01AE0FBF1F1E96E12FF0E01C
:108EFA000E94A4D2AE0FBF1F16960E941FD4F0E0A4
:108F0A00F695E795E370F070E130A0E0FA0721F0FA
:108F1A00E330A0E0FA0709F4232BA9E2B8E0E02F36
:108F2A00F0E0BD01A1E7B0E00E94DDD2DB01AE0FA7
:108F3A00BF1F1E96E12FF0E00E94A4D2AE0FBF1F02
:108F4A0016960E941FD4E17009F0532B1F5F330F4E
:108F5A00BDCFACEBB7E0E02FF0E0BD01A9E1B0E096
:108F6A000E94DDD2E60FF71F2187ACEBB7E0E02FB6
:108F7A00F0E0BD01A9E1B0E00E94DDD2E60FF71FE3
:108F8A00558331E0E0E05E2F2E2F1C3008F040C000
:108F9A00A9E2B8E0E02FF0E0BD01A1E7B0E00E944D
:108FAA00DDD2DB01AE0FBF1F1E96E12FF0E00E945B
:108FBA00A4D2AE0FBF1F16960E941FD4F0E0F695FA
:108FCA00E795E370F070E130A0E0FA0721F0E330B2
:108FDA00A0E0FA0709F4232BA9E2B8E0E02FF0E0B9
:108FEA00BD01A1E7B0E00E94DDD2DB01AE0FBF1FD9
:108FFA001E96E12FF0E00E94A4D2AE0FBF1F169674
:10900A000E941FD4E17009F0532B1F5F330FBDCFAD
:10901A00ACEBB7E0E02FF0E0BD01A9E1B0E00E94BF
:10902A00DDD2E60FF71F2287ACEBB7E0E02FF0E0C6
:10903A00BD01A9E1B0E00E94DDD2E60FF71F568319
:10904A000F5FF6CEE8E4F4E060E070E00E94B1D38E
:10905A00A9E2B8E00E941FD4FF27662777270E945B
:10906A00B1D3AAE9B8E00E941FD4FF276627772761
:10907A000E94B1D388E00E94AFD12C963DC0E23065
:10908A00A0E0FA0769F4E9E5F4E060E070E00E9424
:10909A00B1D380E00E94AFD124960E94CC562CC056
:1090AA00E330A0E0FA0769F4EBE6F4E060E070E090
:1090BA000E94B1D380E00E94AFD124960E94CC5680
:1090CA001BC0E430A0E0FA0769F4EBE7F4E060E0E3
:1090DA0070E00E94B1D380E00E94AFD124960E9432
:1090EA002C5F0AC0E3E8F4E060E070E00E94B1D3CC
:1090FA0080E00E94AFD124960E942FD2269608952E
:10910A00E0E0E093BB07A8E3B1E00E943BD40895F6
:10911A00BA93AA9325970E9428D2AB85BC85EC9175
:10912A00E07109F0E2C1EB85FC85A181EFE7EA2352
:10913A005E2F503009F4D9C130E0323008F0D5C181
:10914A00A9E2B8E0E32FF0E0BD01A1E7B0E00E9498
:10915A00DDD2DB01AE0FBF1F0E941FD45E1709F0DC
:10916A00C2C1ACEBB7E0E32FF0E0BD01A9E1B0E08A
:10917A000E94DDD2DB01AE0FBF1F1296EAE0EC932C
:10918A00EB85FC85A181B281E7E00E9463D2EE8380
:10919A00F0E0EE30A0E0FA0709F4A5C1E330A0E060
:1091AA00FA0709F0A0C1ACEBB7E0E32FF0E0BD018C
:1091BA00A9E1B0E00E94DDD2DB01AE0FBF1FEC9146
:1091CA00E07889F5ACEBB7E0E32FF0E0BD01A9E167
:1091DA00B0E00E94DDD2DB01AE0FBF1FEC91E06868
:1091EA00EC93ACEBB7E0E32FF0E0BD01A9E1B0E00E
:1091FA000E94DDD2DB01AE0FBF1F1196E0E0EC93B7
:10920A00EAE8F4E060E070E00E94B1D3E32FF0E016
:10921A0031966F2F660F660B762F0E94B1D384E0CA
:10922A000E94AFD12896ACEBB7E0E32FF0E0BD0186
:10923A00A9E1B0E00E94DDD2DB01AE0FBF1F12969A
:10924A00E1E1EC93ACEBB7E0E32FF0E0BD01A9E17B
:10925A00B0E00E94DDD2DB01AE0FBF1FEC91EF77C9
:10926A002E2FACEBB7E0E32FF0E0BD01A9E1B0E0AF
:10927A000E94DDD2DB01AE0FBF1F1996EC91E98780
:10928A00ACEBB7E0E32FF0E0BD01A9E1B0E00E944A
:10929A00DDD2DB01AE0FBF1F1796EC91E887ACEB6E
:1092AA00B7E0E32FF0E0BD01A9E1B0E00E94DDD212
:1092BA00DB01AE0FBF1F1596EC91EF83EB85FC85A2
:1092CA004581022F093008F008E010E0E1E0EA8762
:1092DA00101758F5EA85AF81EA23B1F0EA85E4234D
:1092EA0069F0EA85A885EA2341F4EA85A985EA278F
:1092FA00E987EA85A885EA2BE88705C0EA85E0952B
:10930A00A885EA23E8870CC0EA85E42321F0EA85E8
:10931A00A985EA2B04C0EA85E095A985EA23E987AD
:10932A001F5FEA85EE0FEA87D3CFACEBB7E0E32FF6
:10933A00F0E0BD01A9E1B0E00E94DDD2DB01AE0F91
:10934A00BF1F1996AC91E985EA17E9F0ACEBB7E0D3
:10935A00E32FF0E0BD01A9E1B0E00E94DDD2E60F03
:10936A00F71F3996A985A083ACEBB7E0E32FF0E0AD
:10937A00BD01A9E1B0E00E94DDD2DB01AE0FBF1F43
:10938A001396E0E0EC93ACEBB7E0E32FF0E0BD011D
:10939A00A9E1B0E00E94DDD2E60FF71F3796A88553
:1093AA00A083293008F49FC0ACEBB7E0E32FF0E0CC
:1093BA00BD01A9E1B0E00E94DDD2DB01AE0FBF1F03
:1093CA001A96EC91E987ACEBB7E0E32FF0E0BD0128
:1093DA00A9E1B0E00E94DDD2DB01AE0FBF1F1896F3
:1093EA00EC91E887ACEBB7E0E32FF0E0BD01A9E12F
:1093FA00B0E00E94DDD2DB01AE0FBF1F1696EC91E2
:10940A00EF83EB85FC854681E22FE8500E2F10E0B2
:10941A00E1E0EA87101758F5EA85AF81EA23B1F04F
:10942A00EA85E42369F0EA85A885EA2341F4EA8516
:10943A00A985EA27E987EA85A885EA2BE88705C08E
:10944A00EA85E095A885EA23E8870CC0EA85E42343
:10945A0021F0EA85A985EA2B04C0EA85E095A98569
:10946A00EA23E9871F5FEA85EE0FEA87D3CFACEBE1
:10947A00B7E0E32FF0E0BD01A9E1B0E00E94DDD240
:10948A00DB01AE0FBF1F1A96AC91E985EA17E9F026
:10949A00ACEBB7E0E32FF0E0BD01A9E1B0E00E9438
:1094AA00DDD2E60FF71F3A96A985A083ACEBB7E0A9
:1094BA00E32FF0E0BD01A9E1B0E00E94DDD2DB01BB
:1094CA00AE0FBF1F1396E0E0EC93ACEBB7E0E32FCF
:1094DA00F0E0BD01A9E1B0E00E94DDD2E60FF71F7E
:1094EA003896A885A0833F5F28CE0E942FD22D965A
:1094FA0008956F970E9428D2E0916304E07421F4E2
:10950A000E942FD2A596089540E0423010F00C94A4
:10951A001455ACEBB7E0E42FF0E0BD01A9E1B0E0EF
:10952A000E94DDD2DB01AE0FBF1F1296AC91A130B3
:10953A0010F40C941155ACEBB7E0E42FF0E0BD0148
:10954A00A9E1B0E00E94DDD2DB01AE0FBF1FEC91B2
:10955A00EF775E2FACEBB7E0E42FF0E0BD01A9E1B5
:10956A00B0E00E94DDD2DB01AE0FBF1F1396AC91B3
:10957A00A13088F0ACEBB7E0E42FF0E0BD01A9E13F
:10958A00B0E00E94DDD2DB01AE0FBF1F1396EC9153
:10959A00E1500C94FA52ACEBB7E0E42FF0E0BD01D5
:1095AA00A9E1B0E00E94DDD2DB01AE0FBF1F139626
:1095BA00E4E0EC93FE013C96FA93EA93E0E0EA9346
:1095CA00A6E0B0E00E9427CBFE013696FA93EA9312
:1095DA00E0E0EA93A6E0B0E00E9427CB20E0E1E0D9
:1095EA00EE8BE0E1ED8B251708F086C700E030E04E
:1095FA00A9E2B8E0E42FF0E0BD01A1E7B0E00E94E3
:10960A00DDD2DB01AE0FBF1F1E96E22FF0E00E94F3
:10961A00A4D2AE0FBF1F15960E941FD41E2FA12FD2
:10962A000E94157F3E2F3030E9F4A9E2B8E0E42F1A
:10963A00F0E0BD01A1E7B0E00E94DDD2DB01AE0F90
:10964A00BF1F1E96E22FF0E00E94A4D2AE0FBF1FEA
:10965A0014960E941FD41E2F103021F0A12F0E94B1
:10966A00157F3E2F3030E9F4A9E2B8E0E42FF0E0AC
:10967A00BD01A1E7B0E00E94DDD2DB01AE0FBF1F42
:10968A001E96E22FF0E00E94A4D2AE0FBF1F1396DF
:10969A000E941FD41E2F103021F0A12F0E94157F87
:1096AA003E2F303011F0353009F4A1C0E32FF0E03D
:1096BA00E130A0E0FA0729F5A9E2B8E0E42FF0E0EA
:1096CA00BD01A1E7B0E00E94DDD2DB01AE0FBF1FF2
:1096DA001C960E941FD4E295E7700E2FA9E2B8E00B
:1096EA00E42FF0E0BD01A1E7B0E00E94DDD2DB018A
:1096FA00AE0FBF1F1C960E941FD4EE1FE0E0EE1FA4
:10970A0073C0E230A0E0FA07F9F4A9E2B8E0E42F66
:10971A00F0E0BD01A1E7B0E00E94DDD2DB01AE0FAF
:10972A00BF1F1C960E941FD4E7700E2FA9E2B8E053
:10973A00E42FF0E0BD01A1E7B0E00E94DDD2DB0139
:10974A00AE0FBF1F1C964BC0E330A0E0FA0729F505
:10975A00A9E2B8E0E42FF0E0BD01A1E7B0E00E9481
:10976A00DDD2DB01AE0FBF1F1B960E941FD4E2950C
:10977A00E7700E2FA9E2B8E0E42FF0E0BD01A1E7FF
:10978A00B0E00E94DDD2DB01AE0FBF1F1B960E9424
:10979A001FD4EE1FE0E0EE1F27C0E430A0E0FA0776
:1097AA0029F5A9E2B8E0E42FF0E0BD01A1E7B0E0B5
:1097BA000E94DDD2DB01AE0FBF1F1B960E941FD491
:1097CA00E7700E2FA9E2B8E0E42FF0E0BD01A1E7AF
:1097DA00B0E00E94DDD2DB01AE0FBF1F1B960E94D4
:1097EA001FD4E695E695E695E170EF8BF0C0A9E205
:1097FA00B8E0E42FF0E0BD01A1E7B0E00E94DDD2BD
:10980A00DB01AE0FBF1F1E96E22FF0E00E94A4D22A
:10981A00AE0FBF1F12960E941FD41E2F103029F0C0
:10982A00A12F0E94713CE03009F42EC0A9E2B8E0F1
:10983A00E42FF0E0BD01A1E7B0E00E94DDD2DB0138
:10984A00AE0FBF1F1E96E22FF0E00E94A4D2AE0F09
:10985A00BF1F17960E941FD4E295E7700E2FA9E248
:10986A00B8E0E42FF0E0BD01A1E7B0E00E94DDD24C
:10987A00DB01AE0FBF1F1E96E22FF0E00E94A4D2BA
:10988A00AE0FBF1F17969CC0A9E2B8E0E42FF0E024
:10989A00BD01A1E7B0E00E94DDD2DB01AE0FBF1F20
:1098AA001E96E22FF0E00E94A4D2AE0FBF1F1196BF
:1098BA000E941FD41E2F103029F0A12F0E94713C44
:1098CA00E03009F432C0A9E2B8E0E42FF0E0BD01CB
:1098DA00A1E7B0E00E94DDD2DB01AE0FBF1F1E96EA
:1098EA00E22FF0E00E94A4D2AE0FBF1F17960E948B
:1098FA001FD4E7700E2FA9E2B8E0E42FF0E0BD0113
:10990A00A1E7B0E00E94DDD2DB01AE0FBF1F1E96B9
:10991A00E22FF0E00E94A4D2AE0FBF1F17960E945A
:10992A001FD4E695E695E69550C0A9E2B8E0E42F83
:10993A00F0E0BD01A1E7B0E00E94DDD2DB01AE0F8D
:10994A00BF1F1E96E22FF0E00E94A4D2AE0FBF1FE7
:10995A000E941FD41E2F103029F0A12F0E94713CA3
:10996A00E03009F434C0A9E2B8E0E42FF0E0BD0128
:10997A00A1E7B0E00E94DDD2DB01AE0FBF1F1E9649
:10998A00E22FF0E00E94A4D2AE0FBF1F16960E94EB
:10999A001FD4E295E7700E2FA9E2B8E0E42FF0E0B9
:1099AA00BD01A1E7B0E00E94DDD2DB01AE0FBF1F0F
:1099BA001E96E22FF0E00E94A4D2AE0FBF1F1696A9
:1099CA000E941FD4EE1FE0E0EE1FE170EF8B003023
:1099DA0011F4353009F025C0A9E2B8E0E42FF0E02F
:1099EA00BD01A1E7B0E00E94DDD2DB01AE0FBF1FCF
:1099FA001D960E941FD4E7700E2FA9E2B8E0E42F4B
:109A0A00F0E0BD01A1E7B0E00E94DDD2DB01AE0FBC
:109A1A00BF1F1D960E941FD4E695E695E695E17054
:109A2A00EF8BEF89E03009F4ABC2593008F047C038
:109A3A00E02FF0E0E130A0E0FA0729F4EE89AE81E8
:109A4A00EA2BEE833BC0E230A0E0FA0719F4FE01EC
:109A5A0037962EC0E330A0E0FA0741F1E430A0E0E7
:109A6A00FA0739F4EE89AE81EA2BEE83FE013796C6
:109A7A001FC0E530A0E0FA0789F0E630A0E0FA0757
:109A8A0029F4EE89AE81EA2BEE8310C0E730A0E01C
:109A9A00FA07A1F4EE89AE81EA2BEE83FE0137962E
:109AAA000F01E081AE89EA2BD001EC93FE013896D2
:109ABA000F01E081AE89EA2BD001EC9360C25A30E3
:109ACA0009F0C9C0E02FF0E0E130A0E0FA0781F424
:109ADA00283028F4EE89AE81EA2BEE8308C0FE0115
:109AEA0037960F01E081AE89EA2BD001EC93B2C020
:109AFA00E230A0E0FA0771F4283018F4FE01389633
:109B0A0002C0FE0139960F01E081AE89EA2BD0012D
:109B1A00EC93A0C0E330A0E0FA0771F4283018F4FF
:109B2A00FE013A9602C0FE013B960F01E081AE8922
:109B3A00EA2BD001EC938EC0E430A0E0FA07E9F4F6
:109B4A00283028F4EE89AE81EA2BEE8308C0FE01A4
:109B5A0037960F01E081AE89EA2BD001EC932830C9
:109B6A0018F4FE01389602C0FE0139960F01E08111
:109B7A00AE89EA2BD001EC936DC0E530A0E0FA077C
:109B8A00D9F4283018F4FE01389602C0FE0139963D
:109B9A000F01E081AE89EA2BD001EC93283018F44A
:109BAA00FE013A9602C0FE013B960F01E081AE89A2
:109BBA00EA2BD001EC934EC0E630A0E0FA07E9F4B4
:109BCA00283028F4EE89AE81EA2BEE8308C0FE0124
:109BDA0037960F01E081AE89EA2BD001EC93283049
:109BEA0018F4FE013A9602C0FE013B960F01E0818D
:109BFA00AE89EA2BD001EC932DC0E730A0E0FA073A
:109C0A0049F5283018F4FE01389602C0FE0139964B
:109C1A000F01E081AE89EA2BD001EC93283028F4B9
:109C2A00EE89AE81EA2BEE8308C0FE0137960F015A
:109C3A00E081AE89EA2BD001EC93283018F4FE01BA
:109C4A003A9602C0FE013B960F01E081AE89EA2BEB
:109C5A00D001EC9394C15C3009F0C9C0E02FF0E068
:109C6A00E130A0E0FA0781F4283028F4EE89AE81C9
:109C7A00EA2BEE8308C0FE0137960F01E081AE8918
:109C8A00EA2BD001EC93B2C0E230A0E0FA0771F4FB
:109C9A00243018F4FE01379602C0FE0138960F01EF
:109CAA00E081AD89EA2BD001EC93A0C0E330A0E0BB
:109CBA00FA0771F4283018F4FE01399602C0FE0141
:109CCA003A960F01E081AE89EA2BD001EC938EC05F
:109CDA00E430A0E0FA07E9F4283028F4EE89AE81EE
:109CEA00EA2BEE8308C0FE0137960F01E081AE89A8
:109CFA00EA2BD001EC93243018F4FE01379602C007
:109D0A00FE0138960F01E081AD89EA2BD001EC9370
:109D1A006DC0E530A0E0FA07D9F4243018F4FE014A
:109D2A00379602C0FE0138960F01E081AD89EA2B11
:109D3A00D001EC93283018F4FE01399602C0FE01D6
:109D4A003A960F01E081AE89EA2BD001EC934EC01E
:109D5A00E630A0E0FA07E9F4283028F4EE89AE816B
:109D6A00EA2BEE8308C0FE0137960F01E081AE8927
:109D7A00EA2BD001EC93283018F4FE01399602C080
:109D8A00FE013A960F01E081AE89EA2BD001EC93ED
:109D9A002DC0E730A0E0FA0749F5283028F4EE890B
:109DAA00AE81EA2BEE8308C0FE0137960F01E081EF
:109DBA00AE89EA2BD001EC93243018F4FE013796D1
:109DCA0002C0FE0138960F01E081AD89EA2BD0016D
:109DDA00EC93283018F4FE01399602C0FE013A9637
:109DEA000F01E081AE89EA2BD001EC93C8C0E02FC5
:109DFA00F0E0E130A0E0FA0781F4283028F4EE8997
:109E0A00AE81EA2BEE8308C0FE0137960F01E0818E
:109E1A00AE89EA2BD001EC93B2C0E230A0E0FA0797
:109E2A0071F4283018F4FE01389602C0FE01399602
:109E3A000F01E081AD89EA2BD001EC93A0C0E33099
:109E4A00A0E0FA0771F4283018F4FE013A9602C02D
:109E5A00FE013B960F01E081AE89EA2BD001EC931B
:109E6A008EC0E430A0E0FA07E9F4283028F4EE893D
:109E7A00AE81EA2BEE8308C0FE0137960F01E0811E
:109E8A00AE89EA2BD001EC93283018F4FE013896FB
:109E9A0002C0FE0139960F01E081AD89EA2BD0019B
:109EAA00EC936DC0E530A0E0FA07D9F4283018F435
:109EBA00FE01389602C0FE0139960F01E081AD8994
:109ECA00EA2BD001EC93283018F4FE013A9602C02E
:109EDA00FE013B960F01E081AE89EA2BD001EC939B
:109EEA004EC0E630A0E0FA07E9F4283028F4EE89FB
:109EFA00AE81EA2BEE8308C0FE0137960F01E0819E
:109F0A00AE89EA2BD001EC93283018F4FE013A9678
:109F1A0002C0FE013B960F01E081AE89EA2BD00117
:109F2A00EC932DC0E730A0E0FA0749F5283028F471
:109F3A00EE89AE81EA2BEE8308C0FE0137960F0147
:109F4A00E081AE89EA2BD001EC93283018F4FE01A7
:109F5A00389602C0FE0139960F01E081AD89EA2BDD
:109F6A00D001EC93283018F4FE013A9602C0FE01A3
:109F7A003B960F01E081AE89EA2BD001EC93AAC28D
:109F8A00593008F047C0E02FF0E0E130A0E0FA07CE
:109F9A0029F4EE89AC85EA2BEC873BC0E230A0E0DD
:109FAA00FA0719F4FE013D962EC0E330A0E0FA0745
:109FBA0041F1E430A0E0FA0739F4EE89AC85EA2BE6
:109FCA00EC87FE013D961FC0E530A0E0FA0789F054
:109FDA00E630A0E0FA0729F4EE89AC85EA2BEC8793
:109FEA0010C0E730A0E0FA07A1F4EE89AC85EA2BAD
:109FFA00EC87FE013D960F01E081AE89EA2BD00184
:10A00A00EC93FE013E960F01E081AE89EA2BD00166
:10A01A00EC9360C25A3009F0C9C0E02FF0E0E13099
:10A02A00A0E0FA0781F4283028F4EE89AC85EA2BFF
:10A03A00EC8708C0FE013D960F01E081AE89EA2B4C
:10A04A00D001EC93B2C0E230A0E0FA0771F42830F4
:10A05A0018F4FE013E9602C0FE013F960F01E08110
:10A06A00AE89EA2BD001EC93A0C0E330A0E0FA0756
:10A07A0071F4283018F4FE01709602C0FE01719640
:10A08A000F01E081AE89EA2BD001EC938EC0E43057
:10A09A00A0E0FA07E9F4283028F4EE89AC85EA2B27
:10A0AA00EC8708C0FE013D960F01E081AE89EA2BDC
:10A0BA00D001EC93283018F4FE013E9602C0FE014E
:10A0CA003F960F01E081AE89EA2BD001EC936DC077
:10A0DA00E530A0E0FA07D9F4283018F4FE013E96DC
:10A0EA0002C0FE013F960F01E081AE89EA2BD00142
:10A0FA00EC93283018F4FE01709602C0FE017196A6
:10A10A000F01E081AE89EA2BD001EC934EC0E63014
:10A11A00A0E0FA07E9F4283028F4EE89AC85EA2BA6
:10A12A00EC8708C0FE013D960F01E081AE89EA2B5B
:10A13A00D001EC93283018F4FE01709602C0FE019B
:10A14A0071960F01E081AE89EA2BD001EC932DC004
:10A15A00E730A0E0FA0749F5283018F4FE013E96E8
:10A16A0002C0FE013F960F01E081AE89EA2BD001C1
:10A17A00EC93283028F4EE89AC85EA2BEC8708C0EA
:10A18A00FE013D960F01E081AE89EA2BD001EC93E6
:10A19A00283018F4FE01709602C0FE0171960F0174
:10A1AA00E081AE89EA2BD001EC9394C15C3009F0CE
:10A1BA00C9C0E02FF0E0E130A0E0FA0781F42830CE
:10A1CA0028F4EE89AC85EA2BEC8708C0FE013D969F
:10A1DA000F01E081AE89EA2BD001EC93B2C0E230E4
:10A1EA00A0E0FA0771F4243018F4FE013D9602C08B
:10A1FA00FE013E960F01E081AD89EA2BD001EC9376
:10A20A00A0C0E330A0E0FA0771F4283018F4FE0188
:10A21A003F9602C0FE0170960F01E081AE89EA2BDB
:10A22A00D001EC938EC0E430A0E0FA07E9F42830BC
:10A23A0028F4EE89AC85EA2BEC8708C0FE013D962E
:10A24A000F01E081AE89EA2BD001EC93243018F497
:10A25A00FE013D9602C0FE013E960F01E081AD89E6
:10A26A00EA2BD001EC936DC0E530A0E0FA07D9F4EF
:10A27A00243018F4FE013D9602C0FE013E960F01FD
:10A28A00E081AD89EA2BD001EC93283018F4FE0165
:10A29A003F9602C0FE0170960F01E081AE89EA2B5B
:10A2AA00D001EC934EC0E630A0E0FA07E9F428307A
:10A2BA0028F4EE89AC85EA2BEC8708C0FE013D96AE
:10A2CA000F01E081AE89EA2BD001EC93283018F413
:10A2DA00FE013F9602C0FE0170960F01E081AE8931
:10A2EA00EA2BD001EC932DC0E730A0E0FA0749F53C
:10A2FA00283028F4EE89AC85EA2BEC8708C0FE01E9
:10A30A003D960F01E081AE89EA2BD001EC9324300F
:10A31A0018F4FE013D9602C0FE013E960F01E0814F
:10A32A00AD89EA2BD001EC93283018F4FE013F9650
:10A33A0002C0FE0170960F01E081AE89EA2BD001BE
:10A34A00EC93C8C0E02FF0E0E130A0E0FA0781F416
:10A35A00283028F4EE89AC85EA2BEC8708C0FE0188
:10A36A003D960F01E081AE89EA2BD001EC93B2C091
:10A37A00E230A0E0FA0771F4283018F4FE013E96A4
:10A38A0002C0FE013F960F01E081AE89EA2BD0019F
:10A39A00EC93A0C0E330A0E0FA0771F4283018F477
:10A3AA00FE01709602C0FE0171960F01E081AE892E
:10A3BA00EA2BD001EC938EC0E430A0E0FA07E9F46E
:10A3CA00283028F4EE89AC85EA2BEC8708C0FE0118
:10A3DA003D960F01E081AE89EA2BD001EC9328303B
:10A3EA0018F4FE013E9602C0FE013F960F01E0817D
:10A3FA00AE89EA2BD001EC936DC0E530A0E0FA07F4
:10A40A00D9F4283018F4FE013E9602C0FE013F96A8
:10A41A000F01E081AE89EA2BD001EC93283018F4C1
:10A42A00FE01709602C0FE0171960F01E081AE89AD
:10A43A00EA2BD001EC934EC0E630A0E0FA07E9F42B
:10A44A00283028F4EE89AC85EA2BEC8708C0FE0197
:10A45A003D960F01E081AE89EA2BD001EC932830BA
:10A46A0018F4FE01709602C0FE0171960F01E08198
:10A47A00AE89EA2BD001EC932DC0E730A0E0FA07B1
:10A48A0049F5283028F4EE89AC85EA2BEC8708C018
:10A49A00FE013D960F01E081AE89EA2BD001EC93D3
:10A4AA00283018F4FE013E9602C0FE013F960F01C5
:10A4BA00E081AE89EA2BD001EC93283018F4FE0132
:10A4CA00709602C0FE0171960F01E081AE89EA2BF7
:10A4DA00D001EC93EE89EE0FEE8BED89EE0FED8B4A
:10A4EA00EE89E03011F4E1E0EE8BED89E03011F411
:10A4FA00E1E0ED8B2F5F77C8ACEBB7E0E42FF0E03B
:10A50A00BD01A9E1B0E00E94DDD2E60FF71F3B963C
:10A51A00FA93EA93FE013E96FA93EA93A6E0B0E034
:10A52A000E94FCCAE03029F1ACEBB7E0E42FF0E07E
:10A53A00BD01A9E1B0E00E94DDD2E60FF71F3B960C
:10A54A00FA93EA93FE013E96FA93EA93A6E0B0E004
:10A55A000E9415CBACEBB7E0E42FF0E0BD01A9E116
:10A56A00B0E00E94DDD2DB01AE0FBF1F5796E0E0DC
:10A57A00EC93ACEBB7E0E42FF0E0BD01A9E1B0E069
:10A58A000E94DDD2E60FF71F7196FA93EA93FE0155
:10A59A003896FA93EA93A6E0B0E00E94FCCAE0304B
:10A5AA0029F1ACEBB7E0E42FF0E0BD01A9E1B0E09E
:10A5BA000E94DDD2E60FF71F7196FA93EA93FE0125
:10A5CA003896FA93EA93A6E0B0E00E9415CBACEB7A
:10A5DA00B7E0E42FF0E0BD01A9E1B0E00E94DDD2CE
:10A5EA00DB01AE0FBF1F5896E0E0EC93ACEBB7E08F
:10A5FA00E42FF0E0BD01A9E1B0E00E94DDD2DB0169
:10A60A00AE0FBF1F1496AC91A13088F0ACEBB7E047
:10A61A00E42FF0E0BD01A9E1B0E00E94DDD2DB0148
:10A62A00AE0FBF1F1496EC91E150EC9330C1ACEB26
:10A63A00B7E0E42FF0E0BD01A9E1B0E00E94DDD26D
:10A64A00DB01AE0FBF1F5796AC91A13080F0ACEB87
:10A65A00B7E0E42FF0E0BD01A9E1B0E00E94DDD24D
:10A66A00DB01AE0FBF1F5896AC91A13008F40FC1A1
:10A67A00ACEBB7E0E42FF0E0BD01A9E1B0E00E9445
:10A68A00DDD2DB01AE0FBF1F1496E4E6EC93A9E21C
:10A69A00B8E0E42FF0E0BD01A1E7B0E00E94DDD20E
:10A6AA00DB01AE0FBF1F17960E941FD4AE2F0E9468
:10A6BA00713CE03081F1A9E2B8E0E42FF0E0BD019D
:10A6CA00A1E7B0E00E94DDD2DB01AE0FBF1F1896F2
:10A6DA000E941FD4EC8BA9E2B8E0E42FF0E0BD01A0
:10A6EA00A1E7B0E00E94DDD2DB01AE0FBF1F1A96D0
:10A6FA000E941FD4E295EF70EB8BA9E2B8E0E42F39
:10A70A00F0E0BD01A1E7B0E00E94DDD2DB01AE0FAF
:10A71A00BF1F199671C0A9E2B8E0E42FF0E0BD01AD
:10A72A00A1E7B0E00E94DDD2DB01AE0FBF1F149695
:10A73A000E941FD4AE2F0E94713CE03079F1A9E249
:10A74A00B8E0E42FF0E0BD01A1E7B0E00E94DDD25D
:10A75A00DB01AE0FBF1F15960E941FD4EC8BA9E236
:10A76A00B8E0E42FF0E0BD01A1E7B0E00E94DDD23D
:10A77A00DB01AE0FBF1F1A960E941FD4EF70EB8B3E
:10A78A00A9E2B8E0E42FF0E0BD01A1E7B0E00E9441
:10A79A00DDD2DB01AE0FBF1F16962EC0A9E2B8E0CC
:10A7AA00E42FF0E0BD01A1E7B0E00E94DDD2DB01B9
:10A7BA00AE0FBF1F12960E941FD4EC8BA9E2B8E01D
:10A7CA00E42FF0E0BD01A1E7B0E00E94DDD2DB0199
:10A7DA00AE0FBF1F11960E941FD4EF70EB8BA9E238
:10A7EA00B8E0E42FF0E0BD01A1E7B0E00E94DDD2BD
:10A7FA00DB01AE0FBF1F13960E941FD4EA8BE88DB0
:10A80A00E07FE860E88FEF7EE88FA9E2B8E0E42F06
:10A81A00F0E0BD01A1E7B0E00E94DDD2DB01AE0F9E
:10A82A00BF1F0E941FD4F0E0F660E98FFA8FEFE2B3
:10A83A00ED8FE3E0EE8FE0E2EF8FE1E0E8A3EA8953
:10A84A00E9A3E0E0EAA3EBA3ECA3DE0158960E9499
:10A85A003E09E88DE07FE260E88FA9E2B8E0E42FE4
:10A86A00F0E0BD01A1E7B0E00E94DDD2DB01AE0F4E
:10A87A00BF1F0E941FD4F0E0F560E98FFA8FEC89C0
:10A88A00ED8FEB89EE8FDE0158960E943E09593012
:10A89A0010F0E6E001C0E3E0EF700E2EE88DE07FF5
:10A8AA00E029E88FEF7EE88FACEBB7E0E42FF0E029
:10A8BA00BD01A9E1B0E00E94DDD2DB01AE0FBF1FEE
:10A8CA005796AC91A13088F0ACEBB7E0E42FF0E0FA
:10A8DA00BD01A9E1B0E00E94DDD2DB01AE0FBF1FCE
:10A8EA005796EC91E150EC933BC0ACEBB7E0E42F08
:10A8FA00F0E0BD01A9E1B0E00E94DDD2DB01AE0FBC
:10A90A00BF1F5796EAEFEC93A9E2B8E0E42FF0E014
:10A91A00BD01A1E7B0E00E94DDD2DB01AE0FBF1F8F
:10A92A000E941FD4F0E0F260E98FFA8FFE017D9653
:10A93A00FA93EA93ACEBB7E0E42FF0E0BD01A9E1AA
:10A94A00B0E00E94DDD2E60FF71F3B96FA93EA9336
:10A95A00A6E0B0E00E9415CBDE0158960E943E099F
:10A96A00ACEBB7E0E42FF0E0BD01A9E1B0E00E9452
:10A97A00DDD2DB01AE0FBF1F5896AC91A13088F033
:10A98A00ACEBB7E0E42FF0E0BD01A9E1B0E00E9432
:10A99A00DDD2DB01AE0FBF1F5896EC91E150EC936C
:10A9AA003BC0ACEBB7E0E42FF0E0BD01A9E1B0E0B9
:10A9BA000E94DDD2DB01AE0FBF1F5896EAEFEC937F
:10A9CA00A9E2B8E0E42FF0E0BD01A1E7B0E00E94FF
:10A9DA00DDD2DB01AE0FBF1F0E941FD4F0E0F3608F
:10A9EA00E98FFA8FFE017D96FA93EA93ACEBB7E012
:10A9FA00E42FF0E0BD01A9E1B0E00E94DDD2E60F4C
:10AA0A00F71F7196FA93EA93A6E0B0E00E9415CB7D
:10AA1A00DE0158960E943E094F5F0C948A4A0E94B2
:10AA2A002FD2A59608952D970E942AD2E091630409
:10AA3A00E07409F4A8C100E0023008F0A4C1A9E258
:10AA4A00B8E0E02FF0E0BD01A1E7B0E00E94DDD25E
:10AA5A00DB01AE0FBF1F0E941FD4E03081F4ACEBC4
:10AA6A00B7E0E02FF0E0BD01A9E1B0E00E94DDD23D
:10AA7A00DB01AE0FBF1F1296E0E0EC9382C1ACEB94
:10AA8A00B7E0E02FF0E0BD01A9E1B0E00E94DDD21D
:10AA9A00DB01AE0FBF1F1296AC91A13008F46CC057
:10AAAA00ACEBB7E0E02FF0E0BD01A9E1B0E00E9415
:10AABA00DDD2DB01AE0FBF1F1296EC91E150EC9391
:10AACA00ACEBB7E0E02FF0E0BD01A9E1B0E00E94F5
:10AADA00DDD2DB01AE0FBF1F1196AC91A13088F019
:10AAEA00ACEBB7E0E02FF0E0BD01A9E1B0E00E94D5
:10AAFA00DDD2DB01AE0FBF1F1196EC91E150EC9352
:10AB0A003AC0ACEBB7E0E02FF0E0BD01A9E1B0E05C
:10AB1A000E94DDD2DB01AE0FBF1F1196E2E3EC9378
:10AB2A00EC81E07FE860EC83EF7EEC83A9E2B8E099
:10AB3A00E02FF0E0BD01A1E7B0E00E94DDD2DB0129
:10AB4A00AE0FBF1F0E941FD4F0E0F660ED83FE83B4
:10AB5A00EBE2E987E0E0EA87E8E1EB87E5E0EC870A
:10AB6A00E4EFED87E1E0EE87E0E0EF87E88BDE01D6
:10AB7A0014960E943E0905C1ACEBB7E0E02FF0E065
:10AB8A00BD01A9E1B0E00E94DDD2DB01AE0FBF1F1B
:10AB9A00EC91E07809F4C8C0ACEBB7E0E02FF0E044
:10ABAA00BD01A9E1B0E00E94DDD2DB01AE0FBF1FFB
:10ABBA00EC91EF773E2FACEBB7E0E02FF0E0BD0170
:10ABCA00A9E1B0E00E94DDD2DB01AE0FBF1FEC911C
:10ABDA00EF77EC93EAE9F4E060E070E00E94B1D329
:10ABEA00E02FF0E031966F2F660F660B762F0E94EA
:10ABFA00B1D384E00E94AFD1289621E010E0131768
:10AC0A0008F047C0A9E2B8E0E02FF0E0BD01A1E7F3
:10AC1A00B0E00E94DDD2DB01AE0FBF1F1E96E12F0E
:10AC2A00F0E00E94A4D2AE0FBF1F16960E941FD456
:10AC3A00F0E0F695E795E370F070309799F4ACEB95
:10AC4A00B7E0E02FF0E0BD01A9E1B0E00E94DDD25B
:10AC5A00E60FF71F39960F01A081E22FE095EA234C
:10AC6A00D00113C0E130A0E0FA0781F4ACEBB7E001
:10AC7A00E02FF0E0BD01A9E1B0E00E94DDD2DB01E6
:10AC8A00AE0FBF1F1996EC91E22BEC931F5F220FB8
:10AC9A00B6CF21E0131708F047C0A9E2B8E0E02FC9
:10ACAA00F0E0BD01A1E7B0E00E94DDD2DB01AE0F0A
:10ACBA00BF1F1E96E12FF0E00E94A4D2AE0FBF1F65
:10ACCA0016960E941FD4F0E0F695E795E370F070AF
:10ACDA00309799F4ACEBB7E0E02FF0E0BD01A9E1C1
:10ACEA00B0E00E94DDD2E60FF71F3A960F01A0816D
:10ACFA00E22FE095EA23D00113C0E130A0E0FA0781
:10AD0A0081F4ACEBB7E0E02FF0E0BD01A9E1B0E0DF
:10AD1A000E94DDD2DB01AE0FBF1F1A96EC91E22B27
:10AD2A00EC931F5F220FB6CFACEBB7E0E02FF0E059
:10AD3A00BD01A9E1B0E00E94DDD2DB01AE0FBF1F69
:10AD4A001296EAE0EC93EC81E07FE260EC83EF7E1E
:10AD5A00EC83E0E0ED83EE83E1E0E987A9E2B8E085
:10AD6A00E02FF0E0BD01A1E7B0E00E94DDD2DB01F7
:10AD7A00AE0FBF1F0E941FD4EA87DE0114960E94FD
:10AD8A003E090F5F59CE0E9431D2619608950E9402
:10AD9A002AD210E0133008F081C0AEEBB7E0E12F01
:10ADAA00F0E0BD01ACE0B0E00E94DDD2E60FF71F93
:10ADBA003196FF93EF93A9E2B8E0E12FF0E0BD01ED
:10ADCA00AAE0B0E00E94DDD2DB01AE0FBF1F0E94F5
:10ADDA001FD4AF91BF91EC93AEEBB7E0E12FF0E057
:10ADEA00BD01ACE0B0E00E94DDD2E60FF71F32965B
:10ADFA00FF93EF93A9E2B8E0E12FF0E0BD01AAE0EA
:10AE0A00B0E00E94DDD2DB01AE0FBF1F11960E9497
:10AE1A001FD4AF91BF91EC93AEEBB7E0E12FF0E016
:10AE2A00BD01ACE0B0E00E94DDD2E60FF71F359617
:10AE3A00FF93EF93A9E2B8E0E12FF0E0BD01AAE0A9
:10AE4A00B0E00E94DDD2DB01AE0FBF1F12960E9456
:10AE5A001FD4AF91BF91EC93AEEBB7E0E12FF0E0D6
:10AE6A00BD01ACE0B0E00E94DDD2E60FF71F3696D6
:10AE7A00FF93EF93A9E2B8E0E12FF0E0BD01AAE069
:10AE8A00B0E00E94DDD2DB01AE0FBF1F15960E9413
:10AE9A001FD4AF91BF91EC931F5F7CCFE091C007A5
:10AEAA00E093CD07A091C007E091CC07EA0FE093A9
:10AEBA00D907A091D907E091D807EA0FE093BD0717
:10AECA0010E0183108F0E1C0E0E03E2F0E2FA7E4B1
:10AEDA00B8E0E12FF0E0BD01ACE0B0E00E94DDD2C5
:10AEEA00DB01AE0FBF1F11960E941FD4E03009F09C
:10AEFA0031E0A7E4B8E0E12FF0E0BD01ACE0B0E05A
:10AF0A000E94DDD2DB01AE0FBF1F12960E941FD432
:10AF1A00E03009F03260A7E4B8E0E12FF0E0BD01CB
:10AF2A00ACE0B0E00E94DDD2DB01AE0FBF1F159688
:10AF3A000E941FD4E03009F03460A7E4B8E0E12FA2
:10AF4A00F0E0BD01ACE0B0E00E94DDD2DB01AE0F63
:10AF5A00BF1F16960E941FD4E03009F03860A7E49C
:10AF6A00B8E0E12FF0E0BD01ACE0B0E00E94DDD234
:10AF7A00DB01AE0FBF1F19960E941FD4E03009F003
:10AF8A003061A7E4B8E0E12FF0E0BD01ACE0B0E049
:10AF9A000E94DDD2DB01AE0FBF1F1A960E941FD49A
:10AFAA00E03009F03062A7E4B8E0E12FF0E0BD013B
:10AFBA00ACE0B0E00E94DDD2DB01AE0FBF1F1396FA
:10AFCA000E941FD4E03009F000E1A7E4B8E0E12FC5
:10AFDA00F0E0BD01ACE0B0E00E94DDD2DB01AE0FD3
:10AFEA00BF1F17960E941FD4E03009F00062A7E441
:10AFFA00B8E0E12FF0E0BD01ACE0B0E00E94DDD2A4
:10B00A00DB01AE0FBF1F1B960E941FD4E03009F070
:10B01A000064A2EEB7E0E12FF0E00E94A6D2EA0FA8
:10B02A00FB1F0283A2EEB7E0E12FF0E00E94A6D256
:10B03A00EA0FFB1F3383A2EEB7E0E12FF0E00E9494
:10B04A00A6D2EA0FFB1F3296FF93EF93A7E4B8E06C
:10B05A00E12FF0E0BD01ACE0B0E00E94DDD2DB01FF
:10B06A00AE0FBF1F0E941FD4E295EF70E695E695DA
:10B07A00E170AF91BF91E170EE0FEE0F0E2EEC91E1
:10B08A00EB7FE029EC931F5F1CCF0E9431D22496FC
:10B09A000895BA93AA9325970E9428D2E091BB07F4
:10B0AA00F0E0E230A0E0FA0739F4AB85BC85EC9118
:10B0BA00E07109F02AC10AC0E330A0E0FA0731F4CE
:10B0CA00AB85BC85EC91E07109F41FC1E091BB0727
:10B0DA00F0E0E230A0E0FA0729F0E330A0E0FA0756
:10B0EA0009F013C110E0133008F00FC1AEEBB7E05E
:10B0FA00E12FF0E0BD01ACE0B0E00E94DDD2E60F46
:10B10A00F71F2281213008F4FDC0AEEBB7E0E12F32
:10B11A00F0E0BD01ACE0B0E00E94DDD2E60FF71F1F
:10B12A003181A091BB07A23089F4E32FF0E0E05807
:10B13A00FE4F0F01AB85BC851196ED91FC911197DD
:10B14A00E015F10509F0DFC0E1E007C0EB85FC85F9
:10B15A00E181E31709F0D7C0E3E0EA87AEEBB7E095
:10B16A00E12FF0E0BD01ACE0B0E00E94DDD2DB01EE
:10B17A00AE0FBF1FEC91E03079F4AEEBB7E0E12FF0
:10B18A00F0E0BD01ACE0B0E00E94DDD2DB01AE0F21
:10B19A00BF1F1496EFEFEC93AEEBB7E0E12FF0E0B0
:10B1AA00BD01ACE0B0E00E94DDD2DB01AE0FBF1FF3
:10B1BA00ECE0EC93AEEBB7E0E12FF0E0BD01ACE0E0
:10B1CA00B0E00E94DDD2E60FF71F5381E0E04E2F78
:10B1DA00E8870E2F421708F094C0A091BB07A2304F
:10B1EA00A1F4003069F407E0AB85BC851596E885C3
:10B1FA00EF5FE887E150F0E0AE0FBF1FEC9103C0AC
:10B20A000150E985E695E98714C0003069F403E046
:10B21A00AB85BC851596E885EF5FE887E150F0E0DD
:10B22A00AE0FBF1FEC9104C00150E985E695E69583
:10B23A00E987A2EEB7E0E52FF0E00E94A6D2AE0FB2
:10B24A00BF1F1296EC91E47009F43FC0A2EEB7E07A
:10B25A00E52FF0E00E94A6D2AE0FBF1F1296EC9126
:10B26A00E170EF83A2EEB7E0E52FF0E00E94A6D2EC
:10B27A00AE0FBF1F1296EC91E695E170EE83EA8558
:10B28A00A985EA23E13069F4EE81E03049F4E1E08E
:10B29A00EE83EF81E03011F0E0E001C0E1E0EF83FE
:10B2AA0002C0E0E0EE83A2EEB7E0E52FF0E00E94F4
:10B2BA00A6D2AE0FBF1F1296EE81E170EE0F0E2ED0
:10B2CA00EC91ED7FE029EC9309C0EA85A985EA2390
:10B2DA00E13011F4E1E001C0E0E0EF83A2EEB7E073
:10B2EA00E52FF0E00E94A6D2AE0FBF1F1296EF81A3
:10B2FA00E1700E2EEC91EE7FE029EC934F5F5F5FD9
:10B30A0069CF03C002C01F5FEECE0E942FD22D96D6
:10B31A0008952D970E942AD21A2F09893A89EC8119
:10B32A00E061EC83E07FE860EC83F32FE0E06627DE
:10B33A007727E060F0606F6E7861DF01CB01E09102
:10B34A005C04FF2766277727EA2BFB2B682B792BD0
:10B35A00ED83FE836F837887E02FEF5FE987A2EEA4
:10B36A00B7E0E12FF0E00E94A6D2AE0FBF1FEC912A
:10B37A00EA87A2EEB7E0E12FF0E00E94A6D2AE0F74
:10B38A00BF1F1196EC91EB87C9C02D970E9428D256
:10B39A004A2FEE81EF7EEE83E07FE860EE83EC8950
:10B3AA00F0E0E050FE4FEF83F887FE013B96FA93F8
:10B3BA00EA93E0E0EA93A8E0B0E00E9427CB51E0EC
:10B3CA0020E031E0E0E00E2F1E2F141708F04BC0EA
:10B3DA0030E0333008F042C0503051F4E02F0F5FB4
:10B3EA00F0E0DE011B96EA0FFB1F208351E020E00C
:10B3FA00E32FF0E0309769F4A2EEB7E0EB89F0E0D2
:10B40A000E94A6D2AE0FBF1FEC91EF7009F0252B58
:10B41A0022C0E130A0E0FA0769F4A2EEB7E0EB89B6
:10B42A00F0E00E94A6D2AE0FBF1FEC91E07F09F0B8
:10B43A00252B11C0E230A0E0FA0769F4A2EEB7E0CA
:10B44A00EB89F0E00E94A6D2AE0FBF1F1196EC91D5
:10B45A00E03009F0252B550F3F5FBBCF1F5FEB890B
:10B46A00EF5FEB8BB2CFE02FF0E0DE011B96EA0F25
:10B47A00FB1F2083DE0116960E943E090E942FD2EE
:10B48A00659608952D970E942AD21A2F09893A891A
:10B49A00FE013996FA93EA93E0E0EA93A0E0B0E07D
:10B4AA000E9427CBEC81EF7EEC83E07FE860EC839F
:10B4BA00E32FF0E0E050FD4FED83FE831987FE0194
:10B4CA003B96008335C02D970E942AD21A2F0989EC
:10B4DA003A89EC81E061EC83E07FE860EC83F32F4A
:10B4EA00E0E066277727E060F060606D7861DF0151
:10B4FA00CB01E0915C04FF2766277727EA2BFB2B19
:10B50A00682B792BED83FE836F837887E0E0E987E8
:10B51A00FE013A960083FE013B961083FE013C969B
:10B52A00FA93EA93EFEFEA93A5E0B0E00E9427CB03
:10B53A00DE0114960E943E090E9431D26396089554
:10B54A0062970E9428D2E0916304E07409F47BC4F4
:10B55A00A091BC07A43038F4E091BC07EF5FE093F8
:10B56A00BC07E15003C0E0E0E093BC07A091BC0730
:10B57A00A33008F068C4AEEBB7E0E091BC07F0E096
:10B58A00BD01ACE0B0E00E94DDD2E60FF71F5181A9
:10B59A00AEEBB7E0E091BC07F0E0BD01ACE0B0E093
:10B5AA000E94DDD2E60FF71F1281AEEBB7E0E09101
:10B5BA00BC07F0E0BD01ACE0B0E00E94DDD2E60FCE
:10B5CA00F71F3381113010F0103108F03CC4E091BC
:10B5DA00BB07F0E0E230A0E0FA0729F0E330A0E090
:10B5EA00FA0709F030C4AEEBB7E0E091BC07F0E02F
:10B5FA00BD01ACE0B0E00E94DDD2DB01AE0FBF1F9F
:10B60A00AC91A13008F440C0AEEBB7E0E091BC07C2
:10B61A00F0E0BD01ACE0B0E00E94DDD2DB01AE0F8C
:10B62A00BF1FEC91E150EC93AEEBB7E0E091BC07A1
:10B63A00F0E0BD01ACE0B0E00E94DDD2DB01AE0F6C
:10B64A00BF1FEC91E030F9F400E0232F0117D8F482
:10B65A00A2EEB7E0E22FF0E00E94A6D2AE0FBF1F23
:10B66A001296EC91EE7FEC93A2EEB7E0E22FF0E0B7
:10B67A000E94A6D2AE0FBF1F1296EC91E260EC9325
:10B68A000F5F2F5FE3CF48C0A091BB07A23009F03C
:10B69A0043C0AEEBB7E0E091BC07F0E0BD01ACE01F
:10B6AA00B0E00E94DDD2DB01AE0FBF1F1A96AC914B
:10B6BA00A13088F0AEEBB7E0E091BC07F0E0BD0145
:10B6CA00ACE0B0E00E94DDD2DB01AE0FBF1F1A96DC
:10B6DA00EC91E15020C0EE81E07FE260EE83EF7EE4
:10B6EA00EE83E0E0EF83E887E1E0EB87E0E0EC87D8
:10B6FA00DE0116960E943E09AEEBB7E0E091BC0768
:10B70A00F0E0BD01ACE0B0E00E94DDD2DB01AE0F9B
:10B71A00BF1F1A96E4E1EC93AEEBB7E0E091BC07E9
:10B72A00F0E0BD01ACE0B0E00E94DDD2DB01AE0F7B
:10B73A00BF1F1696AC910E94713CE03011F1A9E24C
:10B74A00B8E0E091BC07F0E0BD01AAE0B0E00E94D9
:10B75A00DDD2DB01AE0FBF1F16960E941FD44E2FFB
:10B76A00A9E2B8E0E091BC07F0E0BD01AAE0B0E0D0
:10B77A000E94DDD2DB01AE0FBF1F17960E941FD4B5
:10B78A0037C0AEEBB7E0E091BC07F0E0BD01ACE03A
:10B79A00B0E00E94DDD2DB01AE0FBF1F1596AC915F
:10B7AA000E94713CE03011F1A9E2B8E0E091BC07D7
:10B7BA00F0E0BD01AAE0B0E00E94DDD2DB01AE0FED
:10B7CA00BF1F13960E941FD44E2FA9E2B8E0E09142
:10B7DA00BC07F0E0BD01AAE0B0E00E94DDD2DB01C7
:10B7EA00AE0FBF1F14960E941FD402C040E0E0E0D3
:10B7FA00EF8BAEEBB7E0E091BC07F0E0BD01ACE047
:10B80A00B0E00E94DDD2DB01AE0FBF1F1796AC91EC
:10B81A004A1799F4AEEBB7E0E091BC07F0E0BD013E
:10B82A00ACE0B0E00E94DDD2DB01AE0FBF1F18967C
:10B83A00AC91EF89EA1709F447C0AEEBB7E0E091A3
:10B84A00BC07F0E0BD01ACE0B0E00E94DDD2E60F3B
:10B85A00F71F4783AEEBB7E0E091BC07F0E0BD010C
:10B86A00ACE0B0E00E94DDD2E60FF71F3896AF8950
:10B87A00A083A091BB07A23011F55A93AEEBB7E0B3
:10B88A00E091BC07F0E0BD01ACE0B0E00E94DDD27F
:10B89A00DB01AE0FBF1F1896EC91EA93AEEBB7E04F
:10B8AA00E091BC07F0E0BD01ACE0B0E00E94DDD25F
:10B8BA00DB01AE0FBF1F1796AC91E4DD05C05A93AA
:10B8CA00E88DEA93A42FFFDD00E0232F011708F08B
:10B8DA00E8C1A2EEB7E0E22FF0E00E94A6D2AE0FD6
:10B8EA00BF1F1296EC91EE8BA2EEB7E0E22FF0E0CA
:10B8FA000E94A6D2AE0FBF1F1396EC91ED8BEE8974
:10B90A00E071A1F0A7E4B8E0E22FF0E0BD01ACE0FD
:10B91A00B0E00E94DDD2DB01AE0FBF1F13960E947A
:10B92A001FD4AE2F0E942B66E03009F412C0A7E4A0
:10B93A00B8E0E22FF0E0BD01ACE0B0E00E94DDD259
:10B94A00DB01AE0FBF1F0E941FD4E295E370EF5FC9
:10B95A0055C0ED89E270A1F0A7E4B8E0E22FF0E06B
:10B96A00BD01ACE0B0E00E94DDD2DB01AE0FBF1F2B
:10B97A0012960E941FD4AE2F0E94713CE03009F447
:10B98A0013C0A7E4B8E0E22FF0E0BD01ACE0B0E0FC
:10B99A000E94DDD2DB01AE0FBF1F0E941FD4E695C5
:10B9AA00E695E370EF5F2AC0ED89E170A1F0A7E4A4
:10B9BA00B8E0E22FF0E0BD01ACE0B0E00E94DDD2D9
:10B9CA00DB01AE0FBF1F11960E941FD4AE2F0E943B
:10B9DA00713CE03009F411C0A7E4B8E0E22FF0E0CE
:10B9EA00BD01ACE0B0E00E94DDD2DB01AE0FBF1FAB
:10B9FA000E941FD4E370EF5F01C0E0E0EC8BEE8998
:10BA0A00E072A1F0A7E4B8E0E22FF0E0BD01ACE0FB
:10BA1A00B0E00E94DDD2DB01AE0FBF1F17960E9475
:10BA2A001FD4AE2F0E942B66E03009F411C0A7E4A0
:10BA3A00B8E0E22FF0E0BD01ACE0B0E00E94DDD258
:10BA4A00DB01AE0FBF1F14960E941FD4E29551C0AE
:10BA5A00ED89E870A1F0A7E4B8E0E22FF0E0BD01BB
:10BA6A00ACE0B0E00E94DDD2DB01AE0FBF1F16963C
:10BA7A000E941FD4AE2F0E94713CE03009F412C01C
:10BA8A00A7E4B8E0E22FF0E0BD01ACE0B0E00E942C
:10BA9A00DDD2DB01AE0FBF1F14960E941FD4E695BC
:10BAAA00E69527C0ED89E470A1F0A7E4B8E0E22F9B
:10BABA00F0E0BD01ACE0B0E00E94DDD2DB01AE0FE8
:10BACA00BF1F15960E941FD4AE2F0E94713CE03012
:10BADA0009F416C0A7E4B8E0E22FF0E0BD01ACE03B
:10BAEA00B0E00E94DDD2DB01AE0FBF1F14960E94A8
:10BAFA001FD4E370EF5FE295E07FAC89EA2BEC8B11
:10BB0A00EE89E074A1F0A7E4B8E0E22FF0E0BD010D
:10BB1A00ACE0B0E00E94DDD2DB01AE0FBF1F1B9686
:10BB2A000E941FD4AE2F0E942B66E03009F413C086
:10BB3A00A7E4B8E0E22FF0E0BD01ACE0B0E00E947B
:10BB4A00DDD2DB01AE0FBF1F18960E941FD4E2950B
:10BB5A00E370EF5F57C0ED89E072A1F0A7E4B8E0A7
:10BB6A00E22FF0E0BD01ACE0B0E00E94DDD2DB01E3
:10BB7A00AE0FBF1F1A960E941FD4AE2F0E94713CAF
:10BB8A00E03009F414C0A7E4B8E0E22FF0E0BD0108
:10BB9A00ACE0B0E00E94DDD2DB01AE0FBF1F189609
:10BBAA000E941FD4E695E695E370EF5F2BC0ED89FE
:10BBBA00E071A1F0A7E4B8E0E22FF0E0BD01ACE04B
:10BBCA00B0E00E94DDD2DB01AE0FBF1F19960E94C2
:10BBDA001FD4AE2F0E94713CE03009F412C0A7E4D2
:10BBEA00B8E0E22FF0E0BD01ACE0B0E00E94DDD2A7
:10BBFA00DB01AE0FBF1F18960E941FD4E370EF5FE0
:10BC0A0001C0E0E0EB8BA2EEB7E0E22FF0E00E9489
:10BC1A00A6D2AE0FBF1FAC91EC89EA1769F4A2EE67
:10BC2A00B7E0E22FF0E00E94A6D2AE0FBF1F119636
:10BC3A00AC91EB89EA1791F1A2EEB7E0E22FF0E0BE
:10BC4A000E94A6D2EA0FFB1FAC89A083A2EEB7E03E
:10BC5A00E22FF0E00E94A6D2EA0FFB1F3196AB89D1
:10BC6A00A083AEEBB7E0E091BC07F0E0BD01ACE029
:10BC7A00B0E00E94DDD2DB01AE0FBF1F1996E4E1EE
:10BC8A00EC93A091BB07A23029F45A933A93A12FBF
:10BC9A007CDB04C05A930A93A22F3BDB0F5F2F5F12
:10BCAA0015CEAEEBB7E0E091BC07F0E0BD01ACE029
:10BCBA00B0E00E94DDD2DB01AE0FBF1F1996AC9136
:10BCCA00A13088F0AEEBB7E0E091BC07F0E0BD012F
:10BCDA00ACE0B0E00E94DDD2DB01AE0FBF1F1996C7
:10BCEA00EC91E150AFC0A091BB07A230B1F5AEEB29
:10BCFA00B7E0E091BC07F0E0BD01ACE0B0E00E9423
:10BD0A00DDD2DB01AE0FBF1F1996E9E0EC935A931F
:10BD1A003A93A12F3ADB5A93AEEBB7E0E091BC0716
:10BD2A00F0E0BD01ACE0B0E00E94DDD2DB01AE0F75
:10BD3A00BF1F1896EC91EA93AEEBB7E0E091BC070F
:10BD4A00F0E0BD01ACE0B0E00E94DDD2DB01AE0F55
:10BD5A00BF1F1796AC9196DB76C0AEEBB7E0E091C9
:10BD6A00BC07F0E0BD01ACE0B0E00E94DDD2DB012F
:10BD7A00AE0FBF1F1996EAE0EC93AEEBB7E0E09185
:10BD8A00BC07F0E0BD01ACE0B0E00E94DDD2DB010F
:10BD9A00AE0FBF1F1496AC91A11790F1AEEBB7E0AE
:10BDAA00E091BC07F0E0BD01ACE0B0E00E94DDD25A
:10BDBA00DB01AE0FBF1F1496E0E0EC935A93AEEB93
:10BDCA00B7E0E091BC07F0E0BD01ACE0B0E00E9452
:10BDDA00DDD2DB01AE0FBF1F1896EC91EA93AEEBF2
:10BDEA00B7E0E091BC07F0E0BD01ACE0B0E00E9432
:10BDFA00DDD2DB01AE0FBF1F1796AC9164DB23C007
:10BE0A00AEEBB7E0E091BC07F0E0BD01ACE0B0E01A
:10BE1A000E94DDD2E60FF71F04815A930A93A02FDE
:10BE2A00A30F77DAAEEBB7E0E091BC07F0E0BD0113
:10BE3A00ACE0B0E00E94DDD2DB01AE0FBF1F14966A
:10BE4A00EC91EF5FEC930E942FD2689608950E94BE
:10BE5A002AD2ECEBF7E0FA93EA93E0E0EA93A9E658
:10BE6A00B0E00E9427CBA9E2B8E00E941FD4E09379
:10BE7A00BD07AAE2B8E00E941FD4E093E50710E0EC
:10BE8A00123008F0A2C0ABE2B8E0E12FF0E0BD0149
:10BE9A00AAE0B0E00E94DDD2DB01AE0FBF1F0E9414
:10BEAA001BD49F01ADEBB7E0E12FF0E0BD01A8E2A2
:10BEBA00B0E00E94DDD2E60FF71F3496FF93EF93AE
:10BECA00ABE2B8E0E12FF0E0BD01AAE0B0E00E94E9
:10BEDA00DDD2DB01AE0FBF1F12960E941FD4AF91B5
:10BEEA00BF91EC93ADEBB7E0E12FF0E0BD01A8E222
:10BEFA00B0E00E94DDD2E60FF71F3596FF93EF936D
:10BF0A00ABE2B8E0E12FF0E0BD01AAE0B0E00E94A8
:10BF1A00DDD2DB01AE0FBF1F16960E941FD4AF9170
:10BF2A00BF91EC93ADEBB7E0E12FF0E0BD01A8E2E1
:10BF3A00B0E00E94DDD2E60FF71F2787308BADEB0A
:10BF4A00B7E0E12FF0E0BD01A8E2B0E00E94DDD247
:10BF5A00DB01AE0FBF1F1E96EC91E07FE460EC930D
:10BF6A00ADEBB7E0E12FF0E0BD01A8E2B0E00E943E
:10BF7A00DDD2DB01AE0FBF1F1196F9013196ED93A9
:10BF8A00FC93ADEBB7E0E12FF0E0BD01A8E2B0E031
:10BF9A000E94DDD2DB01AE0FBF1F5C96F901349619
:10BFAA00ED93FC93ADEBB7E0E12FF0E0BD01A8E221
:10BFBA00B0E00E94DDD2DB01AE0FBF1F5B96EC91B1
:10BFCA00E07FE860EC931F5F5BCFAFE3B8E00E94CD
:10BFDA001FD4E093C507A0E4B8E00E941FD4E09301
:10BFEA00C807A1E4B8E00E941FD4E093ED07A2E4D9
:10BFFA00B8E00E941FD4E093F00710E01831A0F5D2
:10C00A0000E0A3E4B8E0E12FF0E00E94A6D2AE0F70
:10C01A00BF1F11960E941FD4E03009F001E0A3E48B
:10C02A00B8E0E12FF0E00E94A6D2AE0FBF1F129631
:10C03A000E941FD4E03009F00260A3E4B8E0E12FC7
:10C04A00F0E00E94A6D2AE0FBF1F13960E941FD423
:10C05A00E03009F00460ADE0B8E0E12FF0E0EA0F6B
:10C06A00FB1F00831F5FCACF0E9431D22496089516
:10C07A00BA93AA930E9428D210E0123008F0CDC0D9
:10C08A00ADEBB7E0E12FF0E0BD01A8E2B0E00E941D
:10C09A00DDD2DB01AE0FBF1FEC91E030B1F0ADEBAA
:10C0AA00B7E0E12FF0E0BD01A8E2B0E00E94DDD2E6
:10C0BA00E60FF71F01801280AE81BF811196ED91C4
:10C0CA00FC911197E015F10509F0A5C0EE81FF81F9
:10C0DA000581ADEBB7E0E12FF0E0BD01A8E2B0E0E9
:10C0EA000E94DDD2E60FF71F2681ADEBB7E0E12F04
:10C0FA00F0E0BD01A8E2B0E00E94DDD2E60FF71F32
:10C10A005085ADEBB7E0E12FF0E0BD01A8E2B0E069
:10C11A000E94DDD2E60FF71F37812523A02FA52322
:10C12A00EFEFE327EA232E27E52FE095E0232E2BD6
:10C13A00ADEBB7E0E12FF0E0BD01A8E2B0E00E946C
:10C14A00DDD2E60FF71F2683ADEBB7E0E12FF0E073
:10C15A00BD01A8E2B0E00E94DDD2E60FF71F078317
:10C16A00EE81FF81E681EF700E2FADEBB7E0E12F94
:10C17A00F0E0BD01A8E2B0E00E94DDD2E60FF71FB1
:10C18A002185ADEBB7E0E12FF0E0BD01A8E2B0E018
:10C19A000E94DDD2E60FF71F5385ADEBB7E0E12F22
:10C1AA00F0E0BD01A8E2B0E00E94DDD2E60FF71F81
:10C1BA0032852523A02FA523EFEFE327EA232E2795
:10C1CA00E52FE095E0232E2BADEBB7E0E12FF0E071
:10C1DA00BD01A8E2B0E00E94DDD2E60FF71F218779
:10C1EA00ADEBB7E0E12FF0E0BD01A8E2B0E00E94BC
:10C1FA00DDD2E60FF71F0287ADEBB7E0E12FF0E0E3
:10C20A00BD01A8E2B0E00E94DDD2DB01AE0FBF1F84
:10C21A001396EAE0EC931F5F30CF0E942FD2289644
:10C22A00089524970E9428D2E0916304E07409F4E7
:10C23A00BBC3A091BC07A43038F4E091BC07EF5F00
:10C24A00E093BC07E15003C0E0E0E093BC07A09193
:10C25A00BC07A23008F0A8C3ADEBB7E0E091BC0779
:10C26A00F0E0BD01A8E2B0E00E94DDD2DB01AE0F32
:10C27A00BF1FEC91E03009F497C3ADEBB7E0E09152
:10C28A00BC07F0E0BD01A8E2B0E00E94DDD2DB010C
:10C29A00AE0FBF1F1396AC91A13008F463C0ADEB8B
:10C2AA00B7E0E091BC07F0E0BD01A8E2B0E00E946F
:10C2BA00DDD2DB01AE0FBF1F1396EC91E150EC9378
:10C2CA00ADEBB7E0E091BC07F0E0BD01A8E2B0E059
:10C2DA000E94DDD2DB01AE0FBF1F1396EC91E03056
:10C2EA0009F040C0ADEBB7E0E091BC07F0E0BD015A
:10C2FA00A8E2B0E00E94DDD2DB01AE0FBF1F1696A6
:10C30A00E0E0EC93ADEBB7E0E091BC07F0E0BD01F3
:10C31A00A8E2B0E00E94DDD2DB01AE0FBF1F179684
:10C32A00E0E0EC93ADEBB7E0E091BC07F0E0BD01D3
:10C33A00A8E2B0E00E94DDD2DB01AE0FBF1F199662
:10C34A00E0E0EC93ADEBB7E0E091BC07F0E0BD01B3
:10C35A00A8E2B0E00E94DDD2DB01AE0FBF1F1A9641
:10C36A00E0E0EC93E0E02E2F3E2FE091BC07E030B6
:10C37A0011F450E001C05CE040E011E0103009F433
:10C38A007DC0ADE0B8E0EE27A50FBE1F0C9102FFFD
:10C39A0010C0A3E4B8E0E52FF0E00E94A6D2AE0FE9
:10C3AA00BF1F13960E941FD4AE2F0E942B66E03047
:10C3BA0009F40EC0A3E4B8E0E52FF0E00E94A6D28B
:10C3CA00AE0FBF1F0E941FD4E295E370EE8343C0F5
:10C3DA0001FF10C0A3E4B8E0E52FF0E00E94A6D266
:10C3EA00AE0FBF1F12960E941FD4AE2F0E94713C3F
:10C3FA00E03009F40FC0A3E4B8E0E52FF0E00E94B2
:10C40A00A6D2AE0FBF1F0E941FD4E695E695E37031
:10C41A00EE8321C000FF10C0A3E4B8E0E52FF0E0EE
:10C42A000E94A6D2AE0FBF1F11960E941FD4AE2F34
:10C43A000E94713CE03009F40DC0A3E4B8E0E52F96
:10C44A00F0E00E94A6D2AE0FBF1F0E941FD4E37075
:10C45A00EE8301C010C0EE81F0E0309711F4312B69
:10C46A000AC0E130A0E0FA0729F0E230A0E0FA07BA
:10C47A0011F4312B212B5F5F110F80CFADEBB7E0A9
:10C48A00E091BC07F0E0BD01A8E2B0E00E94DDD275
:10C49A00E60FF71FA0A13A1771F0ADEBB7E0E091F4
:10C4AA00BC07F0E0BD01A8E2B0E00E94DDD2E60FD1
:10C4BA00F71F30A341E0ADEBB7E0E091BC07F0E035
:10C4CA00BD01A8E2B0E00E94DDD2E60FF71FA2A1EB
:10C4DA002A1771F0ADEBB7E0E091BC07F0E0BD01BF
:10C4EA00A8E2B0E00E94DDD2E60FF71F22A341E0E6
:10C4FA00E0E02E2F3E2F11E0103109F47CC0ADE0B0
:10C50A00B8E0EE27A50FBE1F0C9102FF0FC0A3E4EF
:10C51A00B8E0E52FF0E00E94A6D2AE0FBF1F139637
:10C52A000E941FD4AE2F92D3E03009F40EC0A3E4C8
:10C53A00B8E0E52FF0E00E94A6D2AE0FBF1F0E941E
:10C54A001FD4E295E370EE8343C001FF10C0A3E459
:10C55A00B8E0E52FF0E00E94A6D2AE0FBF1F1296F8
:10C56A000E941FD4AE2F0E94713CE03009F40FC024
:10C57A00A3E4B8E0E52FF0E00E94A6D2AE0FBF1FF9
:10C58A000E941FD4E695E695E370EE8321C000FF72
:10C59A0010C0A3E4B8E0E52FF0E00E94A6D2AE0FE7
:10C5AA00BF1F11960E941FD4AE2F0E94713CE0302B
:10C5BA0009F40DC0A3E4B8E0E52FF0E00E94A6D28A
:10C5CA00AE0FBF1F0E941FD4E370EE8301C010C0DC
:10C5DA00EE81F0E0309711F4312B0AC0E130A0E08F
:10C5EA00FA0729F0E230A0E0FA0711F4312B212BE7
:10C5FA005F5F110F81CFADEBB7E0E091BC07F0E0D0
:10C60A00BD01A8E2B0E00E94DDD2E60FF71FA1A1AA
:10C61A003A1771F0ADEBB7E0E091BC07F0E0BD016D
:10C62A00A8E2B0E00E94DDD2E60FF71F31A341E095
:10C63A00ADEBB7E0E091BC07F0E0BD01A8E2B0E0E5
:10C64A000E94DDD2E60FF71FA3A12A1771F0ADEB06
:10C65A00B7E0E091BC07F0E0BD01A8E2B0E00E94BB
:10C66A00DDD2E60FF71F23A341E0403089F4ADEB9A
:10C67A00B7E0E091BC07F0E0BD01A8E2B0E00E949B
:10C68A00DDD2DB01AE0FBF1F1D96AC91A13008F4BD
:10C69A0012C0ADEBB7E0E091BC07F0E0BD01A8E243
:10C6AA00B0E00E94DDD2DB01AE0FBF1F1D96EC91F8
:10C6BA00E150EC9320C0ADEBB7E0E091BC07F0E0AD
:10C6CA00BD01A8E2B0E00E94DDD2DB01AE0FBF1FC0
:10C6DA001D96E0E1EC93ADEBB7E0E091BC07F0E02A
:10C6EA00BD01A8E2B0E00E94DDD2DB01AE0FBF1FA0
:10C6FA005B960E943E09ADEBB7E0E091BC07F0E023
:10C70A00BD01A8E2B0E00E94DDD2DB01AE0FBF1F7F
:10C71A001496AC91A03091F4ADEBB7E0E091BC0770
:10C72A00F0E0BD01A8E2B0E00E94DDD2DB01AE0F6D
:10C73A00BF1F1596AC91A03009F436C140E0E1E084
:10C74A00E987EFE0E887EF83ADEBB7E0E091BC075C
:10C75A00F0E0BD01A8E2B0E00E94DDD2DB01AE0F3D
:10C76A00BF1F1596AC910E94713CE03089F1ABE293
:10C77A00B8E0E091BC07F0E0BD01AAE0B0E00E9499
:10C78A00DDD2DB01AE0FBF1F17960E941FD4E987C7
:10C79A00ABE2B8E0E091BC07F0E0BD01AAE0B0E08E
:10C7AA000E94DDD2DB01AE0FBF1F18960E941FD474
:10C7BA00E887ABE2B8E0E091BC07F0E0BD01AAE08F
:10C7CA00B0E00E94DDD2DB01AE0FBF1F199643C055
:10C7DA00ADEBB7E0E091BC07F0E0BD01A8E2B0E044
:10C7EA000E94DDD2DB01AE0FBF1F1496AC910E94EE
:10C7FA00713CE03099F1ABE2B8E0E091BC07F0E0BF
:10C80A00BD01AAE0B0E00E94DDD2DB01AE0FBF1F7E
:10C81A0013960E941FD4E987ABE2B8E0E091BC0707
:10C82A00F0E0BD01AAE0B0E00E94DDD2DB01AE0F6C
:10C83A00BF1F14960E941FD4E887ABE2B8E0E091CC
:10C84A00BC07F0E0BD01AAE0B0E00E94DDD2DB0146
:10C85A00AE0FBF1F15960E941FD4EF83ADEBB7E052
:10C86A00E091BC07F0E0BD01A8E2B0E00E94DDD291
:10C87A00E60FF71FA489E985EA1781F0ADEBB7E067
:10C88A00E091BC07F0E0BD01A8E2B0E00E94DDD271
:10C89A00E60FF71F7496A985A08341E0ADEBB7E0D8
:10C8AA00E091BC07F0E0BD01A8E2B0E00E94DDD251
:10C8BA00E60FF71FA589E885EA1781F0ADEBB7E027
:10C8CA00E091BC07F0E0BD01A8E2B0E00E94DDD231
:10C8DA00E60FF71F7596A885A08341E0ADEBB7E098
:10C8EA00E091BC07F0E0BD01A8E2B0E00E94DDD211
:10C8FA00E60FF71FA689EF81EA1781F0ADEBB7E0E3
:10C90A00E091BC07F0E0BD01A8E2B0E00E94DDD2F0
:10C91A00E60FF71F7696AF81A08341E0403089F495
:10C92A00ADEBB7E0E091BC07F0E0BD01A8E2B0E0F2
:10C93A000E94DDD2DB01AE0FBF1F1C96AC91A13065
:10C94A0008F412C0ADEBB7E0E091BC07F0E0BD011E
:10C95A00A8E2B0E00E94DDD2DB01AE0FBF1F1C9639
:10C96A00EC91E150EC9320C0ADEBB7E0E091BC074D
:10C97A00F0E0BD01A8E2B0E00E94DDD2DB01AE0F1B
:10C98A00BF1F1C96E0E1EC93ADEBB7E0E091BC076A
:10C99A00F0E0BD01A8E2B0E00E94DDD2DB01AE0FFB
:10C9AA00BF1F1E960E943E090E942FD22A96089502
:10C9BA0008951A931A2FAAE01A9FF001E35FF64F1F
:10C9CA00A081A73B21F4A12F0E94B2873DC1173055
:10C9DA00D0F4103011F42D9815C0113011F41098BC
:10C9EA0011C0123011F42E980DC0133011F4A19811
:10C9FA0009C0143011F4739805C0153011F4A298C7
:10CA0A0001C0A09825C01D30B0F4173011F45F980A
:10CA1A0011C0183011F42F980DC0193011F4139861
:10CA2A0009C01A3011F4749805C01B3011F4149817
:10CA3A0001C075980DC0123158F41D3011F48C984C
:10CA4A0007C01E3011F42C9803C01F3009F48D98CA
:10CA5A00FBC01A931A2F1730D0F4103011F42D9A04
:10CA6A0015C0113011F4109A11C0123011F42E9A17
:10CA7A000DC0133011F4A19A09C0143011F4739A3D
:10CA8A0005C0153011F4A29A01C0A09A25C01D3024
:10CA9A00B0F4173011F45F9A11C0183011F42F9ABC
:10CAAA000DC0193011F4139A09C01A3011F4749A8E
:10CABA0005C01B3011F4149A01C0759A0DC01231C9
:10CACA0058F41D3011F48C9A07C01E3011F42C9AB8
:10CADA0003C01F3009F48D9AB7C01A931A2F173062
:10CAEA00D0F4103011F42D9815C0113011F41098AB
:10CAFA0011C0123011F42E980DC0133011F4A19800
:10CB0A0009C0143011F4739805C0153011F4A298B5
:10CB1A0001C0A09825C01D30B0F4173011F45F98F9
:10CB2A0011C0183011F42F980DC0193011F4139850
:10CB3A0009C01A3011F4749805C01B3011F4149806
:10CB4A0001C075980DC0123158F41D3011F48C983B
:10CB5A0007C01E3011F42C9803C01F3009F48D98B9
:10CB6A0073C01A931A2FEEEAF4E060E070E00E94B4
:10CB7A00B1D3E12FFF27662777270E94B1D384E03C
:10CB8A000E94AFD1289611501730A0F4E12FA1E0EE
:10CB9A000E944AD21E2FA091F608E095EA23E0935C
:10CBAA00F608E091F708E12BE093F708E0E0E0935C
:10CBBA00F30816C01830A0F41850E12FA1E00E9423
:10CBCA004AD21E2FA091F808E095EA23E093F808CC
:10CBDA00E091F908E12BE093F908E0E0E093F4082A
:10CBEA0033C01A931A2FEFEBF4E060E070E00E9472
:10CBFA00B1D3E12FFF27662777270E94B1D384E0BC
:10CC0A000E94AFD128961150173070F4E12FA1E09D
:10CC1A000E944AD21E2FE091F608E12BE093F60813
:10CC2A00E0E0E093F30810C0183070F41850E12FD8
:10CC3A00A1E00E944AD21E2FE091F808E12BE0936E
:10CC4A00F808E0E0E093F408199108950E942AD2C6
:10CC5A003A2F3F3010F03F3108F01EC0E32FEF505B
:10CC6A001E2FAAE01A9FF001E65FF64FE081E470FA
:10CC7A0011F0E1E080C2AAE01A9FF001E65FF64FE8
:10CC8A00E081E295E7700E2F013021F0043011F0B7
:10CC9A00053011F4E1E06FC2A32F0E94E9806BC254
:10CCAA000E942AD2E091FF08EF7EE093FF08EF7D11
:10CCBA00E093FF08E4E1E0930309E091FF08EF7BCA
:10CCCA00E093FF08E0910009EE7FE0930009ED7F11
:10CCDA00E0930009A1E8B9E00E941FD4E093080993
:10CCEA00A2E8B9E00E941FD4E0930909EAE0F9E05A
:10CCFA00FA93EA93E0E0EA93A0EAB0E00E9427CB35
:10CD0A00089A999A9A9A989A0B9A6C9A859AE2B181
:10CD1A00E67EE2B9E5B1EF70E5B95F98EEB1E77C7E
:10CD2A00EEB9E1B3EF7CE1BBE4B3E87FE4BBEFEF3C
:10CD3A00E093F608E093F80810E0103108F008C212
:10CD4A00AAE01A9FF001E35FF64FFF93EF93A5E481
:10CD5A00B1E0E12FF0E0BD01A7E0B0E00E94DDD232
:10CD6A00DB01AE0FBF1F0E941FD4AF91BF91EC939E
:10CD7A00AAE01A9FF001E65FF64FFF93EF93A5E44E
:10CD8A00B1E0E12FF0E0BD01A7E0B0E00E94DDD202
:10CD9A00DB01AE0FBF1F12960E941FD4E07121F56E
:10CDAA00A5E4B1E0E12FF0E0BD01A7E0B0E00E9408
:10CDBA00DDD2DB01AE0FBF1F12960E941FD4E072B4
:10CDCA0099F4A5E4B1E0E12FF0E0BD01A7E0B0E0FD
:10CDDA000E94DDD2DB01AE0FBF1F12960E941FD444
:10CDEA00E07411F4E0E001C0E1E0AF91BF91E170BD
:10CDFA00EE0F0E2EEC91ED7FE029EC93A5E4B1E065
:10CE0A00E12FF0E0BD01A7E0B0E00E94DDD2DB0136
:10CE1A00AE0FBF1F15960E941FD4E07249F0AAE018
:10CE2A001A9FF001E55FF64FDF01EC91E061EC93A8
:10CE3A00A5E4B1E0E12FF0E0BD01A7E0B0E00E9477
:10CE4A00DDD2DB01AE0FBF1F15960E941FD4E0741E
:10CE5A0049F0AAE01A9FF001E55FF64FDF01EC9175
:10CE6A00E062EC93A5E4B1E0E12FF0E0BD01A7E0B8
:10CE7A00B0E00E94DDD2DB01AE0FBF1F12960E9406
:10CE8A001FD4E07859F0183020F4E091FF08E061EF
:10CE9A0003C0E091FF08E062E093FF08A7E6B9E06B
:10CEAA00E12FF0E0F595E795AE0FBF1F0E941FD462
:10CEBA000E2F10FF0DC0E02FE07F49F0AAE01A9F65
:10CECA00F001E65FF64FDF01EC91E068EC930CC0ED
:10CEDA00E02FEF7049F0AAE01A9FF001E65FF64FE3
:10CEEA00DF01EC91E068EC93AAE01A9FF001E35F9E
:10CEFA00F64FA081A63309F03FC0E12FFF2766272E
:10CF0A007727E056FF4F6F4F6BBF3691303148F4A9
:10CF1A00AAE03A9FF001E55FF64FDF01EC91E06489
:10CF2A00EC93E12FF0E0E130A0E0FA0711F4089861
:10CF3A0023C0E330A0E0FA0711F499981DC0E53048
:10CF4A00A0E0FA0711F49A9817C0E630A0E0FA07B1
:10CF5A0011F4989811C0E930A0E0FA0711F40B987F
:10CF6A000BC0EA30A0E0FA0711F46C9805C0EF3064
:10CF7A00A0E0FA0709F48598A5E4B1E0E12FF0E012
:10CF8A00BD01A7E0B0E00E94DDD2DB01AE0FBF1FFA
:10CF9A0015960E941FD4E07409F4D8C0183008F01E
:10CFAA006AC0E12FF0E0309749F4E091F608EE7F8D
:10CFBA00E093F608E091F708E1605AC0E130A0E09A
:10CFCA00FA0749F4E091F608ED7FE093F608E0915C
:10CFDA00F708E2604DC0E230A0E0FA0749F4E091B8
:10CFEA00F608EF7EE093F608E091F708E06140C0AA
:10CFFA00E330A0E0FA0749F4E091F608EF77E0930E
:10D00A00F608E091F708E06833C0E430A0E0FA07D8
:10D01A0049F4E091F608EB7FE093F608E091F7080F
:10D02A00E46026C0E530A0E0FA0749F4E091F6088A
:10D03A00EF7DE093F608E091F708E06219C0E63068
:10D04A00A0E0FA0749F4E091F608EF7BE093F608CE
:10D05A00E091F708E0640CC0E730A0E0FA0751F469
:10D06A00E091F608E77FE093F608E091F708E860B8
:10D07A00E093F7086BC0E12FF0E0E830A0E0FA0790
:10D08A0049F4E091F808EE7FE093F808E091F90896
:10D09A00E1605AC0E930A0E0FA0749F4E091F808E3
:10D0AA00EF77E093F808E091F908E0684DC0EA30BC
:10D0BA00A0E0FA0749F4E091F808EF7BE093F8085A
:10D0CA00E091F908E06440C0EB30A0E0FA0749F4C7
:10D0DA00E091F808EF7DE093F808E091F908E06242
:10D0EA0033C0EC30A0E0FA0749F4E091F808EF7E8B
:10D0FA00E093F808E091F908E06126C0ED30A0E07D
:10D10A00FA0749F4E091F808E77FE093F808E0911C
:10D11A00F908E86019C0EE30A0E0FA0749F4E09196
:10D12A00F808EB7FE093F808E091F908E4600CC096
:10D13A00EF30A0E0FA0751F4E091F808ED7FE093B0
:10D14A00F808E091F908E260E093F9081F5FF5CD6D
:10D15A00E0E0E093F308E093F408E091FF08E0715F
:10D16A0011F0A39A01C0A398E091FF08E07211F0B0
:10D17A00A49A01C0A4980E9431D2249608952797B0
:10D18A000E9428D2E0910109EF73E03100F1A398DF
:10D19A00A498E0910109E07CE0930109E091FE087E
:10D1AA00E770E063E093FE08E2B1E67EE2B9E5B13A
:10D1BA00EF70E5B95F98EEB1E77CEEB9E1B3EF7CC9
:10D1CA00E1BBE4B3E87FE4BBA0E043DCB6C2E09194
:10D1DA00FE08E87FE83008F4B0C2AEEFB8E083E0BA
:10D1EA00EFE10E94E5D3E091FE08E87FE830D1F450
:10D1FA00A1E5B8E0E0910109EF73FF2766277727D9
:10D20A00E054FF4F6F4F6BBFE691F0E0EE0FFF1F48
:10D21A00AE0FBF1FED91FC911197E0930509F093B2
:10D22A0006098BC2E091FE08E87F09F086C2A1E5F3
:10D23A00B8E0E0910109EF73FF2766277727E054EA
:10D24A00FF4F6F4F6BBFE691F0E0EE0FFF1FAE0F7F
:10D25A00BF1FED91FD91A0910509B0910609EA0F52
:10D26A00FB1FE0930509F0930609A0910509B09107
:10D27A000609E0910609F070EA0FFB1FE093050921
:10D28A00F09306090E94B8D2E0930509F0930609C3
:10D29A00E091FE08F0E0E770F070E230A0E0FA07F3
:10D2AA00E1F5A2E3B0E0E0910109EF73F0E0BD011E
:10D2BA00AAE0B0E00E94DDD2DB01AE0FBF1FE09111
:10D2CA000509F09106090E9433D4E0910109EF7330
:10D2DA00FF2766277727E053FF4F6F4F6BBFE69113
:10D2EA00E03061F4EEE4F1E060E070E00E94A0D387
:10D2FA009F01EEE6F1E060E070E00BC0EEE8F1E0DD
:10D30A0060E070E00E94A0D39F01EEEAF1E060E0E5
:10D31A0070E00E94A0D3AF0103C1E330A0E0FA0796
:10D32A00E9F5A2E3B0E0E0910109EF73F0E0BD0195
:10D33A00AAE0B0E00E94DDD2DB01AE0FBF1F129659
:10D34A00E0910509F09106090E9433D4E0910109A0
:10D35A00EF73FF2766277727E053FF4F6F4F6BBFA7
:10D36A00E691E03061F4E0E5F1E060E070E00E940F
:10D37A00A0D39F01E0E7F1E060E070E00BC0E0E9D4
:10D38A00F1E060E070E00E94A0D39F01E0EBF1E0E1
:10D39A0060E070E00E94A0D3AF01C2C0E430A0E018
:10D3AA00FA07E9F5A2E3B0E0E0910109EF73F0E0D2
:10D3BA00BD01AAE0B0E00E94DDD2DB01AE0FBF1FC3
:10D3CA001496E0910509F09106090E9433D4E09180
:10D3DA000109EF73FF2766277727E053FF4F6F4F47
:10D3EA006BBFE691E03061F4E2E5F1E060E070E005
:10D3FA000E94A0D39F01E2E7F1E060E070E00BC079
:10D40A00E2E9F1E060E070E00E94A0D39F01E2EB64
:10D41A00F1E060E070E00E94A0D3AF0181C0E53086
:10D42A00A0E0FA07E9F5A2E3B0E0E0910109EF73A1
:10D43A00F0E0BD01AAE0B0E00E94DDD2DB01AE0F50
:10D44A00BF1F1696E0910509F09106090E9433D490
:10D45A00E0910109EF73FF2766277727E053FF4F13
:10D46A006F4F6BBFE691E03061F4E4E5F1E060E014
:10D47A0070E00E94A0D39F01E4E7F1E060E070E071
:10D48A000BC0E4E9F1E060E070E00E94A0D39F01E4
:10D49A00E4EBF1E060E070E00E94A0D3AF0140C08D
:10D4AA00E630A0E0FA07E1F5A2E3B0E0E091010975
:10D4BA00EF73F0E0BD01AAE0B0E00E94DDD2DB012B
:10D4CA00AE0FBF1F1896E0910509F09106090E9458
:10D4DA0033D4E0910109EF73FF2766277727E053DA
:10D4EA00FF4F6F4F6BBFE691E03061F4E6E5F1E084
:10D4FA0060E070E00E94A0D39F01E6E7F1E060E0FF
:10D50A0070E00BC0E6E9F1E060E070E00E94A0D3B1
:10D51A009F01E6EBF1E060E070E00E94A0D3AF016A
:10D52A00E4EDF4E060E070E00E94B1D3E09101091B
:10D53A00EF73F0E031966F2F660F660B762F0E941D
:10D54A00B1D3E0910509F0910609662777270E9471
:10D55A00B1D388E00E94AFD12C96A0910509B09171
:10D56A000609A217B30718F04A175B0708F402C0A6
:10D57A0011E013C010E0E0910209EC7771F4A2E027
:10D58A00B9E0E0910109EF73EF5FEF71EE0FEE0F73
:10D59A000E2EEC91E378E029EC93A12F0E9493C21E
:10D5AA00E7E0EF83E9EFE887E985E160E987E12FC2
:10D5BA00E170EE0F0E2EE985ED7FE029E987E09113
:10D5CA000109EF73EF5FEF73EE0FEE0F0E2EE98591
:10D5DA00E370E029E987E0910509F0910609EB87F4
:10D5EA00FC87E091FE08F0E0E770F070E230A0E01E
:10D5FA00FA0711F4E1E019C0E330A0E0FA0711F4E8
:10D60A00E2E013C0E430A0E0FA0711F4E3E00DC051
:10D61A00E530A0E0FA0711F4E4E007C0E630A0E044
:10D62A00FA0711F4E5E001C0E0E0EA87E2B1E67E3C
:10D63A00E2B9E5B1EF70E5B95F98EEB1E77CEEB912
:10D64A00E1B3EF7CE1BBE4B3E87FE4BBDE0116960D
:10D65A000E945797E0910109EF73EF3090F4A1E02F
:10D66A00B9E080E0EFE30E94E1D3E091FE08E770C1
:10D67A00E062E093FE08E0910109EF73AE2FE9D969
:10D68A005CC0A2E2B0E00E941FD41E2EE091FE0808
:10D69A00E770E250A1E00E944AD2E129A2E2B0E09A
:10D6AA000E943BD4EFEDF4E060E070E00E94B1D359
:10D6BA0080E00E94AFD12496E0910209EC7791F4C0
:10D6CA00EAEEF4E060E070E00E94B1D380E00E94EC
:10D6DA00AFD12496E091FE08E770E23011F40E947F
:10D6EA002E3614C0EEEEF4E060E070E00E94B1D392
:10D6FA00E0910209E695E695EF71FF2766277727FD
:10D70A000E94B1D384E00E94AFD12896E091FF082D
:10D71A00E07111F0A39A01C0A398E091FF08E072AA
:10D72A0011F0A49A01C0A498E091FE08E87FE16094
:10D73A00E093FE08E6E0E093B70D0E942FD22D9603
:10D74A0008952F970E9428D2E0910109EF73E031E2
:10D75A0000F1E0910109E07CE0930109E091FE0803
:10D76A00E770E062E093FE08A398A498E2B1E67E2F
:10D77A00E2B9E5B1EF70E5B95F98EEB1E77CEEB9D1
:10D78A00E1B3EF7CE1BBE4B3E87FE4BBA0E061D99D
:10D79A0038C2E091FE08E87FE83008F432C2E0912E
:10D7AA000109EF730E2FAEEFB8E083E0EFE10E94BC
:10D7BA00E5D3E091FE08E87FE830D1F40031B8F40F
:10D7CA00A1E5B8E0E02FFF2766277727E054FF4F4F
:10D7DA006F4F6BBFE691F0E0EE0FFF1FAE0FBF1F5A
:10D7EA00ED91FC911197E0930509F093060909C29E
:10D7FA00E091FE08E87F09F004C2E7E0EF83E9EF71
:10D80A00E887E6E0EA87E985E160E987E260E98797
:10D81A00E0910109EF73EF5FEF73EE0FEE0F0E2E3B
:10D82A00E985E370E029E987E0E0EB87EC870031DE
:10D83A0008F0AAC1A1E5B8E0E02FFF2766277727FD
:10D84A00E054FF4F6F4F6BBFE691F0E0EE0FFF1F02
:10D85A00AE0FBF1FED91FD91A0910509B091060988
:10D86A00AE0FBF1FFD010E94B8D29F01A2E3B0E034
:10D87A00E02FF0E0BD01AAE0B0E00E94DDD2DB01BA
:10D88A00AE0FBF1F0E941BD4AF014217530718F0F7
:10D89A0020E030E0E1C0A2E3B0E0E02FF0E0BD011B
:10D8AA00AAE0B0E00E94DDD2DB01AE0FBF1F1296E4
:10D8BA000E941BD4EB8BFC8BE217F30708F1241BA5
:10D8CA00350BF901662777276E2F7F2FE0E0F0E00E
:10D8DA007F936F93FF93EF93EB89FC89E41BF50B1E
:10D8EA0066277727AFE8B2E080E090E00E94E5D2B1
:10D8FA00AF91BF918F919F910E943BD39F01ACC082
:10D90A00A2E3B0E0E02FF0E0BD01AAE0B0E00E949F
:10D91A00DDD2DB01AE0FBF1F14960E941BD4E98B28
:10D92A00FA8BE217F30730F1AB89BC892A1B3B0B50
:10D93A00D90188279927E1E10E9474D27F936F93D6
:10D94A00FF93EF93AB89BC89E989FA89EA1BFB0B40
:10D95A0066277727AFE8B2E080E090E00E94E5D240
:10D96A00AF91BF918F919F910E943BD39F012C59F8
:10D97A003F4F72C0A2E3B0E0E02FF0E0BD01AAE0A1
:10D98A00B0E00E94DDD2DB01AE0FBF1F16960E94E7
:10D99A001BD4EF87F88BE217F30730F1A989BA890C
:10D9AA002A1B3B0BD90188279927E1E10E9474D2EF
:10D9BA007F936F93FF93EF93A989BA89EF85F889CB
:10D9CA00EA1BFB0B66277727A4EBB1E080E090E027
:10D9DA000E94E5D2AF91BF918F919F910E943BD354
:10D9EA009F01245D3E4F38C0A2E3B0E0E02FF0E093
:10D9FA00BD01AAE0B0E00E94DDD2DB01AE0FBF1F7D
:10DA0A0018960E941BD4ED87FE87AF85B8892A1B1A
:10DA1A003B0BD90188279927E3E10E9474D27F93AF
:10DA2A006F93FF93EF93AF85B889ED85FE85EA1B67
:10DA3A00FB0BF695E79566277727ACEEB2E080E018
:10DA4A0090E00E94E5D2AF91BF918F919F910E9481
:10DA5A003BD39F01285A3D4FE3E0F5E060E070E0D8
:10DA6A000E94B1D3E02FF0E031966F2F660F660B5C
:10DA7A00762F0E94B1D3F901662777270E94B8D47E
:10DA8A00DF01CB01E0E0F0E068EC72E40E948FD5A0
:10DA9A000E94B1D388E00E94AFD12C96F6982B87CA
:10DAAA003C8710E0103108F06FC00117B1F5A3EA06
:10DABA00B8E0E12FFF2766277727E055FF4F6F4F22
:10DACA006BBFE691F0E0AE0FBF1FEC91E07421F559
:10DADA00E2E1F5E060E070E00E94B1D3E02FF0E00F
:10DAEA0031966F2F660F660B762F0E94B1D3E12F06
:10DAFA00F0E031966F2F660F660B762F0E94B1D336
:10DB0A0088E00E94AFD12C96E0910209E260E0938E
:10DB1A000209E985ED7FE98735C0A3EAB8E0E12F7C
:10DB2A00FF2766277727E055FF4F6F4F6BBFE691B8
:10DB3A00F0E0AE0FBF1FEC91E07421F1ECE2F5E0EA
:10DB4A0060E070E00E94B1D3E02FF0E031966F2FD1
:10DB5A00660F660B762F0E94B1D3E12FF0E0319663
:10DB6A006F2F660F660B762F0E94B1D388E00E9452
:10DB7A00AFD12C96E0910209E260E0930209E985AF
:10DB8A00ED7FE9871F5F8ECFE0910109EF730E2FBA
:10DB9A00A02F0E947265DE0116960E9457970F30D9
:10DBAA0098F4A1E0B9E080E0EFE30E94E1D3E091CC
:10DBBA000109EF73AE2F0E942E65E091FE08E7700F
:10DBCA00E062E093FE081DC0E9E4F5E060E070E081
:10DBDA000E94B1D380E00E94AFD12496E09102095D
:10DBEA00E695E170A0E0EA17E1E009F0EE27AE2F32
:10DBFA000E9493C2E091FE08E87FE093FE08A39892
:10DC0A00A4980E942FD26596089526970E9428D23A
:10DC1A00E5E5F5E060E070E00E94B1D3ABE1B0E089
:10DC2A000E941BD4662777270E94B1D384E00E9402
:10DC3A00AFD12896ABE1B0E00E941BD4E03CA3E34D
:10DC4A00FA0740F0ABE1B0E00E941BD4E134AFE345
:10DC5A00FA0708F002C021E001C020E0A22F0E94CA
:10DC6A0093C2E6E6F5E060E070E00E94B1D3ADE170
:10DC7A00B0E00E941BD4662777270E94B1D3AFE198
:10DC8A00B0E00E941BD4662777270E94B1D388E0B0
:10DC9A000E94AFD12C96ADE1B0E00E941BD4E53AC8
:10DCAA00A7E1FA07C0F0ADE1B0E00E941BD4E73E5D
:10DCBA00ACE1FA0780F4AFE1B0E00E941BD4E53A88
:10DCCA00A7E1FA0740F0AFE1B0E00E941BD4E73EBB
:10DCDA00ACE1FA0708F002C051E001C050E0A52FFC
:10DCEA000E9493C2EFE7F5E060E070E00E94B1D3D2
:10DCFA00A2E2B0E00E941FD4FF27662777270E947E
:10DD0A00B1D384E00E94AFD12896E0E01E2F3E2FC7
:10DD1A00103108F03EC1E4E9F5E060E070E00E94ED
:10DD2A00B1D3E12FF0E031966F2F660F660B762F95
:10DD3A000E94B1D3A2E3B0E0E12FF0E0BD01AAE076
:10DD4A00B0E00E94DDD2DB01AE0FBF1F0E941BD4E0
:10DD5A00662777270E94B1D3A2E3B0E0E12FF0E073
:10DD6A00BD01AAE0B0E00E94DDD2DB01AE0FBF1F09
:10DD7A0012960E941BD4662777270E94B1D3A2E38A
:10DD8A00B0E0E12FF0E0BD01AAE0B0E00E94DDD2F0
:10DD9A00DB01AE0FBF1F14960E941BD4662777279C
:10DDAA000E94B1D3A2E3B0E0E12FF0E0BD01AAE006
:10DDBA00B0E00E94DDD2DB01AE0FBF1F16960E94B3
:10DDCA001BD4662777270E94B1D3A2E3B0E0E12FE4
:10DDDA00F0E0BD01AAE0B0E00E94DDD2DB01AE0FA7
:10DDEA00BF1F18960E941BD4662777270E94B1D3BB
:10DDFA0088E10E94AFD16C9600E0053008F0B6C009
:10DE0A00E02FF0E0309769F4A2E3B0E0E12FF0E010
:10DE1A00BD01AAE0B0E00E94DDD2DB01AE0FBF1F58
:10DE2A0047C0E130A0E0FA0771F4A2E3B0E0E12FC5
:10DE3A00F0E0BD01AAE0B0E00E94DDD2DB01AE0F46
:10DE4A00BF1F129635C0E230A0E0FA0771F4A2E3D0
:10DE5A00B0E0E12FF0E0BD01AAE0B0E00E94DDD21F
:10DE6A00DB01AE0FBF1F149623C0E330A0E0FA0710
:10DE7A0071F4A2E3B0E0E12FF0E0BD01AAE0B0E066
:10DE8A000E94DDD2DB01AE0FBF1F169611C0E4302F
:10DE9A00A0E0FA0789F4A2E3B0E0E12FF0E0BD01C7
:10DEAA00AAE0B0E00E94DDD2DB01AE0FBF1F1896D8
:10DEBA000E941BD4EE83FF83E12FFF276627772773
:10DECA00E053FF4F6F4F6BBFE691E030C1F4E02F94
:10DEDA00AEE4B1E080E0FF2766277727EE0FFF1F49
:10DEEA00661F771FEA0FFB1F681F791F0E94A0D3C6
:10DEFA00EA87FB87E02FAEE6B1E080E017C0E02FAB
:10DF0A00AEE8B1E080E0FF2766277727EE0FFF1F14
:10DF1A00661F771FEA0FFB1F681F791F0E94A0D395
:10DF2A00EA87FB87E02FAEEAB1E080E0FF276627A9
:10DF3A007727EE0FFF1F661F771FEA0FFB1F681F69
:10DF4A00791F0E94A0D3E887F987EE81FF81AA850D
:10DF5A00BB85EA17FB0738F0E885F985AE81BF81F2
:10DF6A00EA17FB0708F402C00F5F47CFA02FE5E0CE
:10DF7A00EA17E1E009F0EE27AE2F0E9493C20530BE
:10DF8A0010F4303009F003C0E12FEF5F3E2F1F5F1E
:10DF9A00BFCEEFEDF4E060E070E00E94B1D380E024
:10DFAA000E94AFD12496A2E2B0E00E941FD4EF31C2
:10DFBA0081F5203029F4EEEAF5E060E070E022C055
:10DFCA00503029F4E1ECF5E060E070E01BC031303C
:10DFDA00A8F0EEEEF4E060E070E00E94B1D3E091C8
:10DFEA000209E695E695EF71FF27662777270E94D3
:10DFFA00B1D384E00E94AFD128960AC0EAEEF4E0D9
:10E00A0060E070E00E94B1D380E00E94AFD1249614
:10E01A000AC0E3EDF5E060E070E00E94B1D380E071
:10E02A000E94AFD124960E942FD22C9608950E9466
:10E03A002AD20A2F3C81303108F048C0AAE03A9F20
:10E04A00F001E65FF64FDF01EC91E068EC93AAE09D
:10E05A003A9FF001E45FF64FDF01EC91E061EC9347
:10E06A0030FF1CC03695A7E6B9E0EE27A30FBE1F06
:10E07A000E941FD41E2F023019F4E07FE03169F0AC
:10E08A001F70E02FE295E07F1E2BA7E6B9E0EE278E
:10E09A00A30FBE1FE12F0E943BD418C03695A7E6F6
:10E0AA00B9E0EE27A30FBE1F0E941FD41E2F023015
:10E0BA0019F4EF70E13051F0107F102BA7E6B9E0A8
:10E0CA00EE27A30FBE1FE12F0E943BD40E9431D23C
:10E0DA00259608951A930A930A2FE6EEF5E060E072
:10E0EA0070E00E94B1D3E02FFF27662777270E94AE
:10E0FA00B1D384E00E94AFD12896003108F046C01F
:10E10A00AAE00A9FF001E65FF64FDF01EC91EF7794
:10E11A00EC93AAE00A9FF001E45FF64FDF01EC916D
:10E12A00E07FEC9300FF02C01FE001C010EFA7E6FA
:10E13A00B9E0E02FF0E0F595E795AE0FBF1F0E941A
:10E14A001FD4E1230E943BD4AAE00A9FF001E65FB4
:10E15A00F64FE081E17089F00A9FF001E65FF64F21
:10E16A00E081E077E03440F00A9FF001E65FF64F85
:10E17A00DF01EC91EF78EC9309C0AAE00A9FF00165
:10E18A00E65FF64FDF01EC91EF78EC930991199174
:10E19A0008950E9428D2E091FE08E770E23008F064
:10E1AA0012C2A7E2B1E00E941FD4E03079F0A7E2E0
:10E1BA00B1E00E941FD4AE2F0E94713CA0E0B9E0EA
:10E1CA00E1700E2EEC91EE7FE029EC93A8E2B1E02B
:10E1DA000E941FD4E03081F0A8E2B1E00E941FD46F
:10E1EA00AE2F0E94713CA0E0B9E0E170EE0F0E2E56
:10E1FA00EC91ED7FE029EC931FE0103108F0E3C1C8
:10E20A00AAE01A9FF001E35FF64F2081263309F452
:10E21A00D8C1AAE01A9FF001E65FF64FE081E295C5
:10E22A00E7705E2F40E0E091FE08E770E13041F4CC
:10E23A001A9FF001E65FF64FE081E1703E2F73C04E
:10E24A00273B09F4BEC1AAE01A9FF001E65FF64F28
:10E25A00E081E27009F441C0A5E4B1E0E12FF0E009
:10E26A00BD01A7E0B0E00E94DDD2DB01AE0FBF1F07
:10E27A0012960E941FD4E07121F0E0910009E1702A
:10E28A0059F5A5E4B1E0E12FF0E0BD01A7E0B0E067
:10E29A000E94DDD2DB01AE0FBF1F12960E941FD46F
:10E2AA00E07221F0E0910009E270B1F4A5E4B1E076
:10E2BA00E12FF0E0BD01A7E0B0E00E94DDD2DB0172
:10E2CA00AE0FBF1F12960E941FD4E07421F0E09196
:10E2DA00FF08E07809F401C001C002C030E016C0AE
:10E2EA00A22F0E94713C3E2FAAE01A9FF001E55F1F
:10E2FA00F64FE081E07121F0E091B40DE17009F48C
:10E30A0005C0303011F030E001C031E0AAE01A9FB8
:10E31A00F001E65FF64FDF01E32FE1700E2EEC917C
:10E32A00EE7FE029EC93303069F1E52FF0E0309789
:10E33A0021F0E130A0E0FA07D9F4E091FF08E77094
:10E34A00E23098F0E5EFF5E060E070E00E94B1D3CA
:10E35A00E12FF0E031966F2F660F660B762F0E9441
:10E36A00B1D384E00E94AFD1289641E052E009C0BF
:10E37A00E430A0E0FA0721F0E530A0E0FA0709F45A
:10E38A0042E032C0503011F0513009F42DC042E061
:10E39A0050E0AAE01A9FF001E65FF64FDF01EC9128
:10E3AA00EB7FEC93AAE01A9FF001EF5EF64FA0E034
:10E3BA00B0E0A083B183AAE01A9FF001E25FF64FB2
:10E3CA00A0E0A083AAE01A9FF001E45FF64FDF0104
:10E3DA00EC91E07FEC93AAE01A9FF001ED5EF64F14
:10E3EA00DF01EC91EF71EC93E42FF0E0309709F440
:10E3FA0097C0E130A0E0FA0709F06FC0A12F0E9490
:10E40A002E65AAE01A9FF001E55FF64FDF01EC9155
:10E41A00E068EC93AAE01A9FF001E25FF64FA0E0F1
:10E42A00A083AAE01A9FF001E45FF64FDF01EC91A6
:10E43A00E07FEC93AAE01A9FF001ED5EF64FDF0150
:10E44A00EC91E07EEC93AAE01A9FF001E55FF64FAB
:10E45A00E081E07409F440C0E12FFF27662777279F
:10E46A00E056FF4F6F4F6BBF06910A9FF001E65FC0
:10E47A00F64FDF01EC91E160EC93AAE00A9FF0010C
:10E48A00E65FF64FDF01EC91EF78E062EC93AAE0E9
:10E49A000A9FF001E55FF64FDF01EC91E068EC932B
:10E4AA00AAE00A9FF001E25FF64FA0E0A083AAE08B
:10E4BA000A9FF001E45FF64FDF01EC91E07FEC93F5
:10E4CA00AAE00A9FF001ED5EF64FDF01EC91E07ED3
:10E4DA00EC93A02F0E942E6523C0E230A0E0FA0739
:10E4EA00F9F4A12F0E94DE64AAE01A9FF001E55F09
:10E4FA00F64FE081E074A1F0E12FFF276627772726
:10E50A00E056FF4F6F4F6BBF06910A9FF001E65F1F
:10E51A00F64FDF01EC91EE7FEC93A02F0E94DE64B0
:10E52A00E091FF08E770E23050F0AAE01A9FF0018C
:10E53A00E65FF64FE081E295E7705E1709F432C0B4
:10E54A00E1E0F6E060E070E00E94B1D3E12FF0E094
:10E55A0031966F2F660F660B762F0E94B1D3AAE011
:10E56A001A9FF001E65FF64FE081E295E770FF2718
:10E57A00662777270E94B1D3E52FFF2766277727DB
:10E58A000E94B1D3E32FFF27662777270E94B1D3D2
:10E59A00E42FFF27662777270E94B1D384E10E94E0
:10E5AA00AFD16896AAE01A9FF001E65FF64FDF0145
:10E5BA00E52FE770E295E07F0E2EEC91EF78E029E7
:10E5CA00EC9311501ACE0E942FD2269608952797BF
:10E5DA000E942AD28D013B852C85E7E0ED83E9EF85
:10E5EA00EE83EF81E160EF83E32FE170EE0F0E2EF1
:10E5FA00EF81ED7FE029EF83203011F4E7E001C0DD
:10E60A00E8E0E887E22FEF73EE0FEE0F0E2EEF81B0
:10E61A00E370E029EF8309871A87DE0114960E94C6
:10E62A005797A32F0E9493C20E9431D22D96089524
:10E63A0062970E9428D2E091FE08E770E23080F0EB
:10E64A00E091FE08E770E73011F47BD802C00E941F
:10E65A00C468E4E1E09303090E942FD26896089502
:10E66A00E0E0F0E0E0930509F0930609E091020981
:10E67A00E170C9F1E0910209EE7FE0930209E1E25B
:10E68A00F6E060E070E00E94B1D380E00E94AFD172
:10E69A002496E0E0EB8BAB89A03210F5E6E2F6E0D7
:10E6AA0060E070E00E94B1D3EF89FF2766277727E1
:10E6BA000E94B1D3A1E5B8E0EB8DF0E0EE0FFF1FA9
:10E6CA00AE0FBF1FED91FD91662777270E94B1D348
:10E6DA0088E00E94AFD12C96EB89EF5FEB8BDBCF02
:10E6EA00AAE00E949596ABE1B0E00E941BD4ED87A8
:10E6FA00FE87A091BA0DB091BB0DE0917308F0911D
:10E70A0074080E94B8D2EA0FFB1FE093BA0DF09387
:10E71A00BB0DE091B90DEF70E93038F4A9EBBDE01B
:10E72A0080E0EFE00E94E1D36BC0E091B90DE071A7
:10E73A00D1F1E091B90DEF7EE093B90DABE1B0E014
:10E74A00E091BA0DF091BB0D0E9433D4E6E0E0935C
:10E75A00B70DEDE2F6E060E070E00E94B1D3E0911F
:10E76A00BA0DF091BB0D662777270E94B1D384E0DA
:10E77A000E94AFD12896E0E0EA93A091BA0DB09139
:10E78A00BB0DA03CE3E3BE0730F0A134EFE3BE07C4
:10E79A0010F4E1E001C0E0E0EA93A091BA0DB09173
:10E7AA00BB0D15DF22C0E091BA0DF091BB0D6627B3
:10E7BA007727E987FA876B877C87A0EEBEE280E03D
:10E7CA0090E00E94E5D2E987FA876B877C87ED851E
:10E7DA00FE85A985BA858B859C85662777270E9441
:10E7EA003BD3E093BC0DF093BD0DE091B90DE07FF2
:10E7FA00E093B90DE0E0F0E0E093BA0DF093BB0DC1
:10E80A00E0917308F091740866277727E987FA87F9
:10E81A006B877C87ACE2B1E080E090E00E94E5D2B1
:10E82A00E987FA876B877C87ED85FE85F695E795FC
:10E83A00A985BA858B859C8566277727EA0FFB1FF2
:10E84A00681F791FE987FA876B877C87ED85FE85C4
:10E85A00A985BA858B859C85662777270E943BD335
:10E86A00E093BE0DAAE2B1E00E941FD4E13008F4A1
:10E87A00A1C0E091FF08E07809F443C0A091BC0D63
:10E88A00B091BD0DE4E6F0E00E9423D30F01ACE2A3
:10E89A00B1E00E941FD4D001F0E0AE17BF0768F1C3
:10E8AA00ADE2B1E00E941FD4A0910409AE1738F47A
:10E8BA00E0910409EF5FE0930409E1501DC0E7E32A
:10E8CA00F6E060E070E00E94B1D3E091BC0DF091F7
:10E8DA00BD0D662777270E94B1D384E00E94AFD18D
:10E8EA002896A9E00E941A28E091FF08EF77E093A2
:10E8FA00FF08E0E0E093040903C0E0E0E0930409C4
:10E90A0059C0E0E0EA8BABE2B1E00E941FD4EA30E2
:10E91A0058F4AAE2B1E00E941FD4A091BE0DAE172E
:10E92A0010F4E1E0EA8B14C0A091BC0DB091BD0DCA
:10E93A00E4E6F0E00E9423D30F01AAE2B1E00E94CC
:10E94A001FD4D001F0E0AE17BF0710F4E1E0EA8B64
:10E95A00EA89E03061F1ABE2B1E00E941FD4A091F4
:10E96A000409AE1738F4E0910409EF5FE093040953
:10E97A00E1501CC0E7E4F6E060E070E00E94B1D329
:10E98A00E091BE0DFF27662777270E94B1D384E066
:10E99A000E94AFD12896A8E00E941A28E091FF08A9
:10E9AA00E068E093FF08E0E0E093040903C0E0E0D8
:10E9BA00E0930409A091BE0DA83330F5E091030954
:10E9CA00E030E9F4E8E5F6E060E070E00E94B1D3F7
:10E9DA00E091BE0DF0E06F2F660F660B762F0E9456
:10E9EA00B8D4DF01CB01E0E0F0E060E271E40E941C
:10E9FA008FD50E94B1D384E00E94AFD12896EAE075
:10EA0A00E0930309F19A35C0A0910309A13088F176
:10EA1A00E0910309E150E0930309EF5FE0910309F4
:10EA2A00E03039F5E091FF08E07411F1E091FF0858
:10EA3A00EF7BE093FF08E0E7F6E060E070E00E9419
:10EA4A00B1D3E091BE0DF0E06F2F660F660B762F03
:10EA5A000E94B8D4DF01CB01E0E0F0E060E271E4AB
:10EA6A000E948FD50E94B1D384E00E94AFD128962C
:10EA7A00F198A0910309E0E0EA17E1E008F0EE2737
:10EA8A00E88BA0914F08A13008F490C0E0914F089C
:10EA9A00F0E0E130A0E0FA07C1F5E0918108F091D9
:10EAAA00820866277727A8EEB3E080E090E00E940C
:10EABA00E5D27F936F93FF93EF93ADE1B0E00E94AD
:10EACA001BD4AF91BF918F919F91662777270E94A0
:10EADA003BD3E0938508F0938608A0918508B0910E
:10EAEA008608139718F4E0E0F0E00AC0A0918508C0
:10EAFA00B0918608A93FE7E0BE0730F0E8EFF7E0FB
:10EB0A00E0938508F093860851C0E230A0E0FA0746
:10EB1A0021F4E3E0E0934F0849C0E330A0E0FA07AC
:10EB2A0009F044C0E1E0E0934F08E0918108F091D8
:10EB3A008208F695E795ED87FE87ADE1B0E00E9481
:10EB4A0033D4E7E8F6E060E070E00E94B1D3E989E7
:10EB5A00FA89662777270E94B1D384E00E94AFD151
:10EB6A002896E3E0EA93EE85FF85E53AA7E1FA07FE
:10EB7A0040F0AE85BF85A73EECE1BE0710F4E1E0A8
:10EB8A0001C0E0E0EA93AF85B88921DDE1E0E093D6
:10EB9A004F08E6E0E093B70DA0915008A23020F4A8
:10EBAA00F49B02C0F59B01C001C0159AA0915008C0
:10EBBA00A13008F490C0E0915008F0E0E130A0E004
:10EBCA00FA07C1F5A0915108B091520888279927F0
:10EBDA00E8EEF3E060E070E00E94E5D27F936F9385
:10EBEA00FF93EF93AFE1B0E00E941BD4AF91BF91C6
:10EBFA008F919F91662777270E943BD3E0938708DE
:10EC0A00F0938808A0918708B0918808139718F4A0
:10EC1A00E0E0F0E00AC0A0918708B0918808A93F17
:10EC2A00E7E0BE0730F0E8EFF7E0E0938708F093FB
:10EC3A00880851C0E230A0E0FA0721F4E3E0E0934B
:10EC4A00500849C0E330A0E0FA0709F044C0E1E007
:10EC5A00E0935008E0915108F0915208F695E79533
:10EC6A00ED87FE87AFE1B0E00E9433D4E6E0E0939F
:10EC7A00B70DE3E9F6E060E070E00E94B1D3E989FC
:10EC8A00FA89662777270E94B1D384E00E94AFD120
:10EC9A002896E4E0EA93EE85FF85E53AA7E1FA07CC
:10ECAA0040F0AE85BF85A73EECE1BE0710F4E1E077
:10ECBA0001C0E0E0EA93AF85B88989DCE1E0E0933E
:10ECCA005008A0914F08A23020F4F49B02C0F59B93
:10ECDA0001C001C0159AA5E8B9E00E941FD4AE2F61
:10ECEA000E94713CE03061F0E0910009E07439F46F
:10ECFA00E0910009E064E09300090E94A37E05C048
:10ED0A00E0910009EF7BE0930009A0910709A13087
:10ED1A0038F0E0910709E150E0930709EF5F03C07B
:10ED2A00E4E0E0930709EFE0EB8BAB89A03108F050
:10ED3A00F8C6EB89AAE0EA9FF001E55FF64FE081A9
:10ED4A00E07849F0EB89EA9FF001E55FF64FDF01D1
:10ED5A00EC91EF77E1C6EB89AAE0EA9FF001E35F65
:10ED6A00F64FE081E887E0E0EE83EF87A885A633D7
:10ED7A00D9F4EB89FF2766277727E056FF4F6F4FB5
:10ED8A006BBFE691AAE0EA9FF001E65FF64FE081E9
:10ED9A00E170E98BEB89FF2766277727E056FF4F5B
:10EDAA006F4F6BBFE6910AC0EB89AAE0EA9FF001B8
:10EDBA00E65FF64FE081E170E98BEB89AAE0EA9F12
:10EDCA00F001E65FF64FE081E295E770EF83E989AB
:10EDDA00E03009F443C5A1E5B8E0EB89FF276627CF
:10EDEA007727E054FF4F6F4F6BBFE691F0E0EE0FCD
:10EDFA00FF1FAE0FBF1FED91FD91F695E795ED87C9
:10EE0A00FE87A2E3B0E0EB89F0E0BD01AAE0B0E042
:10EE1A000E94DDD2DB01AE0FBF1F0E941BD48F01FF
:10EE2A00AD85BE850A171B0720F0E0E0ED87EE8767
:10EE3A00F1C0A2E3B0E0EB89F0E0BD01AAE0B0E0E6
:10EE4A000E94DDD2DB01AE0FBF1F12960E941BD4B7
:10EE5A009F01AD85BE852A173B0710F1ED85FE851A
:10EE6A00E01BF10BED87FE87662777276E2F7F2F32
:10EE7A00E0E0F0E07F936F93FF93EF93F901E01BDB
:10EE8A00F10B66277727AFE8B2E080E090E00E94B6
:10EE9A00E5D2AF91BF918F919F910E943BD3B8C0A9
:10EEAA00A2E3B0E0EB89F0E0BD01AAE0B0E00E9485
:10EEBA00DDD2DB01AE0FBF1F14960E941BD4AF0137
:10EECA00AD85BE854A175B0738F1ED85FE85E21BE5
:10EEDA00F30BED87FE87AD85BE8588279927E1E18B
:10EEEA000E9474D27F936F93FF93EF93FA01E21B10
:10EEFA00F30B66277727AFE8B2E080E090E00E9444
:10EF0A00E5D2AF91BF918F919F910E943BD3ED873C
:10EF1A00FE87EC59FF4F7CC0A2E3B0E0EB89F0E03A
:10EF2A00BD01AAE0B0E00E94DDD2DB01AE0FBF1F37
:10EF3A0016960E941BD4EE8BFF8BAD85BE85EA1711
:10EF4A00FB0740F1ED85FE85E41BF50BED87FE8797
:10EF5A00AD85BE8588279927E1E10E9474D27F9307
:10EF6A006F93FF93EF93EE89FF89E41BF50B6627F6
:10EF7A007727A4EBB1E080E090E00E94E5D2AF9160
:10EF8A00BF918F919F910E943BD3ED87FE87E45DED
:10EF9A00FE4F3EC0A2E3B0E0EB89F0E0BD01AAE07B
:10EFAA00B0E00E94DDD2DB01AE0FBF1F18960E94AF
:10EFBA001BD4EC8BFD8BAE89BF89ED85FE85EA1BE0
:10EFCA00FB0BED87FE87AD85BE8588279927E3E190
:10EFDA000E9474D27F936F93FF93EF93AE89BF8998
:10EFEA00EC89FD89EA1BFB0BF695E79566277727DF
:10EFFA00ACEEB2E080E090E00E94E5D2AF91BF9122
:10F00A008F919F910E943BD3ED87FE87E85AFD4F6F
:10F01A00ED87FE87A885A73BA1F0A63389F4EB8983
:10F02A00FF2766277727E056FF4F6F4F6BBFE691A2
:10F03A00AAE0EA9FF001E35FF64FA081A73B09F03F
:10F04A006EC0A885A73B19F4EB89EA8B0AC0EB8945
:10F05A00FF2766277727E056FF4F6F4F6BBF069053
:10F06A000A8AA5EBB9E0EA89FF2766277727E052E3
:10F07A00FF4F6F4F6BBFE691F0E00E94A4D2AE0F34
:10F08A00BF1F1196AC91A83C11F4E0E001C0E1E089
:10F09A00EF87AD85BE85A130E0E4BE0720F0E0E051
:10F0AA00F0E4ED87FE87EB89AAE0EA9FF001E15FD1
:10F0BA00F64FCF0160817181EB89AAE0EA9FF001E6
:10F0CA00E15FF64FDF01ED91FD910E94B4D2DF01BD
:10F0DA00FB01EA1BFB0BDC01ED93FC93EB89AAE035
:10F0EA00EA9FF001E15FF64F0F01DF01ED91FD911B
:10F0FA00DF01ED85FE850E94B8D2EA0FFB1FD00121
:10F10A00ED93FC93EB89AAE0EA9FF001E15FF64FE9
:10F11A00DF01ED91FD910E94B8D2ED87FE87E09163
:10F12A000509F0910609AD85BE85EA0FFB1FE0933C
:10F13A000509F0930609EB89AAE0EA9FF001E55F69
:10F14A00F64FE081E074B1F0EB89FF276627772755
:10F15A00E056FF4F6F4F6BBFE691EA9FF001EF5EFB
:10F16A00F64FDF01ED91FD91AD85BE85EA0FFB1FDC
:10F17A00ED87FE87AD85BE85A73FE7E2BE0720F093
:10F18A00E6EFF7E2ED87FE87EB89AAE0EA9FF00156
:10F19A00EF5EF64FAD85BE85A083B183E091FF088F
:10F1AA00E870C9F0EFE9F6E060E070E00E94B1D3E0
:10F1BA00EF89F0E031966F2F660F660B762F0E946B
:10F1CA00B1D3ED89FE89662777270E94B1D388E0FB
:10F1DA000E94AFD12C96EF81F0E0E230A0E0FA076E
:10F1EA0009F0ADC0EB89AAE0EA9FF001E45FF64FAF
:10F1FA00DF01EC91EF7EEC93A889A03039F5A7EDF9
:10F20A00B8E0EB89FF2766277727E054FF4F6F4F57
:10F21A006BBFE691F0E0AE0FBF1FAC91A230A8F42D
:10F22A00AF85A03089F4A9E8B8E0EB89FF27662703
:10F23A007727E055FF4F6F4F6BBFE691F0E0AE0FB7
:10F24A00BF1FEC91E07409F401C001C04FC0EB8903
:10F25A00AAE0EA9FF001E45FF64FE081EF70E43044
:10F26A0058F4EB89EA9FF001E45FF64FDF0180E092
:10F27A00EFE00E94E1D33AC0E5E0EF83E2E0EE83FB
:10F28A00EB89EA93A3E00E941C70EB89AAE0EA9F4B
:10F29A00F001E55FF64FE081EF70EA3098F4EB8910
:10F2AA00EA9FF001E55FF64FDF0180E0EFE00E94A0
:10F2BA00E1D3E6E6EA93EC89E15FEA93A0E0B0E005
:10F2CA000E942328EBEAF6E060E070E00E94B1D3E6
:10F2DA00EF89F0E031966F2F660F660B762F0E944A
:10F2EA00B1D384E00E94AFD1289673C2EB89AAE019
:10F2FA00EA9FF001E25FF64FA081A53058F4EB894E
:10F30A00AAE0EA9FF001E25FF64FDF01EC91EF5FBE
:10F31A00EC9314C0EB89AAE0EA9FF001E25FF64F92
:10F32A00A0E0A083EB89AAE0EA9FF001E45FF64F30
:10F33A00DF01EC91E07FEC93E3E0EF834AC2E33034
:10F34A00A0E0FA0709F045C2A889A03039F5A7ED6F
:10F35A00B8E0EB89FF2766277727E054FF4F6F4F06
:10F36A006BBFE691F0E0AE0FBF1FAC91A230A8F4DC
:10F37A00AF85A03089F4A9E8B8E0EB89FF276627B2
:10F38A007727E055FF4F6F4F6BBFE691F0E0AE0F66
:10F39A00BF1FEC91E07409F401C001C050C0EB89B1
:10F3AA00AAE0EA9FF001E45FF64FE081EF70E330F4
:10F3BA0058F4EB89EA9FF001E45FF64FDF0180E041
:10F3CA00EFE00E94E1D33AC0E5E0EF83E2E0EE83AA
:10F3DA00EB89EA93A3E00E941C70EB89AAE0EA9FFA
:10F3EA00F001E55FF64FE081EF70EA3098F4EB89BF
:10F3FA00EA9FF001E55FF64FDF0180E0EFE00E944F
:10F40A00E1D3E6E6EA93EC89E15FEA93A0E0B0E0B3
:10F41A000E942328EAEBF6E060E070E00E94B1D394
:10F42A00EF89F0E031966F2F660F660B762F0E94F8
:10F43A00B1D384E00E94AFD12896CBC114C0EB8926
:10F44A00AAE0EA9FF001E45FF64FE081EF70E13055
:10F45A0050F0EB89EA9FF001E45FF64FDF0180E0AC
:10F46A00EFE00E94E5D3A885A63309F4B2C1A5E46A
:10F47A00B1E0EB89F0E0BD01A7E0B0E00E94DDD287
:10F48A00DB01AE0FBF1F14960E941BD4FF71ED87DC
:10F49A00FE87EB89AAE0EA9FF001E35FF64FA081BD
:10F4AA00A73B79F4E091FE08E770E13049F4EB8973
:10F4BA00AAE0EA9FF001E65FF64FE081E17009F405
:10F4CA0001C035C0A5EBB9E0EB89FF27662777278E
:10F4DA00E052FF4F6F4F6BBFE691F0E00E94A4D25B
:10F4EA00AE0FBF1F1196EC91EA8BE03029F4ED853F
:10F4FA00FE850E94B6D219C0EA89EC5EEA8BAA8917
:10F50A00A83CA8F4AD85BE8588279927F0E06F2F1F
:10F51A00660F660B762F0E94E5D2DF01CB01E8EC7D
:10F52A00F0E060E070E00E943BD3ED87FE87EB8954
:10F53A00AAE0EA9FF001EF5EF64FDF01ED91FD913F
:10F54A00DF01ED85FE85AE17BF0708F48CC0EB8995
:10F55A00AAE0EA9FF001E65FF64FDF01EC91EB7F4C
:10F56A00EC93EB89AAE0EA9FF001E65FF64FE081AF
:10F57A00E87091F4EB89EA9FF001E65FF64FDF014C
:10F58A00EC91E860EC93EB89AAE0EA9FF001E25F74
:10F59A00F64FA0E0A08366C0EB89AAE0EA9FF001DB
:10F5AA00E25FF64FDF01EC91EF5FEC93EB89AAE0A3
:10F5BA00EA9FF001E25FF64FE081EF93A5E4B1E044
:10F5CA00EB89F0E0BD01A7E0B0E00E94DDD2DB01EB
:10F5DA00AE0FBF1F16960E941FD4AF91AE1708F444
:10F5EA0041C0E4E0EF83E2E0EE83EB89EA93A4E032
:10F5FA000E941C70EB89AAE0EA9FF001E55FF64FD2
:10F60A00E081EF70EA30D8F4EB89EA9FF001E55F18
:10F61A00F64FDF0180E0EFE00E94E1D3E7E6EA93EC
:10F62A00EC89E15FEA93ED89AAE0EA9FF001EF5ED7
:10F63A00F64FDF01ED91FD91DF010E942328E9ECED
:10F64A00F6E060E070E00E94B1D3EF89F0E0319615
:10F65A006F2F660F660B762F0E94B1D384E00E944B
:10F66A00AFD12896B6C0EB89AAE0EA9FF001E65F1F
:10F67A00F64FE081E87089F0EB89EA9FF001E65FD6
:10F68A00F64FDF01EC91E77FEC93EB89AAE0EA9F62
:10F69A00F001E25FF64FA0E0A083A5E4B1E0EB89B8
:10F6AA00F0E0BD01A7E0B0E00E94DDD2DB01AE0FC1
:10F6BA00BF1F11960E941BD4FF70ED87FE87AD8590
:10F6CA00BE8500240A160B0608F083C0EB89AAE05F
:10F6DA00EA9FF001EF5EF64FDF01ED91FD91AD85F6
:10F6EA00BE85EA17FB0708F062C0EB89AAE0EA9F29
:10F6FA00F001E25FF64FE081EF93A5E4B1E0EB8918
:10F70A00F0E0BD01A7E0B0E00E94DDD2DB01AE0F60
:10F71A00BF1F13960E941FD4AF91AE1758F4EB89FE
:10F72A00AAE0EA9FF001E25FF64FDF01EC91EF5F9A
:10F73A00EC933CC0EB89AAE0EA9FF001E65FF64F42
:10F74A00E081E47099F5EB89EA9FF001E65FF64FF4
:10F75A00DF01EC91E460EC93EB89EA93A2E00E946A
:10F76A001C70EB89AAE0EA9FF001E55FF64FE081A1
:10F77A00EF70EA30D8F4EB89EA9FF001E55FF64FC3
:10F78A00DF0180E0EFE00E94E1D3E5E6EA93EC894D
:10F79A00E15FEA93ED89AAE0EA9FF001EF5EF64F96
:10F7AA00DF01ED91FD91DF010E94232812C0EB8950
:10F7BA00AAE0EA9FF001E25FF64FA0E0A083EB899E
:10F7CA00AAE0EA9FF001E65FF64FDF01EC91EB7FDA
:10F7DA00EC93A0910709A03039F4AF81A43020F04E
:10F7EA00A0910809A13008F438C0EB89AAE0EA9F81
:10F7FA00F001ED5EF64FE081EF71AE2FE09108095E
:10F80A00AE1750F4EB89AAE0EA9FF001ED5EF64FDD
:10F81A00DF0180E0EFE11FC0A0910909A03081F06B
:10F82A00EB89AAE0EA9FF001ED5EF64FE081E295EE
:10F83A00EF70E695E770AE2FE0910909AE1768F40C
:10F84A00E0E0EF83EB89AAE0EA9FF001ED5EF64F74
:10F85A00DF0185E0E7E00E94E1D3D0C0EB89AAE0AE
:10F86A00EA9FF001EF5EF64FA0E0B0E0A083B1831B
:10F87A00EB89AAE0EA9FF001E15FF64FA0E0B0E071
:10F88A00A083B183A885A63389F0A5E4B1E0EB890A
:10F89A00F0E0BD01A7E0B0E00E94DDD2DB01AE0FCF
:10F8AA00BF1F12960E941FD4E07809F4A7C0EF8107
:10F8BA00F0E0309709F06CC0E889E03009F09EC0AA
:10F8CA00A3EAB8E0EB89FF2766277727E055FF4FC1
:10F8DA006F4F6BBFE691F0E0AE0FBF1FEC91E07483
:10F8EA0059F4EB89AAE0EA9FF001E45FF64FDF01E1
:10F8FA00EC91E07FEC934BC0EB89AAE0EA9FF00120
:10F90A00E45FF64FE081EF70EF3058F4EB89EA9F3D
:10F91A00F001E45FF64FDF0180E0EFE00E94E1D3FF
:10F92A0036C0E1E0EF83EB89AAE0EA9FF001E45FE9
:10F93A00F64FDF01EC91E07FEC93EB89EA93A1E0CB
:10F94A000E941C70EB89AAE0EA9FF001E55FF64F7E
:10F95A00E081EF70EA30D8F4EB89EA9FF001E55FC5
:10F96A00F64FDF0180E0EFE00E94E1D3E4E6EA939C
:10F97A00EC89E15FEA93ED89AAE0EA9FF001EF5E84
:10F98A00F64FDF01ED91FD91DF010E94232836C079
:10F99A00E130A0E0FA0791F5A3EAB8E0EB89FF2786
:10F9AA0066277727E055FF4F6F4F6BBFE691F0E070
:10F9BA00AE0FBF1FEC91E07409F5EB89AAE0EA9F4C
:10F9CA00F001E45FF64FE081EF70EF3058F4EB8915
:10F9DA00EA9FF001E45FF64FDF0180E0EFE00E946A
:10F9EA00E1D30CC0E0E0EF83EB89AAE0EA9FF001E3
:10F9FA00E45FF64FDF01EC91E07FEC93AE81A23039
:10FA0A00B1F5AB890E94DE64EB89AAE0EA9FF001B6
:10FA1A00E55FF64FE081E07419F4A885A63339F55D
:10FA2A00EB89FF2766277727E056FF4F6F4F6BBF9B
:10FA3A0006900A8AEA89AAE0EA9FF001E65FF64F91
:10FA4A00DF01EC91EE7FEC93EA89AAE0EA9FF001EC
:10FA5A00E65FF64FDF01EF81E770E295E07F0E2E59
:10FA6A00EC91EF78E029EC93AA890E94DE64E09198
:10FA7A00FF08E770E23068F0EB89AAE0EA9FF0013C
:10FA8A00E65FF64FE081E295E770AE2FEF81EA1765
:10FA9A0009F433C0E8EDF6E060E070E00E94B1D30B
:10FAAA00EF89F0E031966F2F660F660B762F0E9472
:10FABA00B1D3EB8DAAE0EA9FF001E65FF64FE08151
:10FACA00E295E770FF27662777270E94B1D3EB8973
:10FADA00FF27662777270E94B1D3E9A1FF27662768
:10FAEA0077270E94B1D3EA8DFF27662777270E94DE
:10FAFA00B1D384E10E94AFD16896EB89AAE0EA9F6C
:10FB0A00F001E65FF64FDF01EF81E770E295E07FF3
:10FB1A000E2EEC91EF78E029EC93EB89E150EB8B18
:10FB2A0004C9E091FF08E87009F475C0E9EFF6E04E
:10FB3A0060E070E00E94B1D380E00E94AFD12496C9
:10FB4A00E0E0EB8BAB89A03108F060C0EB89AAE05A
:10FB5A00EA9FF001E65FF64FE081E17009F452C0D6
:10FB6A00E3E0F7E060E070E00E94B1D3EF89F0E0F3
:10FB7A0031966F2F660F660B762F0E94B1D3A3EAD8
:10FB8A00B8E0EB8DFF2766277727E055FF4F6F4FC9
:10FB9A006BBFE691F0E0AE0FBF1FEC91E07411F07D
:10FBAA00E1E001C0E0E00E94BDD20E94B1D3A1E52C
:10FBBA00B8E0EF8DFF2766277727E054FF4F6F4F96
:10FBCA006BBFE691F0E0EE0FFF1FAE0FBF1FED9186
:10FBDA00FD91662777270E94B1D3EBA1AAE0EA9F9D
:10FBEA00F001EF5EF64FDF01ED91FD91AAE0B0E082
:10FBFA000E94DDD2662777270E94B1D380E10E9456
:10FC0A00AFD16496EB89EF5FEB8B9CCFE091FF0855
:10FC1A00E77FE093FF080E942FD2689608950E941A
:10FC2A0028D2E0E05E2F2E2F3E2F0E2F10E01C3040
:10FC3A0040F5A7E6B9E0EE27A10FBE1F0E941FD428
:10FC4A00E03009F021E0AAE01A9FF001E65FF64FE2
:10FC5A00E081F0E00E94B4D2E770F070E130A0E0F9
:10FC6A00FA0711F451E00BC0E430A0E0FA0711F4EE
:10FC7A0031E005C0E530A0E0FA0709F401E01F5FB2
:10FC8A00D6CF10E0183040F5A3E7B9E0EE27A10F70
:10FC9A00BE1F0E941FD4E03009F021E0AAE01A9F9B
:10FCAA00F001E65FF64FE081F0E00E94B4D2E7701F
:10FCBA00F070E130A0E0FA0711F451E00BC0E43033
:10FCCA00A0E0FA0711F431E005C0E530A0E0FA0738
:10FCDA0009F401E01F5FD6CFA0E0B9E0E02FE170A0
:10FCEA00EE0FEE0F0E2EEC91EB7FE029EC93A0E0E5
:10FCFA00B9E0E32FE170EE0FEE0FEE0F0E2EEC914E
:10FD0A00E77FE029EC93A0E0B9E0E22FE170E29509
:10FD1A00E07FEE0F0E2EEC91EF7DE029EC93A0E050
:10FD2A00B9E0E52FE170E295E07F0E2EEC91EF7ECF
:10FD3A00E029EC930E942FD2269608951A93EDE1BA
:10FD4A00F7E060E070E00E94B1D380E00E94AFD19A
:10FD5A002496ABE7B9E0E0E0F0E00E9433D410E08B
:10FD6A00103108F050C0AAE01A9FF001E55FF64F83
:10FD7A00DF01EC91E07FEC93AAE01A9FF001E65FC5
:10FD8A00F64FDF01EC91EF77EC93AAE01A9FF001AE
:10FD9A00E45FF64FDF01EC91EF7EEC93AAE01A9F45
:10FDAA00F001E45FF64FDF01EC91E07FEC93AAE00B
:10FDBA001A9FF001ED5EF64FDF01EC91EF71EC93C3
:10FDCA00AAE01A9FF001E65FF64FE081F0E00E9498
:10FDDA00B4D2E770F070E130A0E0FA0721F0E43025
:10FDEA00A0E0FA0709F404C0E530A0E0FA0749F4F4
:10FDFA00AAE01A9FF001E65FF64FDF01EC91EF7877
:10FE0A00EC931F5FADCF10E01C3048F4A7E6B9E0D1
:10FE1A00EE27A10FBE1F0E943BD41F5FF5CFD2C1B0
:10FE2A000E942AD23A2F373310F03C3308F064C0CC
:10FE3A0000E010E0103108F05DC0AAE01A9FF0015E
:10FE4A00E35FF64FA0813A1709F052C0AAE01A9F61
:10FE5A00F001E65FF64FE081F0E00E94B4D2E7706D
:10FE6A00F070309761F41A9FF001E65FF64FE08177
:10FE7A00E07811F0003009F001C005E039C0E23045
:10FE8A00A0E0FA0721F0E330A0E0FA07B9F4AAE00B
:10FE9A001A9FF001E65FF64FE081E47011F002E08C
:10FEAA000CC0AAE01A9FF001E65FF64FE081E07805
:10FEBA0011F0003009F001C005E01AC0E130A0E0FD
:10FECA00FA0751F4AAE01A9FF001E65FF64FE081C3
:10FEDA00E07809F001E00CC0E430A0E0FA0711F480
:10FEEA00E4E09BC1E530A0E0FA0711F4E3E095C134
:10FEFA001F5FA0CFE02F91C1E32FEF501E2F1031CB
:10FF0A0008F046C0AAE01A9FF001E65FF64FE081CA
:10FF1A00F0E00E94B4D2E770F070309751F41A9F63
:10FF2A00F001E65FF64FE081E07811F0E5E075C197
:10FF3A0073C1E230A0E0FA0721F0E330A0E0FA074B
:10FF4A00A9F4AAE01A9FF001E65FF64FE081E47097
:10FF5A0011F0E2E062C1AAE01A9FF001E65FF64FF3
:10FF6A00E081E07811F0E5E058C156C1E130A0E047
:10FF7A00FA0711F4E1E051C1E430A0E0FA0711F404
:10FF8A00E4E04BC1E530A0E0FA0711F4E3E045C133
:10FF9A0043C167971A93A5E8B9E0E0E00E943BD411
:10FFAA00A1E8B9E00E943BD4A2E8B9E00E943BD4A0
:10FFBA00A3E8B9E00E943BD4A4E8B9E00E943BD48C
:10FFCA00FE013896FA93EA93E0E0EA93A0E1B0E002
:10FFDA000E9427CBFE013196FA93EA93E0E0EA9376
:10FFEA00A7E0B0E00E9427CBEAE0EC83EF8310E0C1
:06FFFA00103108F058C0B0
:020000021000EC
:0A000000E12FFF2766277727E05362
:10000A00FF4F6F4F6BBFE691E03039F4ED81FE810F
:10001A00E070F07EE062F36006C0ED81FE81E07080
:10002A00F07EE46FF160ED83FE83A5E4B1E0E12F99
:10003A00F0E0BD01A7E0B0E00E94DDD2E60FF71FB5
:10004A00FA93EA93FE013396FA93EA93A7E00E94A1
:10005A00D226FE013896FA93EA93E9E2F7E060E0E5
:10006A0070E00E94B1D3E12FF0E031966F2F660F56
:10007A00660B762F0E94B1D384E00E9474D12A962F
:10008A00E12FF0E0A0E1B8E30E94A2D2EA0FFB1F41
:10009A00FA93EA93FE013A96FA93EA930E94822926
:1000AA00A8951F5FA5CF0E94556618810C94668596
:1000BA001A930A9310E0103108F06DC0E12FF0E0B6
:1000CA00309719F4E5B1E07222C0E130A0E0FA07F6
:1000DA0019F4E2B1E1701BC0E230A0E0FA0719F4AA
:1000EA00E5B1E07414C0E330A0E0FA0719F4E4B310
:1000FA00E2700DC0E430A0E0FA0719F4EEB1E8703E
:10010A0006C0E530A0E0FA0719F4E4B3E4700E2F54
:10011A00E3E3F7E060E070E00E94B1D3E12FF0E0A2
:10012A0031966F2F660F660B762F0E94B1D3AAE025
:10013A001A9FF001E65FF64FE081E295E770FF272C
:10014A00662777270E94B1D31A9FF001E65FF64F20
:10015A00E081E170FF27662777270E94B1D301303B
:10016A0010F0E1E301C0E0E3FF27662777270E944A
:10017A00B1D3AAE01A9FF001EF5EF64FDF01ED91CD
:10018A00FD91662777270E94B1D384E10E94AFD1FF
:10019A0068961F5F90CF0991199108951A9310E0FC
:1001AA00153080F4E12FF0E0E655F64F0F01A5EB8C
:1001BA00B1E0EE27A10FBE1F0E941FD4D001EC931D
:1001CA001F5FEECF199108950E942AD23A2F10E0AC
:1001DA00103110F5AAE01A9FF001E35FF64FA081F3
:1001EA003A17C1F4AAE01A9FF001E65FF64FE081E0
:1001FA00E295E7700E2F1A9FF001E65FF64FE08155
:10020A00E47031F4013021F0043011F0053011F4BA
:10021A00E1E003C01F5FDCCFE0E00E9431D2249608
:10022A00089560971A93FE013196FA93EA93E0E0F3
:10023A00EA93A2E0B0E00E9427CB10E0153080F5E7
:10024A00A5EBB1E0EE27A10FBE1F0E943BD4FE0131
:10025A003196FA93EA93E4E5F7E060E070E00E94F1
:10026A00B1D3E12FF0E031966F2F660F660B762F30
:10027A000E94B1D384E00E9474D12A96E12FF0E063
:10028A00A0E1B9E30E94A2D2EA0FFB1FFA93EA9314
:10029A00FE013396FA93EA930E9482291F5FCECF1A
:1002AA0018816196089562970E9428D2A6E2B1E069
:1002BA000E941FD4E07109F402C4A5E2B1E00E94D1
:1002CA001FD40E2FA6E2B1E00E941FD4EF70ED8B6F
:1002DA0000FF04C0E0919707E17011F501FF04C027
:1002EA00E0919907E170E1F402FF04C0E0919B07F5
:1002FA00E170B1F403FF04C0E0919D07E17081F45D
:10030A00AD89A53060F0ED89F0E03197A7E9B7E053
:10031A00EE0FFF1FAE0FBF1FEC91E17009F412C080
:10032A00A2E3B1E00E941BD4FF70A7EABDE0FF7010
:10033A000F01ED91FD91E070F07FE029F129FE9324
:10034A00EE93BDC3A1E3B1E00E941FD4EE83E03077
:10035A00C1F0AE810E94713CE03091F0A2E3B1E0BD
:10036A000E941BD4FF70A7EABDE0FF700F01ED9158
:10037A00FD91E070F07FE029F129FE93EE939FC38F
:10038A001BC0E091CF03E27021F0A091CE03A1300F
:10039A0008F412C0A2E3B1E00E941BD4FF70A7EADE
:1003AA00BDE0FF700F01ED91FD91E070F07FE02953
:1003BA00F129FE93EE9383C3E091A70DF091A80D66
:1003CA00FF7000240E160F0640F4A7EABDE080E095
:1003DA00EFEFFFE00E940FD472C3A6E2B1E00E94E1
:1003EA001FD4E295EF70E695E170EB8BE03021F0D7
:1003FA00A091F00AA13008F401C061C3E0E0E093E3
:10040A00B30D0E94CE700E94AA36A6E00E941A2856
:10041A00A1E00E944CC0E4E6F7E060E070E00E94D0
:10042A00B1D380E00E94AFD1249616981598E0E0E7
:10043A00E093F508E460E093F508E064E093F508DA
:10044A002898EDB5E093A50DE0E4EEBDEDB5E7FF24
:10045A00FDCFEAE0EEBDEDB5E7FFFDCFE091F5088F
:10046A00EEBDEDB5E7FFFDCF289A07FF3FC0E2B129
:10047A00E67EE2B9E5B1EF70E5B95F98EEB1E77CE7
:10048A00EEB9E1B3EF7CE1BBE4B3E87FE4BBE0E0C3
:10049A00E093F708E093F9082898EDB5E093A50DE5
:1004AA00E2E4EEBDEDB5E7FFFDCFEAE0EEBDEDB566
:1004BA00E7FFFDCFE091F708EEBDEDB5E7FFFDCF11
:1004CA00289A2898EDB5E093A50DE4E4EEBDEDB5C4
:1004DA00E7FFFDCFEAE0EEBDEDB5E7FFFDCFE09126
:1004EA00F908EEBDEDB5E7FFFDCF289AE0E0E98B0C
:1004FA00EA8B00FF0FC0E0919707EC7021F452E0FD
:10050A00E1E0EA8B06C0E0919707EC70E43009F469
:10051A0051E001C050E001FF0FC0E0919907EC7073
:10052A0021F442E0E1E0EA8B06C0E0919907EC7021
:10053A00E43009F441E001C040E002FF11C0E0915B
:10054A009B07EC7029F4E2E0EF8BE1E0E98B07C04E
:10055A00E0919B07EC70E43011F4E1E0EF8B02C00C
:10056A00E0E0EF8B03FF11C0E0919D07EC7029F4E6
:10057A00E2E0EE8BE1E0E98B07C0E0919D07EC70C9
:10058A00E43011F4E1E0EE8B02C0E0E0EE8BE0E053
:10059A00EC8BAD89A53008F1ED89E1501E2FFF27BC
:1005AA0066277727EC56FF4F6F4F6BBFE691E150F6
:1005BA00E8B9E12FA7E9B7E0F0E0EE0FFF1FAE0FB1
:1005CA00BF1FEC91EC70E43029F4ED89EC8BE0E08C
:1005DA00ED8B02C0E1E0EA8B02C0EFE3E8B9E0E0AC
:1005EA00EF87EE87ED87EC87EB8739E120E0E09330
:1005FA00E00DEF83EA87A6E2B1E00E941FD4E295FC
:10060A00EF70E695E695E170E88BA4E3B1E00E940D
:10061A001FD4E887E987E0E0E093D800ECBDA4E1C5
:10062A00B0E00E94F3D5E0E0E093C100E093C2009D
:10063A000E94FA38E1E0E0936900E0E0E4BD0E943C
:10064A006587E0E0E0938000E0938500E093840012
:10065A00E8E1E0938900E9E6E0938800E2E0E6BB9E
:10066A00E0936F00E0E0E0937A00F894E0E8E0932A
:10067A006100E6E0E09361007894EAE0E0938100AB
:10068A00E1E8ECBBE1E0E3BF8895A895E091E00DD5
:10069A00AF81EA0FEF83E0E0E093E00DAF81A53090
:1006AA0088F0EF81E550EF83A4EFB0E1ED91FD9181
:1006BA006D917D91EF5FFF4F6F4F7F4F7E936E93EA
:1006CA00FE93EE93E0E0EA87513089F4669B03C01B
:1006DA00E0E0EF870CC0E889E03039F4AF85A2305A
:1006EA0020F4EF85EF5FEF8702C0E1E0EA8741304F
:1006FA0089F4679B03C0E0E0EE870CC0E889E0302C
:10070A0039F4AE85A23020F4EE85EF5FEE8702C0A1
:10071A00E2E0EA87AF89A13089F4799B0DC0E889C4
:10072A00E03039F4AD85A23020F4ED85EF5FED8736
:10073A0002C0E3E0EA8702C0E0E0ED87AE89A130BB
:10074A0089F47A9B0DC0E889E03039F4AC85A2308F
:10075A0020F4EC85EF5FEC8702C0E4E0EA8702C090
:10076A00E0E0EC87EC89E03089F0359B03C0E0E0FB
:10077A00EB870CC0E889E03039F4AB85A23020F46D
:10078A00EB85EF5FEB8702C0E5E0EA87EA89E030B4
:10079A0019F4E989E030D1F0E0E5ECBDE1E0EDBD26
:1007AA00EA89E03009F0169AE989E03009F0159AE9
:1007BA00AD89A03019F4AC89A03029F088E592E01F
:1007CA000197F1F703C085E88A95F1F7523089F469
:1007DA00669B0DC0E889E03039F4AF85A23020F479
:1007EA00EF85EF5FEF8702C0E1E0EA8702C0E0E051
:1007FA00EF87423089F4679B0DC0E889E03039F40D
:10080A00AE85A23020F4EE85EF5FEE8702C0E2E00B
:10081A00EA8702C0E0E0EE87AF89A23089F4799BCB
:10082A0003C0E0E0ED870CC0E889E03039F4AD851B
:10083A00A23020F4ED85EF5FED8702C0E3E0EA879E
:10084A00AE89A23089F47A9B03C0E0E0EC870CC041
:10085A00E889E03039F4AC85A23020F4EC85EF5F0A
:10086A00EC8702C0E4E0EA87AD89A13088F0359BC5
:10087A000DC0E889E03039F4AB85A23020F4EB856D
:10088A00EF5FEB8702C0E5E0EA8702C0E0E0EB87B2
:10089A00EA89E03009F01698E989E03009F01598FC
:1008AA00313018F131502030F9F020E0E091F508AC
:1008BA00ED7FE093F508E0E5ECBDE1E0EDBD2898B9
:1008CA00EDB5E093A50DE0E4EEBDEDB5E7FFFDCF94
:1008DA00EAE0EEBDEDB5E7FFFDCFE091F508EEBD2C
:1008EA00EDB5E7FFFDCF289A20C031E321E0E09182
:1008FA00F508E260E093F508E0E5ECBDE1E0EDBD66
:10090A002898EDB5E093A50DE0E4EEBDEDB5E7FF5F
:10091A00FDCFEAE0EEBDEDB5E7FFFDCFE091F508CA
:10092A00EEBDEDB5E7FFFDCF289AE0E0ECBDE09122
:10093A00CF03E27029F0E09902C0489901C001C0D2
:10094A0002C0E6E0EA87609902C0E7E0EA87EA8542
:10095A00E03049F0A985A13020F0E985E150E98726
:10096A0001C004C002C0E885E9878CCEF894E0E8AB
:10097A00E0936100E0E0E09361007894EDBBE093DE
:10098A008100E0936F00E1E5ECBDE1E0EDBD719A15
:10099A00E6E0E093C200E8E9E093C100E0E0E0931A
:1009AA00C500E3E0E093C400EDE0E4BDE0E0E093DD
:1009BA00B30DACE6B2E00E941BD4DF010E94CE0464
:1009CA00A0E00E94FF370E94783B07FF02C00E9406
:1009DA00556685D0A2E3B1E00E941BD4FF70A7EA56
:1009EA00BDE0FF700F01ED91FD91E070F07FE0290D
:1009FA00F129FE93EE93AA85A73099F4E091A70D09
:100A0A00F091A80DFF703A9758F4E091A70DF09174
:100A1A00A80DE070F07FEA60E093A70DF093A80DAF
:100A2A0012C0E091A70DF091A80DFF70359758F408
:100A3A00E091A70DF091A80DE070F07FE560E093DA
:100A4A00A70DF093A80DE0E0E093AB0DEFE6F7E019
:100A5A0060E070E00E94B1D3EE85FF276627772712
:100A6A000E94B1D384E00E94AFD12896A0E00E94F0
:100A7A004CC0A7E00E941A280E94B136E889E030EB
:100A8A0029F0AA85A13010F0A53008F018C0EA852F
:100A9A00E150EA87A7E9B7E0F0E0EE0FFF1FAE0FDB
:100AAA00BF1FEC91E160EC93EA85A7E9B7E0F0E0BB
:100ABA00EE0FFF1FAE0FBF1F1196EFE0EC930E94DF
:100ACA002FD268960895EA93EFB7EA93E091E00D82
:100ADA00EF5FE093E00DE991EFBFE9911895229756
:100AEA000E9428D220E050E030E0EAD1EFEAF9E0B3
:100AFA00FA93EA93E0E0EA93AEE3B0E00E9427CBF0
:100B0A0010E0173008F0F7C0E12FFF276627772794
:100B1A00E253FE4F6F4F6BBF4691A5E4B1E0E42F5D
:100B2A00F0E0BD01A7E0B0E00E94DDD2DB01AE0F2C
:100B3A00BF1F0E941FD4E73B09F0DBC0A5EBB9E059
:100B4A00E12FF0E00E94A4D2AE0FBF1FEC91E1604A
:100B5A00EC93113028F0143010F421E001C051E078
:100B6A00ABE3B7E0E12FF0E0BD01A2E2B0E00E9402
:100B7A00DDD2DB01AE0FBF1F0E941FD4E03059F057
:100B8A00A5EBB9E0E12FF0E00E94A4D2AE0FBF1F9F
:100B9A00EC91E260EC93ABE3B7E0E12FF0E0BD014A
:100BAA00A2E2B0E00E94DDD2DB01AE0FBF1F1196B8
:100BBA000E941FD4E03059F0A5EBB9E0E12FF0E034
:100BCA000E94A4D2AE0FBF1FEC91E460EC93ABE39A
:100BDA00B7E0E12FF0E0BD01A2E2B0E00E94DDD271
:100BEA00DB01AE0FBF1F12960E941FD4E03059F0EE
:100BFA00A5EBB9E0E12FF0E00E94A4D2AE0FBF1F2F
:100C0A00EC91E860EC93ABE3B7E0E12FF0E0BD01D3
:100C1A00A2E2B0E00E94DDD2DB01AE0FBF1F139645
:100C2A000E941FD4E03059F0A5EBB9E0E12FF0E0C3
:100C3A000E94A4D2AE0FBF1FEC91E061EC93ABE32C
:100C4A00B7E0E12FF0E0BD01A2E2B0E00E94DDD200
:100C5A00DB01AE0FBF1F14960E941FD4E03059F07B
:100C6A00A5EBB9E0E12FF0E00E94A4D2AE0FBF1FBE
:100C7A00EC91E062EC93ABE3B7E0E12FF0E0BD0169
:100C8A00A2E2B0E00E94DDD2DB01AE0FBF1F1896D0
:100C9A000E9417D430976040704061F031E0A5EBB4
:100CAA00B9E0E12FF0E00E94A4D2AE0FBF1FEC9191
:100CBA00E064EC93ABE3B7E0E12FF0E0BD01A2E220
:100CCA00B0E00E94DDD2DB01AE0FBF1F53960E9437
:100CDA0017D430976040704061F031E0A5EBB9E07D
:100CEA00E12FF0E00E94A4D2AE0FBF1FEC91E068A2
:100CFA00EC931F5F06CFE32FE170EE0F0E2EE0910B
:100D0A00AF09ED7FE029E093AF09E091B509E17001
:100D1A0021F4203011F4503029F0E091AF09E1605C
:100D2A00E093AF09E091B509E170A1F1A6E3B7E05C
:100D3A000E941FD4F0E0309711F4E7E629C0E130B1
:100D4A00A0E0FA0711F4EFE623C0E230A0E0FA07C8
:100D5A0011F4E6E61DC0E330A0E0FA0711F4E5E677
:100D6A0017C0E430A0E0FA0711F4E4E611C0E53058
:100D7A00A0E0FA0711F4E3E60BC0E630A0E0FA07B8
:100D8A0011F4EBE605C0E730A0E0FA0719F4E2E651
:100D9A00E093B009203009F446C0A7E3B7E00E9407
:100DAA001BD4EE83FF83AE81BF81AA3FE0E0BE077A
:100DBA0060F001E0EE81FF8166277727A0E0B4E2C8
:100DCA0084EF90E00E943BD31BC0AE81BF81939712
:100DDA0060F002E0EE81FF8166277727A0E8B4E899
:100DEA008EE190E00E943BD30BC003E0EE81FF81CD
:100DFA0066277727A0E9B0ED83E090E00E945FD3F1
:100E0A00EE83FF83E093B109F093B209EF81E09397
:100E1A008700EE81E0938600E2E0E0938000E02F15
:100E2A00E85EE0938100503009F446C0A9E3B7E0D8
:100E3A000E941BD4EE83FF83AE81BF81AA3FE0E00C
:100E4A00BE0760F001E0EE81FF8166277727A0E008
:100E5A00B4E284EF90E00E943BD31BC0AE81BF8115
:100E6A00939760F002E0EE81FF8166277727A0E87A
:100E7A00B4E88EE190E00E943BD30BC003E0EE8120
:100E8A00FF8166277727A0E9B0ED83E090E00E9412
:100E9A005FD3EE83FF83E093B309F093B409EF8144
:100EAA00E0939700EE81E0939600E2E0E0939000F1
:100EBA00E02FE85EE09391000E942FD228960895D1
:100ECA001A93E0E0E093B000E0918000E370E093D1
:100EDA008000E0919000E370E093900010E01730FA
:100EEA00C0F4A5EBB9E0E12FF0E00E94A4D2AE0F66
:100EFA00BF1F1196E0E0EC93A5EBB9E0E12FF0E01B
:100F0A000E94A4D2AE0FBF1FEC91ED7FEC931F5F3E
:100F1A00E6CF10E01031F8F4AAE01A9FF001E35F7F
:100F2A00F64FA081A73BA9F4AAE01A9FF001E65F59
:100F3A00F64FDF01EC91EE7FEC93AAE01A9FF001E5
:100F4A00E65FF64FDF01EC91EF78EC93A12F0E9458
:100F5A00DE641F5FDFCF199108951A930A930A2F4F
:100F6A00E02FFF2766277727E052FF4F6F4F6BBFAF
:100F7A001691183308F0CCC0A5EBB9E0E12FF0E0E8
:100F8A000E94A4D2AE0FBF1F1196E0E0EC93E12FAE
:100F9A00F0E03097B1F4E0E0E093B000E091B509F9
:100FAA00E47069F0ACE3B7E00E941FD4AE2F0E9450
:100FBA00713CE03011F02C9A01C02C9801C02C9899
:100FCA00A7C0E130A0E0FA07C1F4E0918000EF7316
:100FDA00E0938000E091BD09E47069F0AEE5B7E006
:100FEA000E941FD4AE2F0E94713CE03011F02D9A5E
:100FFA0001C02D9801C02D988BC0E230A0E0FA07FD
:10100A00C1F4E0918000EF7CE0938000E091C50993
:10101A00E47069F0A0E8B7E00E941FD4AE2F0E94E6
:10102A00713CE03011F02E9A01C02E9801C02E9822
:10103A006FC0E330A0E0FA07C1F4E0918000E37FDB
:10104A00E0938000E091CD09E47069F0A2EAB7E08C
:10105A000E941FD4AE2F0E94713CE03011F02F9AEB
:10106A0001C02F9801C02F9853C0E430A0E0FA07BE
:10107A00C1F4E0919000EF73E0939000E091D509FC
:10108A00E47069F0A4ECB7E00E941FD4AE2F0E946E
:10109A00713CE03011F0739A01C0739801C07398E3
:1010AA0037C0E530A0E0FA07C1F4E0919000EF7C88
:1010BA00E0939000E091DD09E47069F0A6EEB7E0F4
:1010CA000E941FD4AE2F0E94713CE03011F0749A36
:1010DA0001C0749801C074981BC0E630A0E0FA07FA
:1010EA00B9F4E0919000E37FE0939000E091E50984
:1010FA00E47069F0A8E0B8E00E941FD4AE2F0E9405
:10110A00713CE03011F0759A01C0759801C075986C
:10111A00099119910895BA93AA9326970E9428D201
:10112A00E091AF09E17021F0E091AF09E27009F4B2
:10113A00CCC1AC85BD85EC91E295E1703E2F303093
:10114A0041F011960E949AD3EE83FF8368877987CC
:10115A0008C0AC85BD851196ED91FC911197EA877F
:10116A00FB8710E0173008F0B0C1A5EBB9E0E12F1A
:10117A00F0E00E94A4D2AE0FBF1FEC91E17009F417
:10118A00A2C1A5EBB9E0E12FF0E00E94A4D2AE0F14
:10119A00BF1FEC91E07409F4C5C03030B1F0ABE385
:1011AA00B7E0E12FF0E0BD01A2E2B0E00E94DDD29B
:1011BA00DB01AE0FBF1F18960E9417D4AE81BF8104
:1011CA00888599850E94D5D213C0ABE3B7E0E12F99
:1011DA00F0E0BD01A2E2B0E00E94DDD2DB01AE0F79
:1011EA00BF1F18960E941BD4AA85BB850E94C3D232
:1011FA002E2F203009F496C0ABE3B7E0E12FF0E0E0
:10120A00BD01A2E2B0E00E94DDD2DB01AE0FBF1F3A
:10121A001C960E941FD4EF700E2F013010F0083078
:10122A0008F046C0AC85BD851596E02FF0E03197F1
:10123A00AE0FBF1F4C915527542F4427ABE3B7E09D
:10124A00E12FF0E0BD01A2E2B0E00E94DDD2DB01B5
:10125A00AE0FBF1F1C960E941FD4E295EF700E2F8F
:10126A00013010F0083008F022C0AC85BD85159613
:10127A00E02FF0E03197AE0FBF1FEC91F0E04E2B5C
:10128A005F2BA5EBB9E0E12FF0E00E94A4D2EA0FB0
:10129A00FB1F43835483A5EBB9E0E12FF0E00E94E2
:1012AA00A4D2AE0FBF1F1296E0915E04EC933AC02F
:1012BA00ABE3B7E0E12FF0E0BD01A2E2B0E00E94AB
:1012CA00DDD2DB01AE0FBF1F1C960E941FD4E29530
:1012DA00EF700E2F013010F0083008F023C0A5EB94
:1012EA00B9E0E12FF0E00E94A4D2EA0FFB1F339687
:1012FA000F01AC85BD851596E02FF0E03197AE0F52
:10130A00BF1FEC91D001F0E0ED93FC93A5EBB9E09F
:10131A00E12FF0E00E94A4D2AE0FBF1F1296E09117
:10132A005E04EC93A5EBB9E0E12FF0E00E94A4D2B1
:10133A00AE0FBF1FEC91E07809F4C5C03030B1F0B0
:10134A00ABE3B7E0E12FF0E0BD01A2E2B0E00E941A
:10135A00DDD2DB01AE0FBF1F53960E9417D4AE81B8
:10136A00BF81888599850E94D5D213C0ABE3B7E0C7
:10137A00E12FF0E0BD01A2E2B0E00E94DDD2DB0184
:10138A00AE0FBF1F53960E941BD4AA85BB850E942D
:10139A00C3D22E2F203009F496C0ABE3B7E0E12F79
:1013AA00F0E0BD01A2E2B0E00E94DDD2DB01AE0FA7
:1013BA00BF1F57960E941FD4EF700E2F013010F0F6
:1013CA00083008F046C0AC85BD851596E02FF0E0E0
:1013DA003197AE0FBF1F4C915527542F4427ABE3CB
:1013EA00B7E0E12FF0E0BD01A2E2B0E00E94DDD259
:1013FA00DB01AE0FBF1F57960E941FD4E295EF7014
:10140A000E2F013010F0083008F022C0AC85BD85DF
:10141A001596E02FF0E03197AE0FBF1FEC91F0E088
:10142A004E2B5F2BA5EBB9E0E12FF0E00E94A4D28E
:10143A00EA0FFB1F46835783A5EBB9E0E12FF0E0E3
:10144A000E94A4D2AE0FBF1F1596E0915E04EC93E2
:10145A003AC0ABE3B7E0E12FF0E0BD01A2E2B0E0B1
:10146A000E94DDD2DB01AE0FBF1F57960E941FD428
:10147A00E295EF700E2F013010F0083008F023C00B
:10148A00A5EBB9E0E12FF0E00E94A4D2EA0FFB1F1E
:10149A0036960F01AC85BD851596E02FF0E03197A1
:1014AA00AE0FBF1FEC91D001F0E0ED93FC93A5EBDA
:1014BA00B9E0E12FF0E00E94A4D2AE0FBF1F15964B
:1014CA00E0915E04EC931F5F4DCE0E942FD22E96C0
:1014DA00089563970E9428D2E091AF09E17029F03C
:1014EA00E091FE08E770E13021F40E942FD269965C
:1014FA000895A7E2B1E00E941FD4E03011F4E0E0C1
:10150A0007C0A7E2B1E00E941FD4AE2F0E94713C2F
:10151A00EB8BA8E2B1E00E941FD4E03011F4E0E0C6
:10152A0007C0A8E2B1E00E941FD4AE2F0E94713C0E
:10153A00EA8BA0E024FCA1E0E1E0EA27E894EE23AC
:10154A0009F0689424F810E0173010F00C94BC9459
:10155A00A5EBB9E0E12FF0E00E94A4D2AE0FBF1FC5
:10156A00EC91E17011F40C94B994E12FFF276627EE
:10157A007727E253FE4F6F4F6BBF06900C8AEC89B8
:10158A00AAE0EA9FF001E65FF64FE081E295E77094
:10159A00E98BA5EBB9E0E12FF0E00E94A4D2AE0FEF
:1015AA00BF1FEC91E270A1F0ABE3B7E0E12FF0E0EE
:1015BA00BD01A2E2B0E00E94DDD2DB01AE0FBF1F87
:1015CA000E941FD4AE2F0E94713CE03009F442C041
:1015DA00EB89E03089F0A5E4B1E0EC89F0E0BD01E7
:1015EA00A7E0B0E00E94DDD2DB01AE0FBF1F12966A
:1015FA000E941FD4E07151F5EA89E03089F0A5E430
:10160A00B1E0EC89F0E0BD01A7E0B0E00E94DDD2D4
:10161A00DB01AE0FBF1F12960E941FD4E072B1F415
:10162A00E0910409E03089F0A5E4B1E0EC89F0E04A
:10163A00BD01A7E0B0E00E94DDD2DB01AE0FBF1F03
:10164A0012960E941FD4E07409F402C030E001C06F
:10165A0031E001C030E050E0303009F451C4A5EB6C
:10166A00B9E0E12FF0E00E94A4D2AE0FBF1FEC91C7
:10167A00E87009F4BDC0ABE3B7E0E12FF0E0BD01CB
:10168A00A2E2B0E00E94DDD2DB01AE0FBF1F1296CC
:10169A000E941FD4E88BA889A83B09F053C0E091A7
:1016AA008508F091860834960E94B6D20E2FA6ECD1
:1016BA00B1E00E941FD4EE8BA7ECB1E00E941FD4C8
:1016CA00ED8BAE89A017E8F50E1758F5A02FBB27AA
:1016DA00EE89F0E0AE1BBF0BAE87BF87ABE3B7E086
:1016EA00E12FF0E0BD01A2E2B0E00E94DDD2DB0111
:1016FA00AE0FBF1F15960E941FD4F0E0AE85BF85BE
:10170A000E94DDD2EE87FF87AD89BB27EE89F0E024
:10171A000E94C1D3EA1BFB0BAE85BF850E9423D36F
:10172A000FC0ABE3B7E0E12FF0E0BD01A2E2B0E009
:10173A000E94DDD2DB01AE0FBF1F15960E941FD497
:10174A005E0F56C0A889A93B09F052C0E0918708EC
:10175A00F091880834960E94B6D20E2FAAECB1E016
:10176A000E941FD4EE8BABECB1E00E941FD4ED8B2C
:10177A00AE89A017E8F50E1758F5A02FBB27EE89FA
:10178A00F0E0AE1BBF0BAE87BF87ABE3B7E0E12F3C
:10179A00F0E0BD01A2E2B0E00E94DDD2DB01AE0FB3
:1017AA00BF1F15960E941FD4F0E0AE85BF850E9428
:1017BA00DDD2EE87FF87AD89BB27EE89F0E00E9474
:1017CA00C1D3EA1BFB0BAE85BF850E9423D30FC092
:1017DA00ABE3B7E0E12FF0E0BD01A2E2B0E00E9486
:1017EA00DDD2DB01AE0FBF1F15960E941FD45E0F1C
:1017FA00A5EBB9E0E12FF0E00E94A4D2AE0FBF1F23
:10180A00EC91E07109F4C0C0ABE3B7E0E12FF0E07E
:10181A00BD01A2E2B0E00E94DDD2DB01AE0FBF1F24
:10182A0013960E941FD4E88BA889A83B09F053C0DD
:10183A00E0918508F091860834960E94B6D20E2F60
:10184A00A6ECB1E00E941FD4EE8BA7ECB1E00E9497
:10185A001FD4ED8BAE89A017E8F50E1758F5A02F07
:10186A00BB27EE89F0E0AE1BBF0BAE87BF87ABE3A9
:10187A00B7E0E12FF0E0BD01A2E2B0E00E94DDD2C4
:10188A00DB01AE0FBF1F16960E941FD4F0E0AE8593
:10189A00BF850E94DDD2EE87FF87AD89BB27EE891F
:1018AA00F0E00E94C1D3EA1BFB0BAE85BF850E9404
:1018BA0023D30FC0ABE3B7E0E12FF0E0BD01A2E212
:1018CA00B0E00E94DDD2DB01AE0FBF1F16960E9468
:1018DA001FD45E0F56C0A889A93B09F052C0E091F7
:1018EA008708F091880834960E94B6D20E2FAAEC87
:1018FA00B1E00E941FD4EE8BABECB1E00E941FD482
:10190A00ED8BAE89A017E8F50E1758F5A02FBB2767
:10191A00EE89F0E0AE1BBF0BAE87BF87ABE3B7E043
:10192A00E12FF0E0BD01A2E2B0E00E94DDD2DB01CE
:10193A00AE0FBF1F16960E941FD4F0E0AE85BF857A
:10194A000E94DDD2EE87FF87AD89BB27EE89F0E0E2
:10195A000E94C1D3EA1BFB0BAE85BF850E9423D32D
:10196A000FC0ABE3B7E0E12FF0E0BD01A2E2B0E0C7
:10197A000E94DDD2DB01AE0FBF1F16960E941FD454
:10198A005E0F553608F054E6A5EBB9E0E12FF0E01A
:10199A000E94A4D2AE0FBF1FEC91E07209F4C0C03E
:1019AA00ABE3B7E0E12FF0E0BD01A2E2B0E00E94B4
:1019BA00DDD2DB01AE0FBF1F14960E941FD4E88B45
:1019CA00A889A83B09F053C0E0918508F0918608E0
:1019DA0034960E94B6D20E2FA6ECB1E00E941FD414
:1019EA00EE8BA7ECB1E00E941FD4ED8BAE89A01755
:1019FA00E8F50E1758F5A02FBB27EE89F0E0AE1BCD
:101A0A00BF0BAE87BF87ABE3B7E0E12FF0E0BD01C4
:101A1A00A2E2B0E00E94DDD2DB01AE0FBF1F179633
:101A2A000E941FD4F0E0AE85BF850E94DDD2EE870A
:101A3A00FF87AD89BB27EE89F0E00E94C1D3EA1B7C
:101A4A00FB0BAE85BF850E9423D30FC0ABE3B7E083
:101A5A00E12FF0E0BD01A2E2B0E00E94DDD2DB019D
:101A6A00AE0FBF1F17960E941FD45E0F56C0A889DB
:101A7A00A93B09F052C0E0918708F0918808349692
:101A8A000E94B6D20E2FAAECB1E00E941FD4EE8BB0
:101A9A00ABECB1E00E941FD4ED8BAE89A017E8F53C
:101AAA000E1758F5A02FBB27EE89F0E0AE1BBF0B2F
:101ABA00AE87BF87ABE3B7E0E12FF0E0BD01A2E25A
:101ACA00B0E00E94DDD2DB01AE0FBF1F17960E9465
:101ADA001FD4F0E0AE85BF850E94DDD2EE87FF8776
:101AEA00AD89BB27EE89F0E00E94C1D3EA1BFB0B4C
:101AFA00AE85BF850E9423D30FC0ABE3B7E0E12FC9
:101B0A00F0E0BD01A2E2B0E00E94DDD2DB01AE0F3F
:101B1A00BF1F17960E941FD45E0F553608F054E671
:101B2A00A5EBB9E0E12FF0E00E94A4D2AE0FBF1FEF
:101B3A00EC91E07461F0A5EBB9E0E12FF0E00E94CE
:101B4A00A4D2AE0FBF1F1296AC91A13008F483C085
:101B5A00A5EBB9E0E12FF0E00E94A4D2AE0FBF1FBF
:101B6A001296EC91E150EC93A5EBB9E0E12FF0E08D
:101B7A000E94A4D2AE0FBF1F1296EC91E03071F40E
:101B8A00A5EBB9E0E12FF0E00E94A4D2AE0FBF1F8F
:101B9A001396E0E0F0E0ED93FC935DC0A5EBB9E0AD
:101BAA00E12FF0E00E94A4D2AE0FBF1F1396ED9171
:101BBA00FD91FF93EF93ABE3B7E0E12FF0E0BD01B6
:101BCA00A2E2B0E00E94DDD2DB01AE0FBF1F1D967C
:101BDA000E941BD4AF91BF91EA23FB23EE87FF87B4
:101BEA00ABE3B7E0E12FF0E0BD01A2E2B0E00E9472
